:020000040800F2
:10300000B8490020716C0008ED640008EF64000806
:10301000F1640008F3640008F56400080000000093
:10302000000000000000000000000000F76400083D
:10303000F964000800000000FB640008FD6400085B
:103040008B6C00088B6C00088B6C0008B536000890
:103050008B6C00088B6C0008C5400008FD40000820
:103060008B6C00088B6C00088B6C00088B6C000864
:103070008B6C00088B6C00088B6C00088B6C000854
:103080008B6C00088B6C00088B6C00088B6C000844
:1030900007D100088B6C00088B6C000835410008D4
:1030A0008B6C00088B6C00088B6C00088B6C000824
:1030B000CB6800088B6C00088B6C00088B6C0008D8
:1030C0008B6C00088B6C00088B6C00088B6C000804
:1030D0008B6C0008FF6400088B660008AB67000873
:1030E0008B6C0008D33600088B6C0008DFF80CD01E
:1030F00010F060FF00480047953C0008B8490020E8
:10310000012080F310887047002080F310887047FA
:1031100008B5002000906A460121452004F02BFBF1
:103120009DF8000000F0020008BD08B500200090E6
:103130006A460121452004F01EFB9DF8000000F0C6
:10314000010008BD38B500246A46012140200094E2
:1031500004F011FBFE4841680A68806882430A60F7
:10316000FC4D6C629DF80000810607D520F020021E
:103170008DF800204021342004F067FAEC7038BD4F
:10318000F8B500266A4601214020009604F0F3FAC3
:10319000F04DEF4C687950B9EF48016809688068D4
:1031A000014204D1287910B9EC48007898B16068E0
:1031B0000168A268914301606E629DF8000081067B
:1031C00007D520F020028DF800204021342004F0A3
:1031D0003CFAEE70F8BDE248C08840F2EE21884229
:1031E00016D29DF8000081060BD440F020028DF825
:1031F00000204021342004F028FA4FF4FA7003F044
:10320000C5FE60680168A268914301606E620EE0CD
:10321000686A0A2806D2401C686260680168A26871
:10322000114303E060680168A268914301600120D6
:10323000E870F8BD38B500246A46012140200094AA
:1032400004F099FA9DF80000C10607D520F010029D
:103250008DF800204021342004F0F7F9BD48847037
:1032600038BD38B500256A4601214020009504F09C
:1032700082FAB84C607910B1B848007820B19DF856
:103280000000C10612D40FE0B348016809688068E5
:103290004FF00105014200D125719DF80000C106E3
:1032A00002D440F0100203E0A57038BD20F01002F7
:1032B0008DF800204021342004F0C7F9F4E710B560
:1032C00001200EF057FF45F255500EF0D9FD0620B3
:1032D0000EF0D9FD40F6FA700EF0D8FD0EF0D9FDD3
:1032E000BDE810400EF0DABD70470CF014BF9D49E8
:1032F0004868026889680A4302609B494868026816
:1033000089680A43026099494868026889688A4363
:10331000026097494868026889688A4302608C495C
:103320004868026889688A4302609249486802686E
:1033300089680A43026090494868026889688A433C
:1033400002608E494868026889680A4302607047D3
:103350001FB5012109200EF087FF4024ADF80C4075
:1033600004208DF80F0003A985480EF03BFC0621D0
:1033700001200EF04DFD00208DF804000C2000947B
:103380008DF8050001248DF8064068460EF06CF8B3
:1033900017208DF8080002208DF809008DF80A002A
:1033A0008DF80B4002A80CF03CFF1FBD1FB501219A
:1033B00009200EF059FF4024ADF80C4004208DF890
:1033C0000F0003A96E480EF00DFC062101200EF03F
:1033D0001FFD009400248DF804400C208DF805009A
:1033E0008DF8064068460EF03FF817208DF808006B
:1033F00002208DF809008DF80A008DF80B4002A814
:103400000CF00FFF1FBD7FB5012109200EF02CFF2E
:103410000224ADF80C4004208DF80F0003A9584891
:103420000EF0E0FB012108460EF0F2FC00208DF8C2
:1034300004000C208DF80500012500948DF806503D
:1034400068460EF011F807208DF808008DF8094045
:103450008DF80A408DF80B5002A80CF0E2FE7FBDFB
:103460007FB5012109200EF0FFFE0224ADF80C40CB
:1034700004208DF80F0003A941480EF0B3FB012191
:1034800008460EF0C5FC00258DF804500C208DF880
:10349000050000948DF8065068460DF0E5FF072002
:1034A0008DF808008DF809408DF80A408DF80B5012
:1034B00002A80CF0B6FE7FBD1FB5012105200EF05D
:1034C000D3FE4FF48074ADF80C4004208DF80F004B
:1034D00003A92C480EF086FB082100200EF098FC72
:1034E00000208DF804000C2000948DF805000124C4
:1034F0008DF8064068460DF0B7FF17208DF80800DC
:1035000002208DF809008DF80A008DF80B4002A802
:103510000CF087FE1FBD1FB5012105200EF0A4FE93
:103520004FF48074ADF80C4004208DF80F0003A90F
:1035300014480EF057FB082100200EF069FC00949F
:1035400000248DF804400C208DF805001CE00000DC
:10355000DC0A0020000000200C0B002034030020B7
:1035600070030020940A0020A00A0020AC0A00206A
:10357000D00A0020C40A0020E80A0020F40A002033
:10358000000C0140000801408DF8064068460DF02F
:103590006BFF17208DF8080002208DF809008DF8C8
:1035A0000A008DF80B4002A80CF03BFE1FBD1FB5B2
:1035B000012105200EF058FE0124ADF80C40042036
:1035C0008DF80F0003A9FC480EF00CFB0021084603
:1035D0000EF01EFC00208DF804000C208DF8050074
:1035E00000948DF8064068460DF03EFF06208DF8E9
:1035F000080002208DF809008DF80A008DF80B40B4
:1036000002A80CF00EFE1FBD1FB5012105200EF013
:103610002BFE0124ADF80C4004208DF80F0003A907
:10362000E5480EF0DFFA002108460EF0F1FB0094A9
:1036300000248DF804400C208DF805008DF806401C
:1036400068460DF011FF06208DF8080002208DF865
:1036500009008DF80A008DF80B4002A80CF0E1FD7E
:103660001FBD10B5FFF7A3FFFFF726FFFFF7CBFE47
:10367000BDE810406CE610B5FFF74DFFFFF7F0FE18
:10368000FFF794FEBDE81040BEE708B54FF4C060F8
:103690000CF0C2FD03208DF8000002208DF801001F
:1036A00000208DF8020001208DF8030068460CF020
:1036B000B8FD08BD10B501200EF0C4FE20B10120F8
:1036C0000EF0D0FE0EF090FEBDE8104003200EF08C
:1036D000C9BE10B54FF400300DF03DFF02200EF0D2
:1036E000B1FE10B103200EF0BDFE0EF07DFE0020F5
:1036F0000EF047FE0EF078FEB048C079002803D0E7
:10370000BDE810400CF0E8BA10BD10B5FFF71AFD87
:10371000FFF7EDFD002007F0BAFD012007F0B7FD2F
:10372000022007F0B4FD4FF49674204603F02EFCFF
:10373000FFF797FF204603F029FC012108070EF050
:10374000A0FD4FF0E020016921F00101016102219B
:10375000BDE8104000200EF0D1BB012080F313889B
:1037600097480168974A01F4E06111430160BFF393
:103770004F8FFEE72DE9F0419348904C0025B0F8BB
:10378000400098BB9149924AB1F8A2101288914228
:103790002CD3A08A0C2803D2401CA082BDE8F08163
:1037A000002007F074FD012007F071FD022007F0F2
:1037B0006EFD8848A58241680A68806882430A6075
:1037C00041F28834204603F0E1FB83494A681068DF
:1037D00089688843106081494868026889688A431B
:1037E00002602046BDE8F04103F0D0BB7C49098867
:1037F00051BB48BB207A38BB7A480368D3F800C075
:1038000082686E48784FDFF8E481408A1CEA020F34
:1038100000F101014FF0010689B20ED1B0F5347FFD
:1038200010D373A010F0E6FCE671752007F02FFDB1
:103830006582C8F80070FFF790FF1B68134203D041
:103840000228F1D2618200E06582A582A6E72DE917
:10385000F04F5E496B484FF0000BB1F88040B1F873
:103860009820944203D3028C42F001020284028821
:10387000944203D8028C22F001020284B1F89A200B
:10388000944203D8028C42F002020284428894429D
:1038900003D3028C22F0020202844C4B00225A4DC8
:1038A0004FF0010ADFF8649193F8D230B1F89C70C0
:1038B000B1F89E600CE000BF39F812C0BC4501D9D8
:1038C00005F802A0B44501D205F802B0521CD2B2EC
:1038D0009342F1D80026324604E0AF5C521C3E44CD
:1038E000F6B2D2B29342F8D8028C16B142F004027A
:1038F00001E022F004020284434D00222035B1F899
:10390000A2C0D046B1F8A4700CE000BF39F8126034
:10391000664501D205F80280BE4201D905F802B021
:10392000521CD2B29342F1D80026324604E0AF5C7A
:10393000521C3E44F6B2D2B29342F8D8028C16B171
:1039400042F0080201E022F008020284304A204BD3
:1039500012881B88D21AB1F8A8309A4203DB028C75
:1039600042F010020284028A944203D8028C22F0B0
:1039700010020284B1F8AA2002EBC20303EB021486
:10398000174A1388028CB3EB840F02D342F0200253
:1039900001E022F0200202840B4AB1F8AE50B2F8E6
:1039A000404005EBC50606EB0515B4EB850F048C0E
:1039B00030D344F040042FE0000801400000002014
:1039C0000CED00E00400FA0554140020E00E002085
:1039D000A4000020D00A0020F40A0020880A002059
:1039E0009A0000200C0B00200030000808ED00E0D9
:1039F00053705F505F536C656570315F4F6E0D0A99
:103A000000000000AC130020C803002000090020C3
:103A1000A200002024F04004048491F8314104EB1A
:103A20004405C5EBC414B3EBC40F038C02D343F0BD
:103A3000800301E023F080030384B2F94630B1F83B
:103A4000B840A34203DB048C44F480740484B1F8CE
:103A5000BA40A34203DC038C23F480730384B2F9DD
:103A60004220B1F8BC309A4203DB038C43F400736C
:103A70000384B1F8BE309A4203DC028C22F4007257
:103A80000284FD4AB2F90030FC4AB2F900209342A8
:103A900001DD9C1A00E0D41AB1F8C05024B2A5424E
:103AA00003DC058C45F480650584C58AA54203DBEB
:103AB000048C24F480640484B1F8C2409C4201DD8B
:103AC000944203DC048C44F400640484B1F8C440E0
:103AD0009C4205DB944203DB048C24F400640484E0
:103AE000B1F8C6409C4201DD944203DC048C44F4EE
:103AF00080540484B1F8C8409C4205DB944203DB47
:103B0000048C24F480540484B1F9CA409C4201DA44
:103B1000944203DB048C44F400540484B1F9CC4097
:103B20009C4205DC944203DC048C24F4005404849D
:103B3000B1F9CE409C4201DA944203DB048C44F498
:103B400080440484B1F9D0409C4205DC944203DCFB
:103B5000028C22F480420284B1F89210C904018CD4
:103B600002D541F4004101E0C1F30E01018488B2A5
:103B7000BDE8F08F2DE9F043C448C34B0026314621
:103B8000BF4D4FF00108BF4C93F8D220B0F804C0ED
:103B9000C788B1460CE000BF34F81160664501D912
:103BA00005F80180BE4201D205F80190491CC9B256
:103BB0008A42F1D80026314604E06F5C491C3E443D
:103BC000F6B2C9B28A42F8D8B049498C16B141F070
:103BD000040101E021F004014184A94D00212035B8
:103BE0004689C44687890BE034F81180B04501D27C
:103BF00005F801C0B84501D905F80190491CC9B2C2
:103C00008A42F1D80024214604E06E5C491C344409
:103C1000E4B2C9B28A42F8D8418C14B141F008012B
:103C200001E021F008014184B3F8361101EBC10233
:103C300002EB0111964A1288B2EB810F418C02D33C
:103C400041F0200101E021F0200141849149428AA4
:103C5000B1F8401002EBC20404EB0212B1EB820F88
:103C6000418C02D341F0400101E021F04001418448
:103C7000B3F892108904418C05D541F40041418488
:103C800041F4004102E0C1F30E014184418488B255
:103C9000BDE8F0831CB5012700268048DFF8F8B1A5
:103CA00001963546C0F800B0DFF8F4A17D48B9466A
:103CB0008AF80C70C846544606700CF02CFA88F34B
:103CC0001088E583258465737748A5732570057092
:103CD0007648057003F036F902F0DCFF03F01AFABB
:103CE0000BF0F0FE03F0EBF808F0E1FF04F050F801
:103CF0000AF12800416810F02BFA03F087FB06F068
:103D0000A3F96148A0F8345184F80B804FF47A7815
:103D1000404603F03BF901AA0121402003F02BFDAE
:103D20009DF80400624C010701D5400611D460687B
:103D30000168A26811430160642003F027F978222A
:103D40004021342003F081FC60680168A26891433F
:103D5000016001AA0121002003F00DFD9DF804007F
:103D6000702811D060680168A26811430160642066
:103D700003F00CF970220021342003F066FC606827
:103D80000168A2689143016064214A4803F016F972
:103D90004FF4FA71484803F011F94FF4487147485D
:103DA00003F00CF94146464803F008F94FF4FA6174
:103DB000444803F003F941F28831434803F0FEF828
:103DC0004EF66021414803F0F9F841A010F012FAD4
:103DD00054469AF80C1040A010F00CFA2F49658256
:103DE000A582C1F800B0FFF746FC85F31088E079A2
:103DF00008B1FFF78AFCFFF762FA002080F3108811
:103E0000DFF8E8B04FF4257AE0790028FCD12448A7
:103E1000283010F0B1F90EF03CF8264803F0D5F840
:103E200048B30BF063FBFFF712FD10B9FFF7A2FEDA
:103E300008B3FFF70CFDDFF8B880B8F87E108842B1
:103E400005D1FFF797FEB8F8801088425AD0FFF7E7
:103E5000FEFCA8F87E00FFF78DFEA8F8800098F819
:103E6000830008F017F898F883001E2842D2401CFF
:103E700088F8830040E045E0B6000020B80000204C
:103E80000804002000090020E00E0020AC130020F0
:103E90009A000020541400200030000808ED00E0D3
:103EA000000000208E000020400100204101002081
:103EB0007C0A0020400900204C09002058090020FD
:103EC00064090020700900207C0900208809002076
:103ED0003132330D0A000000466972737453746105
:103EE0007274203D2025640D0A000000180B00208C
:103EF000D013002088F88350742007F0C8F971208F
:103F000007F0C5F9A34803F060F830B32079A0B1F9
:103F1000022802D0012808D00FE09F4801680968F4
:103F20008068014209D1257107E09B480168096852
:103F30008068014201D0022020719848007810B9B1
:103F4000012003F05BFF00F0FFF90BF083FB0BF0A7
:103F5000ADFB0BF09FFC0BF0F2FC914803F035F841
:103F600008B10BF053FE8F4803F02FF808B10BF0A7
:103F700074FC8D4803F029F8002844D027B10027AD
:103F8000607A012802D00CE00127F9E7A07A401CF2
:103F9000C0B2A072052801D3A5726572834803F0F0
:103FA0005BF8607958B1A079052802D2401CA07155
:103FB00005E07F48B0F8400000B96571A571DBF8F5
:103FC00000201368DBF808100B4208D17848B0F8DD
:103FD000400020B97748008808B984F80590106837
:103FE000084201D074A000E077A010F003F9DFF8D8
:103FF000E8817AA0B8F8201010F0FCF8B8F8221088
:104000007EA010F0F7F8854802F0DFFF78B1208A33
:10401000761C401CF6B280B22082062E00D3002609
:104020003C2802D37E4981F80090FFF7A3FB7D482E
:1040300002F0CBFF10B96078012836D1208B401CEC
:104040002083608B401C6083A08B401CA083E08A8F
:10405000401C80B2E0823C2802D26078012806D160
:10406000E582657084F80990504802F0F5FF208BD6
:10407000D046404506D32583322007F008F9712049
:1040800007F005F9608B404500D36583A08B40F2B3
:104090009321884209D3A583022007F0F8F8002075
:1040A00007F0F5F8012007F0F2F805F02FFF05F012
:1040B000A8FF05F016FF5C48016900910FC80AF0DF
:1040C0008DFEA1E601200DF046FA38483038C1795E
:1040D00001290BD10021C171752007F0D8F800210A
:1040E0004FF080500EF0CDF8FFF7C5FA504D4F4C11
:1040F0002C600CF010F82C60FFF72FFB02200DF065
:104100002AFA2A483038C17901290BD10021C1711E
:10411000752007F0BCF800214FF080500EF0B1F888
:10412000FFF7A9FA424D414C2C600BF0F4FF2C60D4
:10413000FFF713FB40200DF0FDF910B140200DF00A
:104140000AFA4FF4807420460DF0F4F910B12046BD
:104150000DF001FA40200DF0FEF920460DF0FBF9BC
:1041600012483038C17901290BD10021C171752065
:1041700007F08DF800214FF080500EF082F8FFF725
:104180007AFA2B4D294C2C600BF0C5FF2C60FFF701
:10419000E4FA00004C0900200C0B0020D50200209E
:1041A0005809002064090020700900203000002018
:1041B000541400209A0000204348475F444554208F
:1041C0003D20310D0A0000004348475F444554201C
:1041D0003D20300D0A000000AC13002050745F44F5
:1041E0006174612E50727074656374696F6E315FB3
:1041F000466C67203D2025640D0A000050745F4422
:104200006174612E50727074656374696F6E325F91
:10421000466C67203D2025640D0A00007C090020C3
:104220008800002088090020041B002000300008BE
:1042300008ED00E010B50FF0BAFCFC490FF0DCFA15
:104240000FF01EFD10F0BCFC0FF02DFDF8490FF033
:10425000D3FAF8490FF046FA01464FF07E500FF0BE
:10426000CBFAF5490FF090FAF44900F1FF428A4287
:1042700001D8490213E0F24A0244B2F5000F01D21C
:10428000F0490CE0F04A0244B2F5A00F02D24FF020
:10429000814104E0ED4A0244B2F5401F01D20FF023
:1042A00073FABDE810400FF0A5BC70B5E849E94AC3
:1042B000B1F8424040F6E441B2F89E508C4201D23F
:1042C0004FF005000CD3A5420AD3A4F6B2400FF07C
:1042D00073FCE14AE14B0FF0F2FB0FF0B8FCC0B207
:1042E000A54200D2642070BDD949B1F84210A1F5B1
:1042F0002F62C82A00D80520A1F6B932632A00D857
:104300001420A1F61D42632A00D82820A1F681427C
:10431000632A00D83C20CF4A40F6E4439942B2F8E1
:104320009E2002D98A4200D350208A4200D26420C3
:10433000704708B5002000906A460121452003F02F
:104340001AFA9DF8000008BD2DE9F04FABB000202F
:10435000064601904FF01009402105A80FF0B7F96B
:10436000402115A80FF0B3F9BA48DFF8F4B20124E0
:1043700090F80B11BB48B64D0129B0F86C70B548E8
:10438000B0F8DA0028901AD1380416D428980FF023
:1043900024FC00225B460FF020FB80468A4638460C
:1043A0000FF01BFC0022B04B0FF017FB42465346A8
:1043B0000FF085FB0FF077FCA86785F83840DFF831
:1043C000AC8298F81C0001281DD1380419D5D8F802
:1043D00018000FF002FC00225B460FF0FEFA824646
:1043E0004FF6FF708B46C01B0FF0F7FB00229E4B71
:1043F0000FF0F3FA52465B460FF061FB0FF053FCEF
:10440000E86785F83940DFF84CA299A028990FF0A9
:10441000F1FEA86F0FF034FC02460B4697A00FF098
:10442000E9FE474699A0D8F818100FF0E3FEE86FB0
:104430000FF026FC02460B4698A00FF0DBFE9AF820
:104440000B014FF0000840B995F83800012804D15D
:10445000332006F01CFF85F83880387FBA4640B913
:1044600095F83900012804D16F2006F010FF85F877
:1044700039807C4F97F8330000F07F000FF0ADFBE0
:104480008B4A8C4B0FF0A9FA4FF033328A4B0FF066
:10449000FDF90FF008FC0390A5F84890A88F1028AC
:1044A00005D06B4985F815808031C1F80080A5F8EA
:1044B0003C9000206B4901EB4001401CB1F84C10CE
:1044C000C0B20E444845F5D330460FF086FB7B4A18
:1044D0007B4B0FF0F4FA00227A4B0FF0F0FA0FF05A
:1044E000B6FB794986B22F46CE86A5F84A60019878
:1044F00009EB000528460D870FF06FFB8346304619
:1045000025910FF06AFB00226E4B0FF066FA5A46B7
:10451000259B0FF0D4FA0FF09AFBA7F846004D4800
:10452000D0F80C010FF059FB06468B46386E0FF0A1
:10453000A7FB32465B460FF0C2FA0022634B0FF036
:104540004CFA0FF084FB86B2314661A00FF052FEA8
:104550000A20B6FBF0F100FB116000284FF00A00C2
:10456000B6FBF0F0394600D0401CB8720846897A94
:10457000642901D964218172354887F80B80464649
:10458000817A5148DFF8CC80BB464187D8F80C01CE
:10459000474648430FF021FB0022504B0FF08FFAA3
:1045A00000224E4B0FF019FA0FF051FB4649888755
:1045B000B7F886000F21B0FBF1F0C0B2C0F1640083
:1045C000C0B20FF00AFB0022444B0FF078FA002231
:1045D000434B0FF0FFF90FF066FB1D49C8663A48E0
:1045E000C08E00EB800041003EA00FF003FE1D488E
:1045F0004049B0F86C00009000047FD53E48007838
:104600000028DBF87C007BD00FF0C4F80FF038FBFB
:1046100026900F4600984FF6FF71081A0FF0DDFA4A
:104620000022114B0FF0D9F9269A7DE000401C467C
:1046300000B056450FCF5B3B339388430000A0404A
:10464000FFFFDF3E00004040FFFF5F3EFFFF0F3EE9
:1046500060000020E00E0020CDCCCCCCCCCC2140A2
:1046600080F7D440300B002000006940AC130020DC
:10467000437572724A5A3A25640D0A004375727284
:104680005F5265733A256C660D0A00004F757443DE
:104690007572724A5A3A25640D0A000043757272A7
:1046A0005F4F75745F5265733A256C660D0A0000A2
:1046B0009A9999999999A93F33331B40E926310872
:1046C000AC9C1940000024405414002000408F404E
:1046D000536F635F583A25640D0A0000000059408B
:1046E0000000F03FD7DCB5E7D1B925646D560D0A5F
:1046F0000000000000BCA746CE0200208AE0FFE7D1
:104700000FF048F80FF0BCFA04900F4600984FF6EF
:10471000FF71081AFE49098808440FF05EFA00226A
:10472000FC4B0FF05AF9049A3B460FF0C8F90022EF
:10473000F94B0FF0C4F90FF08AFAABF83A00F748DA
:104740000670BBF83A105846142901D84687867778
:10475000BBF83A005F4600EB80004100F0A00FF08C
:1047600049FDF248A0F84060A7F84060387DE0BB02
:10477000788F2790142840D9B87F401CC0B2B877F2
:104780007D2801D90320B877B8F8AA00143000EBCF
:10479000C00101EB00112798B0EB810F2DD8386FC5
:1047A0000FF06EFA04912690F96E786E0EF09AFF73
:1047B0000FF066FA0090259127980FF00EFA00226C
:1047C000DB4B0FF07CF9DB4ADB4B0FF006F9259B46
:1047D000009A0FF002F9049B269A0FF0FEF8CDE93B
:1047E0002510386E0FF04CFA00E006E0DDE92532C6
:1047F0000FF0EDF80FF057FA3866396E384611F1C0
:10480000FF4F00D30666386E0FF03AFA02460B46A9
:10481000CAA089E0ABF83A605F46DBF878000EF09A
:10482000B9FF0FF02DFACDE9251000980FF0D5F95A
:104830000022B84B0FF0D1F8DDE925320FF03FF937
:104840000022B54B0FF03BF90FF001FA81B2B748E7
:104850003229A0F8401007D8BC49A0F840607E7506
:104860000E60A7F84060FE77B048B0F8400000EB5B
:1048700080004100B6A00FF0BDFCF87CF0BBAB4857
:10488000B0F840000490322848D9F87F401CC0B2EC
:10489000F8777D2801D90320F877B8F8AE0004999D
:1048A000143000EBC00202EB0010B1EB800F35D8E2
:1048B000A6483E707E700021C0E9061187F8366078
:1048C000386F0FF0DDF900912890D7E91A010EF04A
:1048D00009FF0FF0D5F9CDE9251004980FF07DF907
:1048E0000022934B0FF0EBF8924A934B0FF075F8C0
:1048F000DDE925320FF071F8009B00E00EE0289A08
:104900000FF06BF8CDE92510386E0FF0B9F9DDE93D
:1049100025320EF0BBFF0FF0C6F93866386E0FF087
:10492000AFF902460B468EA00FF064FCBBF83A00CC
:104930005F46142801D87E87BE778D48B0F86C009A
:10494000010442F2107006D5798F084481B2A8F8AC
:10495000821088A007E07549B1F84010401A81B272
:10496000A8F8821087A00FF045FC7048B0F84010FE
:10497000322908D87549A0F840607E750E60A7F806
:104980004060FE7711E0B8F8AE2002EBC20303EB03
:104990000212B1EB820F08D86C490A68521C0A60F7
:1049A0000A2A02D37C750A220A60798F142903D956
:1049B000B97F032900D27E878346B0F840003228B1
:1049C00004D9F87F03287CD2ABF84060BBF83600EE
:1049D00042F22831884274D2397FB1B30FF0FDF82A
:1049E0000022534B0FF06BF802460B46002069493A
:1049F0000FF065F80FF057F92990386F0FF040F974
:104A0000CDE92710F96E786E0EF06CFE0FF038F9D4
:104A1000CDE9251029980FF033F900225E4B0FF0F5
:104A20004EF8444A444B0EF0D8FFDDE925320EF033
:104A3000D4FFDDE927320EF0D0FF25910090386ECB
:104A40000FF01EF9259B009A3EE0FFE7797A3A7A4B
:104A5000114301D0386E3CE00FF0BFF80022344B18
:104A60000FF02DF80B46024600204C490FF027F8B6
:104A70000FF019F92990386F0FF002F9CDE92510E0
:104A8000F96E786E0EF02EFE0FF0FAF80490009199
:104A900029980FF0F5F800223F4B0FF010F8254A47
:104AA000254B0EF09AFF009B049A0EF096FFDDE96D
:104AB00025320EF092FFCDE92510386E0FF0E0F8A8
:104AC00000E00AE0DDE925320EF081FF0FF0EBF89F
:104AD000386610F1FF4F00D33E662548B0F8441009
:104AE0002591C1F500400FF059F8049025980FF07A
:104AF0005EF804990EF080FE03990EF04BFE2599A6
:104B0000A1F5FE42FF3A7DD025490EF043FE49E073
:104B1000D20200200000694000002440CE020020A4
:104B2000B7C5B5E73A25644D410D0A00541400207D
:104B300000005940DFBC9A785634223FB7C5B5E72C
:104B4000C1BF3A256C66410D0A000000E00000205C
:104B5000B3E4B5E7313A25644D410D0A0000000089
:104B6000B3E4B5E7C1BF3A256C66410D0A00000009
:104B7000300B0020D7DCB7C5B5E7C1F7313A256463
:104B80000D0A0000D7DCB3E4B5E7C1F7313A25647C
:104B90000D0A000000C0824000408F4000008940A4
:104BA00000007A440FF03FF8FFF744FBABF84200F7
:104BB000FE48B0F94210FEA00FF01CFBDFF800B475
:104BC000BBF800000EF0F3FF6FF00B010EF052FE89
:104BD0000FF056F84FF06632FA4B0EF0FEFE002250
:104BE000F94B0EF06CFF0022F84B0EF0F3FE02467C
:104BF0000B460020F6490EF062FF0022F44B0EF047
:104C0000E6FE00E009E00FF04EF8BBF80010B1F549
:104C10007A6F06D96FF077000AE07821ABF842107E
:104C2000C6E7EC490EF0B6FD0EF0FDFFFFF702FB04
:104C3000A7F85A00E848B0F95A10E8A00FF0DAFADD
:104C4000DFF8B0B3BBF84670C7F500400EF0A6FF22
:104C5000049038460EF0ABFF04990EF0CDFD039999
:104C60000EF098FDA7F5FE41FF393AD0D9490EF074
:104C700091FD0EF0D8FFFFF7DDFA00B2D649A1F89A
:104C80005600DC48B0F84870C7F500400EF086FFCB
:104C9000834638460EF08BFF59460EF0ADFD039962
:104CA0000EF078FDA7F5FE41FF391CD0C9490EF082
:104CB00071FD0EF0B8FFFFF7BDFA00B2C64ABB495E
:104CC000A2F85800B1F8423002F1A8010B80B2F806
:104CD0005A304B80B2F856208A80C8800022104695
:104CE00005E07820CAE77820E8E700200DE001EB36
:104CF000400C31F91030BCF90270BB4203DD21F8E1
:104D00001070ACF80230401CC0B2C2F10303834201
:104D1000EDDC521CD2B2042AE7D38B46C988BBF81B
:104D20000000081A07B23946B3A00FF063FAB7487B
:104D3000B0F8C010B648B94204DC0470B5A00FF05A
:104D400059FA04E0BAF81610B94200DB0670A2481E
:104D5000B0F95610B2A00FF04DFA9F48B0F95810B4
:104D6000B4A00FF047FABBF90610DFF840B2B6A0C6
:104D7000ABF844100FF03EFADFF844824746B8F82B
:104D800002000EF014FF6FF00B010EF073FD0EF039
:104D900077FF4FF066328B4B0EF01FFE00228A4BDE
:104DA0000EF08DFE0022894B0EF014FE02460B46DB
:104DB000002087490EF083FE0022854B0EF007FE8F
:104DC0000EF071FF7988B1F57A6F02D96FF077072D
:104DD00007E080490EF0DEFC0EF025FFFFF72AFA0F
:104DE00007B27D483946A0F85C709CA00FF002FA2B
:104DF000B8F804000EF0DBFE6FF00B010EF03AFD88
:104E00000EF03EFF4FF066326E4B0EF0E6FD0022D4
:104E10006D4B0EF054FE00226C4B0EF0DBFD024693
:104E20000B4600206A490EF04AFE0022684B0EF045
:104E3000CEFD0EF038FFB8F80410B1F57A6F02D944
:104E40006FF0770007E063490EF0A4FC0EF0EBFE74
:104E5000FFF7F0F900B2804601465F48A0F85E1007
:104E600083A00FF0C7F9474502DDABF8467001E0BB
:104E7000ABF84680584FBBF944108C37BB1D3980C6
:104E8000BBF942207A80BBF94600B88019805A806D
:104E9000114498800144032091FBF0F0DFF8388141
:104EA0000021A8F85400084601E000200DE007EBBF
:104EB000400337F910C0B3F90220944503DDA3F88D
:104EC00002C027F81020401CC0B2C1F10202824289
:104ED000EDDC491CC9B20229E7D3B7F90410A8F8E0
:104EE000501068A00FF086F9B8F95010002000BFEC
:104EF00037F910208A4202D188F8340003E0401CC0
:104F0000C0B20328F4D30021334F0846923701E0A2
:104F100000200DE007EB400337F910C0B3F9022081
:104F2000944503DAA3F802C027F81020401CC0B251
:104F3000C1F102028242EDDC491CC9B20229E7D369
:104F4000DFF89480B7F9041052A0A8F852100FF0BF
:104F500051F9B8F95210002037F910208A4203D1D4
:104F60001D4981F8350003E0401CC0B20328F3D38B
:104F7000DFF8308100271F4800EB4700B0F84C00F5
:104F80000EF02BFE484A43460EF099FD0EF05FFEF0
:104F90000649DFF818B101EB4701A1F848002BF8EA
:104FA00017007F1CFFB24F45E5D381E05414002069
:104FB000BBB7BEB3CEC2B6C8203D2025640D0A00E3
:104FC0007003002066660A4000000A400000F03FBF
:104FD0000000244000007A4460000020D4A4B7C53B
:104FE000B5E74D4F53CEC2B6C8203D2025640D0A0B
:104FF00000000000300B0020B5E7D0BECEC2B6C81E
:10500000B2EE203D2025640D0A000000E00E0020D5
:1050100034030020CEC2B2EEB1A8BEAF0D0A00002C
:10502000B5E7D0BE31CEC2B6C8203D2025640D0AFA
:1050300000000000B5E7D0BE32CEC2B6C8203D2089
:1050400025640D0A00000000D7EEB8DFB5E7D0BE3A
:10505000CEC2B6C8203D2025640D0A00B3E4B5E7F2
:105060004D4F53CEC2B6C8203D2025640D0A000026
:10507000B7C5B5E74D4F53CEC2B6C8203D20256415
:105080000D0A0000D7EEB8DFCEC2B6C825640D0AFF
:1050900000000000D7EEB5CDCEC2B6C825640D0A1B
:1050A00000000000AC9C1940E926310800090020EE
:1050B0006A0000279046594605A80EF0EFFA4246CE
:1050C000594615A80EF0EAFAFE480078012843D0A8
:1050D00059464246A1F583600EF0E0FAFA4890F88E
:1050E000311061BBF949A5F1010EB1F8A820F849CA
:1050F00031F81730403131F817108B4201D3591A6B
:1051000000E0C91AA0F84C10F04B89B28A4217D8B7
:10511000DFF8C0C3BCF840C0BCF1640F10D3B0F8D6
:105120004E10491C89B2A0F84E10B3F8B030B1EB64
:10513000530F0DD3A0F84E6000F8314F44700BE0D0
:10514000BAF810308B4203D3A0F84E6080F831607B
:105150007F1CFFB2BE45CADC4246DF49DC480EF088
:105160009DFA0022681E05A903900020AB1A5B1E61
:105170000EE000BF01EB400831F810C0B8F8027033
:10518000BC4503D9A8F802C021F81070401CC0B279
:105190008342EFDC521C0398D2B29042E5DC01EB73
:1051A0004500C94F30F8021CCCA027F8421F0FF071
:1051B00021F8398800205A4632F810308B4203D14A
:1051C000C14981F8260003E0401CC0B28542F3D8F3
:1051D000002215A90020AB1A5B1E0DE001EB400870
:1051E00031F810C0B8F80270BC4503D2A8F802C06C
:1051F00021F81070401CC0B28342EFDC521C0398AF
:10520000D2B29042E6DC01EB4500AF4F30F8021C11
:10521000B7A0A7F844100EF0EDFFB7F84410002037
:10522000AD4A32F810C08C4502D187F8270003E060
:10523000401CC0B28542F3D8B7F84200B846421AC3
:10524000A249B1F8A8008242404611DD90F825201D
:10525000C2B910F8242F521CD2B20270B1F8B0308B
:10526000B2EB530F0ED39B4A947088F8254009E0A7
:10527000BAF810309A4205DC80F82460954888F826
:1052800025608670934AB1F8AE008E46B2F8403081
:1052900000EBC00101EB0017DFF868B2B3EB870F3A
:1052A00011D9BAF8121001EBC10C0CEB0111B3EBE0
:1052B000810F08D88BF86140BBF82611BAF81400AA
:1052C00081420DD224E01146B3EB870F584609D92D
:1052D00080F86140BBF82601BEF8B070B84217D321
:1052E000D47015E090F86170012F03D180F86160EF
:1052F000A0F82661CF78012F01D180F86340B0F883
:105300002A713C2F04D3D67080F86360ABF82A6111
:105310006E48B8F83A70B0F8AA0000EBC00101EB93
:10532000001E4146B7EB8E0F12D96848B0F836C15F
:105330000CEBCC0808EB0C1CB7EB8C0F08D88BF8E7
:105340006040BBF824C1B0F8380184450ED229E092
:10535000DFF878C1B7EB8E0F584609D980F8604066
:10536000BBF82401BCF8ACC060451BD3147119E034
:1053700090F860C0BCF1010F03D180F86060A0F824
:10538000246192F804C0BCF1010F01D180F86240A1
:10539000B0F828C1BCF13C0F04D3167180F86260EC
:1053A000ABF82861584890F84000800601D5547148
:1053B00000E056719646B2F94400444AB2F8C2C0C1
:1053C000604526DB92F834C15FEA8C7C07D500BFCC
:1053D0008EF8066091F819C02CF0040C07E0322B0F
:1053E00007D38EF8064091F819C04CF0040C81F8F0
:1053F00019C0B2F8C6C0604527DB92F834C15FEA35
:105400008C7C0BD58EF8076091F819C02CF0010C3C
:105410000CE0B2F8C4804045DADDEAE7142F07D388
:105420008EF8074091F819C04CF0010C81F819C0B2
:10543000B2F9CAC0F046604514DC92F834C15FEAA4
:105440008C7C07D588F8086012E0B2F8C880404527
:10545000D8DDEDE7322B0FD38EF808404B7E43F0BA
:10546000080308E0B2F9CCC0604505DB8EF808609F
:105470004B7E23F008034B76B2F9CE30C4469842F7
:105480000EDC92F83401800702D588F809600DE03F
:10549000142F0FD388F80940487E40F0020008E03E
:1054A000B2F9D030984205DB8CF80960487E20F0D4
:1054B0000200487681F82B60B646334681F82C60AE
:1054C00024E000000C00002060000020E00E00201E
:1054D000A8040020541400200009002063656C6CAF
:1054E0005F766F6C5F6D61783A25644D560D0A00EA
:1054F00063656C6C5F766F6C5F6D696E3A25644DA9
:10550000560D0A0082110020300B0020FF4881F860
:1055100029600673C68EB2F89800864204D38AF8D2
:105520001D4081F8294005E0BAF80070BE4201D85C
:105530008AF81D30F649002091F82910CDE926138C
:10554000F4492893B1F89C70B1F89E30F24ADFF824
:10555000C4B332F8101099422FD3A2F5767606EB39
:10556000000CCDF8A8C08CF82C4106EB400CBBF821
:10557000A060BCF86C81B04508D301262896ACF831
:105580006CE1DDF8A8C076468CF82C615E46994245
:105590001CD3E24A02EB000B02EB400C8BF84C41AF
:1055A000BCF8AC21B6F8A080424518D3012227925E
:1055B000ACF8ACE18BF84CE111E0DFF864C376465F
:1055C0000CEB40088444A8F86CE1DDE7DFF84CC33D
:1055D0000CEB40088444A8F8ACE18CF84CE1DFF80F
:1055E0003883B9420CD9BAF804C0614508D9CD490D
:1055F0000C5401EB4001BAF80820B1F8641009E03E
:10560000B9420FD9C7490C5401EB4001B6F8A020AC
:10561000B1F86410914217D3C149E0390C5401210B
:10562000269111E0DFF8FCC2724699420CF800E0C6
:105630000CEB400CACF864E006D2BAF806C0614549
:1056400002D2B749E0390A54401CC0B285423FF645
:105650007DAFAF482699724600F8291F2799C1707F
:1056600028998170284604E0AD49E0390A54401C6D
:10567000C0B21828F8D3002007F1320B4FEA080116
:10568000A84F31F810C0DC4514D907EB000C07EB2C
:1056900040078CF84040B7F8E470B6F8A0C0674502
:1056A0001CD3142802D2994F07447C739C4FC03FEF
:1056B0003C5413E007EB000807EB400788F8402054
:1056C000A7F8E42003F13207BC4507D2142802D220
:1056D0008E4F07447A73924FC03F3A54401CC0B279
:1056E0008542CDD88A4A894882F82AE0C38EB6F826
:1056F0009A00834204D88AF81E4082F82A4005E0C6
:10570000BAF80270BB4201D38AF81EE0804AB6F8AC
:10571000A270002092F82AB031F81030BB421DD29E
:10572000BAF80AC0634519D27E4B03EB000C03EBB9
:1057300040038CF82040B3F8A430BAF80E2093420E
:1057400037D300BF4FF0010B142803D26F4A024435
:1057500082F82140724AA03A14542AE0BB420CD28B
:10576000704A131802EB400283F82040B2F8A420DC
:10577000B6F8A6309A42E5D21BE0DFF8A8C172461F
:105780000CEB00080CEB400C88F820E0ACF8A4E02F
:10579000B6F8A4C063450CD9BAF80CC0634508D963
:1057A000142803D2594B034483F821205C4BA03BBF
:1057B0001A54401CC0B28542AED85548774680F88E
:1057C0002AB0284604E0564AC03A1754401CC0B2DA
:1057D0001828F8D3284604E0514AA03A1754401C30
:1057E000C0B21828F8D3002000EB400333444A49E4
:1057F000421C9A7631F810004FEA102C83F81BC037
:105800001877D0B28542EFD8484607E0411C00EB3C
:10581000400030448176C7760777C8B21028F5D3A8
:10582000DFF8E8804FF08C0BB8F94600002809DB60
:10583000B8F84600A6F87A0064280DD96420A6F8C6
:105840007A0009E0C0F1640080B2A6F87A008C28E2
:1058500002D95846A6F87AB081B233A00EF0CAFC3D
:10586000B8F94200002809DBB8F84200A6F87C002D
:1058700064280DD96420A6F87C0009E0C0F164001A
:1058800080B2A6F87C008C2802D95846A6F87CB0D5
:1058900081B229A00EF0AEFCB8F94400002809DB63
:1058A000B8F84400A6F87E0064280DD96420A6F854
:1058B0007E0009E0C0F1640080B2A6F87E008C286A
:1058C00002D95846A6F87EB081B2B3461FA00EF0AA
:1058D00091FC0E48DFF83880C18E26F8801F90F8C2
:1058E0003A00307104207071B6F88C0000EBC001F2
:1058F00001EB00114FF6FF7000EA81003081B8F82B
:105900003A60142E7DD9BBF8AA0027E05414002079
:1059100060000020E00E0020000900201407002095
:1059200028050020821100204D4F53B9DCCEC2B6AD
:10593000C83A25640D0A0000B5E7B3D8CFE4C4DA4D
:10594000CEC2B6C83A25640D0A000000B5E7B3D848
:10595000CEC2B6C83A25640D0A00000000EBC001B3
:1059600001EB0011B6EB810F4BD8D8F870000EF0A8
:1059700087F903910090D8F86C10D8F864000DF006
:10598000B1FE0EF07DF90490259130460EF025F918
:105990000022FE4B0EF093F8FD4AFE4B0EF01DF870
:1059A000259B049A0EF019F8039B009A0EF015F847
:1059B000064608F18000259180680EF061F93246B4
:1059C000259B0DF063FF0EF06EF908F1800106468D
:1059D0008860D8F874000EF0EAF831460DF082FEC7
:1059E00006460EF020F9CBF88C0030460EF048F950
:1059F00008F180020B46C2E908010246E6A00EF05B
:105A0000F9FBDBF8D410DBF88C005E46B0FBF1F05C
:105A1000E649ABF88600088FABF890009BF8E020D1
:105A200098F80A3040469A4205D93470B6F8922068
:105A300042F0010204E03770B6F8922022F0010231
:105A4000A6F89220B6F87A20642A0DD8B6F8B830B5
:105A50009A4205D37470B6F8922042F0020208E030
:105A6000B6F8BA309A4206D27770B6F8922022F091
:105A70000202A6F8922005228B185B78012B12D027
:105A80003771B6F89230521C23F01003D2B2A6F848
:105A90009230062AF0D9CA786AB17471B6F89220A9
:105AA00042F020020CE03471B6F8922042F010026D
:105AB000A6F89220EFE77771B6F8922022F0200244
:105AC000A6F892200A792AB1B471B6F8922042F071
:105AD000400204E0B771B6F8922022F04002A6F826
:105AE00092208A782AB1F471B6F8922042F08002AE
:105AF00004E0F771B6F8922022F08002A6F8922016
:105B0000B6F87C20642A11D8B6F8BC309A4209D97C
:105B100096F83421920709D43472B6F8922042F4F0
:105B2000807208E0B6F8BE309A4206D23772B6F8F4
:105B3000922022F48072A6F8922007229B498B18AB
:105B40005B78012B3BD07772B6F89230521C23F46D
:105B50000073D2B2A6F89230082AEFD9944A0021F5
:105B6000535C012B33D0491CC9B2B7728D42F7D8B0
:105B700000218F4A2032535C012B2AD0B6F8923094
:105B8000491C23F48063C9B2A6F892308D42F0D844
:105B90000021874A4032535C012B21D0F772B6F8BE
:105BA0009230491C23F40063C9B2A6F892308D42AA
:105BB000EFD8DFF800B29BF84030E3B918E0747218
:105BC000B6F8921041F40071A6F89210C6E7B472CC
:105BD000CEE7B6F8921041F48061A6F89210D7E7AC
:105BE000F472B6F8921041F40061A6F89210E0E762
:105BF0009BF8411021B1B6F8921041F4805103E0B6
:105C0000B6F8921021F4805189B221F40051A6F81F
:105C1000921080F82D7096F82E21012A16D196F850
:105C20002F2196F830C1624504D980F82D4080F8C4
:105C30002E4022E090F82E80B8F1010F06D10A32F2
:105C4000624518D880F82D7080F82E7021F48041BC
:105C500089B2A6F89210012902D009B1C187047651
:105C6000417E804611B1817688F81B40DFF848B14B
:105C7000D80709D104E080F82D4041F48041E7E7DE
:105C80009BF84000C00709D098F81500012805D1FD
:105C9000D6F80C010DF08BFFC8F8600088F8307062
:105CA000FEF747FB88F830000146C843800709D05B
:105CB00001F003024046022A0DD0012A15D08A07BE
:105CC0001FD027E0B6F8940040F00300A6F8940037
:105CD00088F8097012E0B6F8942022F0020242F02F
:105CE0000102A6F89420477212E0B6F8942022F040
:105CF000010242F00202A6F89420447288F808706B
:105D000008E0B6F8942022F00302A6F8942044722A
:105D100088F808402748C08F10B9BBF83E0020B172
:105D2000B6F8940040F0040003E0B6F8940020F0C8
:105D30000400A6F894008B07204A98F809304046E2
:105D400003D533B1012B0CD017E0012B01D043B1A7
:105D500013E0B6F8943023F01003A6F894301770CF
:105D60000BE013785B1CDBB21370022B05D1B6F885
:105D7000942042F01002A6F89420CB07104A037A30
:105D800024D02BB3012B28D0DBB21BE000005940FC
:105D9000DFBC9A785634223FCAB5BCCAB7C5B5E74E
:105DA000C1BF3A256C660D0A0000000054140020A3
:105DB00048040020300B0020A20B00203B000020F4
:105DC0003C00002053EAC17107D013E0012BDBD166
:105DD000B6F8941021F0200109E01178491CC9B2ED
:105DE0001170022906D1B6F8941041F02001A6F8EE
:105DF00094101770B6F8941041F00801A6F89410AA
:105E0000017B0029B6F8961002D041F0010101E0B3
:105E100021F00101A6F89610417B0029B6F89610F2
:105E200002D041F0020101E021F00201A6F8961033
:105E3000817B0029B6F8961002D041F0040101E000
:105E400021F00401A6F89610C17B0029B6F896103F
:105E500002D041F0080101E021F01001A6F89610EF
:105E6000017C0029B6F8961002D041F0100101E043
:105E700021F01001A6F89610417C0029B6F8961082
:105E800002D041F0200101E021F02001A6F8961097
:105E900098F81200002888B202D040F0400001E0DB
:105EA00020F0400081B241F46F41B346A6F896104D
:105EB0002846FA4A03E01118401C4F73C0B2142858
:105EC000F9D32946F64802E04754491CC9B21829BB
:105ED000FAD3F249897801297ED0F049CA78012A9B
:105EE0007AD08A79012A77D098F82D204646012A5F
:105EF00072D0F278012A6FD0097A01296CD001782A
:105F0000012969D04178012966D08178012963D0BF
:105F1000C178012960D0017901295DD04179012939
:105F20005AD08179012957D0C179012954D0017AF9
:105F3000012951D0417A01294ED0817A01294BD0D3
:105F4000C17A012948D0017B012945D0417B012933
:105F500042D0817B01293FD0C17B01293CD0017C0B
:105F6000012939D0417C012936D0817C012933D0E7
:105F7000C17C012930D0017D01292DD0417D01292D
:105F80002AD0817D012927D0C07D012824D09BF80B
:105F90000110584601291FD0817801291CD00179B0
:105FA000012919D04179012916D0C179012913D0CD
:105FB000017A012910D09BF80A0001280CD096F82C
:105FC0003700012808D09AF81D00012804D0377145
:105FD000B07950B112E0FFE7464688F80440FDF77B
:105FE00029F9F47486F8334008E0FDF73AF9AD4832
:105FF000F77441680A68806882430A603E46284612
:10600000A64F04E03918401C81F82160C0B2142862
:10601000F8D3A3482946203002E04654491CC9B2AF
:106020001829FAD3397901297CD0F979012979D055
:10603000797A012976D09C490978012972D098F89B
:1060400002204146012A6DD091F82D20012A69D005
:106050000278012A66D04278012A63D08278012A28
:1060600060D0C278012A5DD00279012A5AD04279E3
:10607000012A57D08279012A54D0C279012A51D0FD
:10608000027A012A4ED0427A012A4BD0827A012A22
:1060900048D0C27A012A45D0027B012A42D0427BF5
:1060A000012A3FD0827B012A3CD0C27B012A39D011
:1060B000027C012A36D0427C012A33D0827C012A1C
:1060C00030D0C27C012A2DD0027D012A2AD0427D07
:1060D000012A27D0827D012A24D0C07D012821D029
:1060E0009BF801205846012A1CD0C278012A19D0F9
:1060F0000279012A16D08279012A13D0C279012AA5
:1061000010D0027A012A0DD09BF80B00012809D08B
:106110009AF81E00012805D04E7198F8070050B17A
:106120000DE0FFE788F80540FDF70CF888F814400B
:1061300088F8334003E0FDF723F888F81460B8F8D6
:106140003AC04146BCF1320F06D9CE743E72487E49
:1061500020F00800487603E08879012800D1CC744B
:106160004E48B0F840E0BEF1320F07D90E754672C6
:10617000487E20F0020088F8190004E0C879012860
:1061800001D188F81440494900221346B1F84470FF
:1061900091F828101046E246CDF89410BAF1000F9D
:1061A00026D1BEF1320F01D8259909B34049BBF879
:1061B000B28031F810C05946C44519D9B1F8B4803D
:1061C000ACEB070CC44513DD9BF8B61001290FD1C9
:1061D000484504D204FA00F141EA02018AB207D329
:1061E000854205D9A0EB090104FA01F119438BB2EC
:1061F000401CC0B28542D1D82C4D100A84356A703B
:106200002870180AA8702B48EB7012B10BB10470FB
:1062100000E006702848007850B9244A02218432F0
:10622000412001F095FAAA1C0221412001F02BFC2B
:1062300003F0E7FE03F055FE1C4D95F82100012800
:1062400004D0022807D0032809D00DE085F820608B
:1062500085F8224008E085F82060022002E085F8F9
:106260002060032085F8220085F8216095F822003F
:1062700088B195F82000401CC0B285F820000A289B
:1062800009D30E4985F8206085F8226048680268C5
:1062900089680A4302606A7A297A11E0541400205E
:1062A000680400207C0A00205800002060000020C4
:1062B0000009002008000020D5020020940A0020D8
:1062C00071A00DF097FF287A012802D080B103D089
:1062D00011E0697A012902D0697A99B10BE073481B
:1062E00085F8236041680A68806802430A600EE00E
:1062F000697A012903D0697A084305D007E085F857
:10630000234004E0022000E0032085F82300688F8A
:10631000142805D86649B1F84010142902D806E0BF
:1063200085F828606349C8280E8000D96E776248D6
:10633000017801293FD1067085F82F60A87DE97D9D
:10634000084338D19BF8DD005F4620B1012805D015
:10635000022806D015E0FDF7C7FF11E0FDF7A5FF05
:106360000EE0B5F84200B0F5E16F0AD9A0F5E160A2
:106370000DF022FC0022514B0DF0A1FB0DF067FC4B
:10638000A872A87A642801D96420A872D7F80C01F1
:106390000DF023FC07468846A87A0DF01EFC00226B
:1063A000474B0DF08CFB3A4643460DF016FB0DF0C3
:1063B0007AFC2866EC7595F82900424F012815D122
:1063C0006420A872387830B1286E0DF02CFCCBF820
:1063D0000C013E7004E0DBF80C010DF0E8FB2866D0
:1063E000002004F054FF012004F051FF95F82A002A
:1063F000012809D1AE726C7000202E6604F047FFB0
:10640000012004F044FF3C70A97A2FA00DF0F2FEA9
:10641000DFF8C090264CB9F80000E0872878012802
:106420002AD16878A846012826D1DBF8D4005C215F
:1064300048430DF0D2FB0F4627490546D1E9062314
:10644000D1E908010DF0C3FA0022244B0DF0C5FA82
:106450002A463B460DF033FB0DF0F9FB81B2E18794
:10646000A9F80010642903D96421E187A9F8001074
:1064700088F8006088F80160E18F19A00DF0BAFE7D
:106480002BB0BDE8F08F00000D0A44535F4D43551B
:106490005F466C61673D25640D0A43485F4D435577
:1064A0005F466C61673D25640D0A0000A00A00206C
:1064B00054140020100000200C00002000001440A4
:1064C00000005940D0020020534F433A25640D0A82
:1064D000000000002E030020E00000200088C340E0
:1064E000534F483A25640D0A000000007047FEE74C
:1064F000FEE7FEE7FEE770477047704770472DE9FB
:10650000F041FF4C082120460DF06EF8251D28B102
:1065100021882046298808210DF073F8042120469F
:106520000DF062F828B121882046298804210DF059
:1065300068F8022120460DF057F828B1218820463E
:10654000298802210DF05DF8012120460DF04CF85C
:1065500028B121882046298801210DF052F840F207
:106560002556314620460DF055F800286AD03146B0
:1065700020460DF079F828880325C1B2E148421C75
:10658000B0F802349954B0F8023400220124EBB37D
:10659000012B44D0022B47D0032B48D00CD903F158
:1065A00001039BB2A0F80234C67806F10306B34299
:1065B00002D1A0F802240470D348431CB0F86461EF
:1065C000F154B0F8643173B3012B3DD0022B41D0AC
:1065D000CE4ECF4D40F26311032B3ED0042B31D36E
:1065E0005B1C9BB2A0F86431B0F803707FBABF1C8B
:1065F000BB4227D1071FDB5DA0F86421482B3CD0AC
:1066000032802A70BDE8F041401C00E001E00DF04E
:106610005EB8A52901D000230CE001230AE05A2925
:10662000F9D1022306E008E0A0F80254C4E7832968
:10663000F1D10423A0F80234BEE74C2906D1012190
:10664000A0F86411BDE8F081442901D00021F7E7EA
:106650000221F5E7A0F86451F4E72C700423A0F8B8
:106660006431C3781C0203792343B3F5967FE9D3E1
:1066700032802A70A0F86421C4E70470A548047031
:10668000A548047032802A70DCE72DE9F041A34C64
:10669000082120460CF0A8FF251D40B1208828883D
:1066A00020460CF037FF082120460CF0AAFF0421F9
:1066B00020460CF099FF28B1218820462988042122
:1066C0000CF09FFF022120460CF08EFF28B121889C
:1066D0002046298802210CF094FF012120460CF06D
:1066E00083FF28B121882046298801210CF089FFE9
:1066F00040F22556314620460CF08CFF0028A1D0F0
:10670000314620460CF0B0FF2888C1B28448421CB4
:10671000B0F864319954B0F86431E3B1012B20D062
:10672000022B24D0002201267E4D7F4C40F26311C3
:10673000032B1ED0042B85D35B1C9BB2A0F86431C5
:10674000B0F803707FBABF1CBB4209D1071FDB5DE5
:10675000482B22D018E04C2905D10121A0F8641162
:1067600070E7442901D00021F8E70221F6E7032170
:10677000F4E726700423A0F86431C3781E0203797D
:106780003343B3F5967FEBD3A0F8642122702A80BF
:10679000BDE8F041401C0CF09ABFA0F864210670DF
:1067A0006248067022702A804CE72DE9F041604C67
:1067B000082120460CF018FF251D28B1218820460D
:1067C000298808210CF01DFF042120460CF00CFF45
:1067D00028B121882046298804210CF012FF0221CB
:1067E00020460CF001FF28B121882046298802218B
:1067F0000CF007FF012120460CF0F6FE28B121889D
:106800002046298801210CF0FCFE40F22556314635
:1068100020460CF0FFFE002838D0314620460CF010
:1068200023FF2888C1B24348421CB0F86431995410
:10683000B0F8643123B3012B29D0022B2DD00022D4
:1068400001263D4D3D4C40F26311032B27D0042B14
:106850001CD35B1C9BB2A0F86431B0F803707FBA04
:10686000BF1CBB4212D1071FDB5DA0F86421482B7F
:1068700025D02A802270BDE8F041401C0CF027BFD3
:106880004C2906D15FF00101A0F86411DAE6442931
:1068900001D00021F8E70221F6E70321F4E7267092
:1068A0000423A0F86431C3781E0203793343B3F59F
:1068B000967FEBD32A802270A0F86421DBE7067074
:1068C0001F4806702A802270BCE62DE9F04F4FF079
:1068D0008049B9F81000C0077ED00F48194C828853
:1068E000511C0021818023780122012B30D1036AC1
:1068F000154D5B1C0362AB422AD90162217025E071
:1069000000380140901D0020140C00201E000020C3
:106910000D00002040010020140100200044004030
:106920001C100020200000200E000020410100204B
:10693000004800407A0D0020560000205A00002038
:10694000420100205503002020BF0200AA4B1A700C
:10695000C3884FF4FA7B5B1C9FB2A84BC7801B789F
:10696000012B07D183695B1C83615B4502D3A44B78
:106970001A708161A34B4FF47A7C1B78012B07D1ED
:10698000C3695B1CC361634502D39F4B1A70C1612D
:10699000DFF8788241F2883498F80030012B0BD16F
:1069A0009B4D2E88731C2B80A64205D9994B2980BC
:1069B00088F80010A3F86411DFF85CA240F6B8383C
:1069C0009AF80030012B0CD1944D2E88731C2B802B
:1069D000464506D9298000E00CE1914B8AF8001069
:1069E0001A70DFF840A29AF80030012B0BD18E4DBF
:1069F0002E88731C2B80A64205D98C4B29808AF8DF
:106A00000010A3F86411DFF828A29AF80030012BD7
:106A10000BD1884E33885D1C3580A34205D9864B47
:106A200031808AF80010A3F86411642F68D3834B77
:106A3000C1801C78641CE4B21C70082C02D3804C0A
:106A4000227019707F4B804C00229D1895F82C51B4
:106A500035B103EB4205B5F86C61761CA5F86C61A5
:106A6000A51895F84C5135B104EB4205B5F8AC6169
:106A7000761CA5F8AC61521CD2B2202AE5D3734A29
:106A80000023D45C2CB102EB430434F8645F6D1C2A
:106A90002580D41894F820502DB102EB430535F829
:106AA000A46F761C2E8094F840402CB102EB430575
:106AB00035F8E44F641C2C805B1CDBB2202BE0D348
:106AC00092F8603023B1B2F824315B1CA2F8243173
:106AD00092F8613023B1B2F826315B1CA2F826315E
:106AE00092F8623023B1B2F828315B1CA2F8283149
:106AF00092F8633023B1B2F82A315B1CA2F82A3134
:106B0000534A13685B1C1360524A13685B1C136082
:106B1000514A13685B1C13608268521C8260C36810
:106B20005B1CC3600469641C046145694B4C6D1CAB
:106B300045612478032C0DD0022C13D0012C14D0E5
:106B4000C4B1474A467894685268002E16680FD040
:106B5000A6430EE07D2AF4DB8160427882F00102D8
:106B60004270EEE76245F7DAEBE74245F4DAE8E730
:106B7000264316603B4A14783B4A032C0ED0022C65
:106B800014D0012C15D0CCB18378002B53681E682B
:106B9000976811D03E431E6084B114E0FA2BF3DBFA
:106BA000C160837883F001038370EDE75B45F7DA1A
:106BB000EAE76345F4DAE7E7BE43ECE753681C68AD
:106BC000926814431C604EF6602295420CD34161DA
:106BD000C278521CD2B2C2703C2A05D3C17023487D
:106BE00050F8F81F491C0160B9F8101021F001019C
:106BF000A9F81010BDE8F08F6E0300203D000020C2
:106C00003E0000203F000020400000200D0000203A
:106C10001E000020140C0020590000205400002009
:106C2000580000200E000020200000201C10002032
:106C30005A000020560000207A0D0020120100208A
:106C40008F0000202805002014070020821100205A
:106C5000AC0300203C010020101A0020830000201B
:106C6000A00A002082000020940A0020E00E0020EC
:106C70000648804706480047FEE7FEE7FEE7FEE7D6
:106C8000FEE7FEE7FEE7FEE7FEE7FEE71701010885
:106C9000ED3000081CB50020009001213D200BF0D4
:106CA000E3FA1B4C009813E004EBC000C1798DF8A7
:106CB00007108188ADF8041080798DF806000098DF
:106CC00001A954F830000AF08DFF0098401C009094
:106CD0001928E9D301210F480BF055F81CBD38B530
:106CE0000446012108200BF0BFFA4FF44070ADF8C4
:106CF0000000012C0AD010208DF8030003208DF82D
:106D00000200694604480AF06DFF38BD1420F3E71D
:106D1000884F010800023000000C014030B501210D
:106D200085B088030BF0A0FA00244FF4E130009006
:106D3000ADF808400C20804DADF80440ADF80A00D5
:106D4000ADF80640ADF80C40694628460CF0E5FA6F
:106D5000012128460CF06DFB77480C30018841F08A
:106D6000200101804FF4E06009F056FA25208DF8EB
:106D700010008DF811408DF8124001208DF813009D
:106D800004A809F04EFA05B030BD30B5012185B038
:106D900048040BF076FA00244FF416500090ADF83A
:106DA00008400C20654DADF80440ADF80A00ADF880
:106DB0000640ADF80C40694628460CF0AEFA0121B9
:106DC00028460CF036FB5D480C30018841F020016C
:106DD00001804FF4E06009F01FFA26208DF81000C2
:106DE0008DF8114001208DF812008DF8130004A8D1
:106DF00009F017FAC7E730B5012185B088040BF018
:106E000040FA00244FF47A300090ADF808400C208E
:106E10004B4DADF80440ADF80A00ADF80640ADF8B2
:106E20000C40694628460CF078FA012128460CF0FF
:106E300000FB43480C30018841F0200101804FF4F1
:106E4000E06009F0E9F927208DF810008DF8114075
:106E50008DF8124001208DF8130004A809F0E1F923
:106E600091E77FB5012108460BF00BFA40F2E730BD
:106E7000ADF804004720ADF8000000244FF0804535
:106E8000ADF80640ADF80240694628460BF0C8FB55
:106E90000122114628460BF03AFF012128460BF04B
:106EA0001BFF1C208DF80C008DF80D4001208DF883
:106EB0000E008DF80F0003A809F0B3F97FBD10B5DF
:106EC000FFF7CFFFFFF72AFFFFF75FFFFFF793FF03
:106ED000194C0122282120460CF0B7FA012260212A
:106EE00020460CF0B2FA154C0122282120460CF065
:106EF000ACFA20460122BDE8104060210CF0A5BA92
:106F000070B50F4D0446C1B228460CF0FFFA40217F
:106F100028460CF069FB0028F9D0204670BD10B55A
:106F2000074C202120460CF05FFB0028F9D02046BA
:106F3000BDE810400CF0EEBA0038014000440040BB
:106F4000004800404FF0E020016921F00401016198
:106F500070471649098848434FF0E02148610020F6
:106F600088610A6942F001020A610A69D203FCD50C
:106F70000A6922F001020A6188617047C10000209D
:106F800001E000BF401C8842FBD3704710B50446A7
:106F90000AF07FFF40F69F7203E01046401E80B269
:106FA000FCD2641EA4B2F8D210BD0000380100204B
:106FB0000D490968491A8142FDD370470A4A12688F
:106FC000C0E90021012101727047017A31B10649FF
:106FD0000268436809688A1A9A4201D20020704701
:106FE00001600120704700003C01002045490A88EB
:106FF0005206FCD54349091D0880704742490A885A
:107000005206FCD54049091D088070473F490A884F
:107010005206FCD53D49091D0880704710B504464D
:10702000002303E0FFF7E2FF5B1CDBB2E05C00281B
:10703000F8D10D20FFF7DAFFBDE810400A20D5E7B0
:1070400010B50446002303E0FFF7E0FF5B1CDBB252
:10705000E05C0028F8D110BD10B50446002303E021
:10706000FFF7D4FF5B1CDBB2E05C0028F8D110BD59
:1070700010B50C46034603E013F8010BFFF7B6FF0B
:10708000641EA4B2F8D210BD10B50C46034603E04E
:1070900013F8010BFFF7AAFF641EA4B2F8D210BDCB
:1070A00030B50C4603461A4D13E0687818B113F852
:1070B000010BFFF7A3FF2878E978084303D013F802
:1070C000010BFFF793FFA87818B113F8010BFFF736
:1070D0009DFF641EA4B2E8D230BD704708B5002001
:1070E0008DF800008DF800009DF8000066289DF8DE
:1070F000000000F10100F5D38DF8000001208DF8AB
:10710000000008BD00380140004400400048004035
:10711000400100202DE9F041B74C4FF48073251F4A
:1071200022462946B5480DF007F8B44863152246B3
:1071300029460C300DF000F8B14EB048371F20231F
:107140003246394618300CF0F7FFAC48102332466F
:10715000394624300CF0F0FFA8484FF40043224693
:10716000294630300CF0E8FFA4484FF48043224613
:1071700029463C300CF0E0FFA048802322462946F7
:1071800048300CF0D9FF9D48102322462946543040
:107190000CF0D2FF99484FF4004332463946A830EC
:1071A0000CF0CAFF9548202322462946B4300CF043
:1071B000C3FF924804232246294684300CF0BCFFCA
:1071C0008E4808232246294690300CF0B5FF8B48A4
:1071D000A31422462946C0300CF0AEFF8748631442
:1071E0002246294678300CF0A7FF864A8348A2F150
:1071F0000408631441469C300CF09EFF7F484FF416
:107200008043804A414660300CF096FF7B484FF443
:1072100000437C4A41466C300CF08EFF77480123D6
:1072200032463946CC300CF087FF7448A3153246FD
:107230003946D8300CF080FF704802232246294698
:10724000E4300CF079FF6D48402322462946F030A7
:107250000CF072FF01200AF03EFE00200AF071FFE0
:10726000002009F07AFA00200AF035FE634948311F
:107270004868026889688A430260604960314868EA
:10728000026889680A4302605C496C314868026898
:1072900089680A430260FBF755FFFBF7CBFF5749AC
:1072A00054314868026889680A4302605349903142
:1072B0004868026889688A43026050498431486896
:1072C000026889680A4302604C497831486802685C
:1072D00089680A43026049499C31486802688968A4
:1072E0000A4302604549A8314868026889688A43B0
:1072F00002604249B4314868026889680A43026002
:107300003E49C0314868026889680A430260BDE8A6
:10731000F0813A4B10B50021B3F1A00301EB8104D9
:1073200003EBC404844201D10A4602E0491C04294B
:10733000F4DB354901201AB1012A00D1487010BD93
:10734000087010BD2D4B10B50021A03B01EB81044E
:1073500003EBC404844201D10A4602E0491C04291B
:10736000F4DB294900201AB1012A00D1487010BD70
:10737000087010BDF0B500206425AFF26906AFF2C9
:107380003B071E490524A0398446012200EB8003F7
:1073900001EBC303C3E90445C3E9076748B101280A
:1073A0000AD002280ED0032812D0401C0428EDDB9E
:1073B000F0BD8A760120E9E71048A03880F842C085
:1073C0000220E3E70D48A03880F86A200320DDE7BB
:1073D0000A48A03880F89220F0BD70B5074D00240F
:1073E000B5F1A00504EB840005EBC0000CF06DFEC8
:1073F000641C042CF6DB70BD0C0C0140340A002028
:107400000C0801400C1001404401002038B50E4D1D
:1074100000240E480CF03EFE05EB041211680860D3
:10742000010006D4D0680090137A526807480CF027
:10743000FFFD641C062CECD338BD704770477047C5
:10744000704770477047000060010020280000204E
:1074500010B502460020FE4B06E000BF12F8014BBB
:107460004440491E185DC9B20029F7D110BD38B596
:107470000446012108200AF0F7FE4FF48070ADF8B1
:10748000000003208DF80200012C08D05FF01000EE
:107490008DF803006946EF480AF0A4FB38BD0420CC
:1074A000F6E770B50020FFF7E2FFEB4C606801687B
:1074B000A26811430160E94D68680168AA68114338
:1074C00001600D20FFF75AFD60680168A2689143D2
:1074D00001600D20FFF752FD68680168AA689143BA
:1074E000016070BD70B50020FFF7C1FFDA4C606825
:1074F0000168A26891430160D84D68680168AA6874
:10750000914301600D20FFF739FD68680168AA68A2
:10751000114301600D20FFF731FD60680168A2682A
:107520001143016070BD2DE9F04107460020FFF7CF
:107530009EFFC94CC94E00254FF0800828FA05F07F
:10754000384260680168A26801D0114300E09143AD
:1075500001600D20FFF712FD70680168B2681143E9
:1075600001600D20FFF70AFD70680168B268914361
:1075700001606D1CEDB2082DE0D30120FFF777FF0D
:107580000D20FFF7FBFC70680168B26811430160D1
:1075900020680068A168084201D0012400E00024AE
:1075A0000D20FFF7EBFC70680168B2689143016041
:1075B0002046BDE8F0812DE9F047814600250120F5
:1075C000FFF755FFA44EA54C00274FF080080D2073
:1075D000FFF7D4FC60680168A2681143016030685D
:1075E0000068B168084228FA07F001D0054300E0BE
:1075F00085430D20FFF7C2FC60680168A2689143D3
:1076000001607F1CFFB2082FE1D30020FFF72FFF9E
:107610005FEAC97070680168B26801D0114300E088
:10762000914301600D20FFF7A9FC60680168A26822
:10763000114301600D20FFF7A1FC60680168A2689A
:10764000914301602846BDE8F087F8B50D468DF8F6
:1076500000008DF80110064614468DF80220032123
:107660006846FFF7F5FE8DF80300FFF71AFF304676
:10767000FFF759FF2846FFF756FF2046FFF753FF55
:107680009DF80300FFF74FFFFFF72CFF3220FFF7B5
:1076900060FCF8BD2DE9F04104461E4615460F4634
:1076A0000520FFF76BFCFFF7FCFE2046FFF73BFFD2
:1076B0003846FFF738FF2846FFF735FF0D20FFF764
:1076C0005DFCFFF7EEFE44F00100FFF72CFF002405
:1076D0006F1C0BE0AC4203D10020FFF76CFF03E00E
:1076E0000120FFF768FF3055641CE4B2BC42F1D3BF
:1076F000BDE8F041F6E608B534208DF80000EA2038
:107700008DF80100C0208DF8020003216846FFF7C4
:107710009FFE8DF80300FFF7C4FE3420FFF703FF40
:10772000EA20FFF700FFC020FFF7FDFE9DF80300F1
:10773000FFF7F9FEFFF7D6FE3220FFF70AFC3220F2
:10774000FFF707FC782240213420FFF77EFF08BDB9
:107750002DE9F04117460E460546002408E03A5D43
:1077600029463420FFF771FF6D1C641CEDB2E4B2B2
:10777000B442F4D31DE72DE9F04116460F46054605
:1077800000240AE03346012229463420FFF782FF15
:107790006D1C641CEDB2E4B2761CBC42F2D308E767
:1077A00038B50446012104200AF05EFD2020ADF822
:1077B000000003208DF80200012C08D05FF01000BB
:1077C0008DF80300694626480AF00CFA38BD0420FB
:1077D000F6E770B50020FFF7E3FF224C6068016810
:1077E000A26811430160204D68680168AA681143CE
:1077F00001600D20FFF7C2FB60680168A268914339
:1078000001600D20FFF7BAFB68680168AA68914320
:10781000016070BD70B50020FFF7C2FF114C6068B9
:107820000168A268914301600F4D68680168AA6809
:10783000914301600D20FFF7A1FB68680168AA6809
:10784000114301600D20FFF799FB606801680DE0AE
:10785000CE010020000C0140340A0020400A002024
:10786000000801404C0A0020580A0020A268114379
:10787000016070BD2DE9F04107460020FFF790FF41
:10788000FC4CFD4E00254FF0800800BF28FA05F0A3
:10789000384260680168A26801D0114300E091435A
:1078A00001600D20FFF76AFB70680168B268114340
:1078B00001600D20FFF762FB70680168B2689143B8
:1078C00001606D1CEDB2082DE0D30120FFF768FFC9
:1078D0000D20FFF753FB70680168B2681143016027
:1078E00020680068A168084201D0012400E000245B
:1078F0000D20FFF743FB70680168B2689143016097
:10790000204656E62DE9F047814600250120FFF785
:1079100047FFD84ED84C00274FF080080D20FFF7C6
:107920002DFB60680168A26811430160306800683F
:10793000B168084228FA07F001D0054300E085430A
:107940000D20FFF71BFB60680168A268914301608E
:107950007F1CFFB2082FE1D30020FFF721FF5FEA71
:10796000C97070680168B26801D0114300E09143AA
:1079700001600D20FFF702FB60680168A2681143F7
:1079800001600D20FFF7FAFA60680168A268914370
:107990000160284657E6F8B50D468DF800008DF8D1
:1079A0000110064614468DF8022003216846FFF7B1
:1079B0004FFD8DF80300FFF70CFF3046FFF75AFF2D
:1079C0002846FFF757FF2046FFF754FF9DF80300B6
:1079D000FFF750FFFFF71EFF3220FFF7BAFAF8BD9E
:1079E0002DE9F0411E4615460F460446FFF7F1FE0D
:1079F0002046FFF73FFF3846FFF73CFF2846FFF7DA
:107A000039FF0D20FFF7BAFAFFF7E3FE44F001005B
:107A1000FFF730FF00246F1C0BE0AC4203D10020C5
:107A2000FFF770FF03E00120FFF76CFF3055641C87
:107A3000E4B2BC42F1D3BDE8F041EBE608B5342036
:107A40008DF80000EA208DF80100C0208DF80200BA
:107A500003216846FFF7FCFC8DF80300FFF7B9FE31
:107A60003420FFF707FFEA20FFF704FFC020FFF7ED
:107A700001FF9DF80300FFF7FDFEFFF7CBFE32206C
:107A8000FFF767FA08BD2DE9F04117460E46054697
:107A9000002408E03A5D29463420FFF77CFF6D1C86
:107AA000641CEDB2E4B2B442F4D382E52DE9F041B6
:107AB00016460F46054600240AE0334601222946B1
:107AC0003420FFF78DFF6D1C641CEDB2E4B2761C10
:107AD000BC42F2D36DE538B50446012108200AF016
:107AE000C3FB4FF40040ADF8000003208DF8020006
:107AF000012C08D05FF010008DF8030069465F4844
:107B00000AF070F838BD0420F6E7704770B5002021
:107B1000FFF7E1FF5A4C60680168A26811430160F9
:107B2000584D68680168AA68114301600D20FFF78D
:107B300025FA60680168A268914301600D20FFF793
:107B40001DFA68680168AA689143016070BD70B54C
:107B50000020FFF7C0FF4B4C60680168A2689143AA
:107B60000160474D68680168AA68914301600D2073
:107B7000FFF704FA60680168A268114301600D20F4
:107B8000FFF7FCF968680168AA681143016070BDDD
:107B90002DE9F04107460020FFF79DFF394E706840
:107BA0000168B26891430160354C00254FF08008B0
:107BB00028FA05F0384260680168A26801D01143D4
:107BC00000E0914301600D20FFF7D8F9706801686B
:107BD000B268114301600D20FFF7D0F970680168A9
:107BE000B268914301606D1CEDB2082DE0D3012015
:107BF000FFF771FF0D20FFF7C1F970680168B268E7
:107C0000114301600620FFF7B9F920680068A168F8
:107C1000084201D0012400E000240D20FFF7AEF956
:107C200070680168B268914301602046C1E42DE9A3
:107C3000F047814600250120FFF74DFF104E114C03
:107C400000274FF0800860680168A26891430160D6
:107C50000D20FFF793F960680168A2681143016085
:107C600030680068B168084228FA07F00CD0054374
:107C70000BE000004C0A0020580A0020000C0140D4
:107C8000640A0020700A002085430D20FFF776F972
:107C900060680168A268914301607F1CFFB2082FF1
:107CA000D1D30020FFF717FF5FEAC9707068016841
:107CB000B26801D0914300E0114301600D20FFF74D
:107CC0005DF960680168A268114301600D20FFF74B
:107CD00055F960680168A268914301602846B2E4E2
:107CE00010B5FFF713FF7020FFF752FFE120FFF7F9
:107CF0004FFF0820FFF74CFF0020FFF749FFFFF779
:107D000026FFBDE810403220FFF723B910B5FFF77A
:107D1000FDFE7020FFF73CFFAC20FFF739FF33205A
:107D2000FFF736FF0020FFF733FFFFF710FFBDE836
:107D300010406420FFF70DB92DE9F04105460E46CD
:107D40000520FFF71BF9FFF7E1FE7120FFF720FF89
:107D500000246F1C0BE0AC4203D10020FFF767FF4B
:107D600003E00120FFF763FF3055641CE4B2BC421E
:107D7000F1D3BDE8F041EAE610B5FFF7C7FE702089
:107D8000FFF706FFBA20FFF703FFBDE81040DEE66D
:107D9000A6E710B5184C002020606060FFF7B6FF22
:107DA00004F108010620FFF7C7FF04F1080001787D
:107DB00001F06801082901D0002010BD41788278C7
:107DC000C07842EA012140EA012000094FF47A71AB
:107DD0004843000D0A21B0FBF1F2B2FBF1F301FBC5
:107DE00013216422B0FBF2F000EB800001EB4000B5
:107DF000606080B210BD0000C0010020F8B59D4950
:107E000000250095097801297ED101287CD16A4698
:107E10000020FFF7B0FC984C9DF800006A46A07661
:107E2000012119202E34FFF7A6FC9DF80000607197
:107E30006A4601214020FFF79EFC9DF80000A073D8
:107E40006A4602214120FFF796FCBDF800006A4611
:107E500040BA208201214320FFF78DFC9DF80000ED
:107E6000A0746A4601214420FFF785FC9DF80000BC
:107E7000E0746A4601214520FFF77DFC9DF8000073
:107E800020756A4602214620FFF775FCBDF8000008
:107E90006A4640BAE08202214820FFF76CFCBDF838
:107EA00000006A4640BA208302214A20FFF763FCA3
:107EB000BDF800006A4640BA60838DF800508DF826
:107EC000015002214C20FFF756FCBDF800006A4625
:107ED00040BAA08302214E20FFF74DFCBDF8000000
:107EE0006A4640BAE08302215020FFF744FCBDF807
:107EF00000006A4640BA208402215220FFF73BFC72
:107F0000BDF8000040BA00E0B3E060846A46022198
:107F10005420FFF730FCBDF800006A4640BAA08448
:107F200002215620FFF727FCBDF800006A4640BA40
:107F3000E08402215820FFF71EFCBDF800006A46CD
:107F400040BA208502215A20FFF715FCBDF8000039
:107F50006A4640BA608502215C20FFF70CFCBDF840
:107F600000006A4640BAA08502215E20FFF703FCAC
:107F7000BDF800006A4640BAE08502216020FFF7A4
:107F8000FAFBBDF800006A4640BA20860221622052
:107F9000FFF7F1FBBDF800006A4640BA6086022197
:107FA0006420FFF7E8FBBDF800006A4640BAA086EF
:107FB00002216620FFF7DFFBBDF800006A4640BAE9
:107FC000E08602216820FFF7D6FBBDF800006A4674
:107FD00040BA208702216A20FFF7CDFBBDF80000E0
:107FE0006A4640BA608702216C20FFF7C4FBBDF8E7
:107FF00000006A4640BAA08702216E20FFF7BBFB53
:10800000BDF800001D4E41BAE18770782E3C18B1D2
:1080100075704FF6EF70B08019A00CF0EBF8B4F863
:108020006C00B188884208D2081A4FF6FF71081A0E
:10803000A4F86C000120307002E0401AA4F86C0033
:1080400034F86C1F13A00CF0D5F8B17814A00CF024
:10805000D1F86A4601217020FFF78DFB9DF80000E2
:10806000A0706A4601217120FFF785FB9DF8000092
:10807000E070F8BD0B000020300B0020CE02002085
:108080004375725F4F6666736574313A3078257850
:108090000D0A0000434144433A307825780D0A0028
:1080A00043656C6C5F526C5F466C673A25780D0ACD
:1080B000000000002DE9F043ADF5537D0F46DDE9EA
:1080C000DA480546994616464FF4D27168460BF0D9
:1080D000FEFA44F64440ADF8A4016A9504F112009A
:1080E0008DF8AC710025ADF8A6018DF8AD518DF875
:1080F000AE610DF2AF102246494606460BF0CEFAAD
:1081000048208DF84403D295BDF8A401CDF84083F2
:10811000010A8DF800108DF80100BDF8A601224675
:10812000010A8DF802108DF803006A983146000E9E
:108130008DF804006A98000C8DF805006A98000A12
:108140008DF806006A988DF807009DF8AC018DF84F
:1081500008009DF8AD018DF809009DF8AE018DF87D
:108160000A000DF10B000BF099FAD0986A46010E47
:108170000DEB040004F11003C172D099090C0173D6
:10818000D099090A4173D09981739DF84413C17342
:10819000002105E0575CD29E491C3E4489B2D2962C
:1081A0009942F7D305744574D2991434090A81743D
:1081B000D299C174A1B21046FEF772FF0DF5537D3E
:1081C000BDE8F0832DE9F04F044600220078E9B0C5
:1081D0001746012878D100262670B4F803003146EE
:1081E00040BA831E04E06518491C6D7889B22A44A0
:1081F0009942F8DB204492B2B0F8011049BA8A42A1
:1082000041F06786B4F805104FF4B0734ABAB4F879
:10821000071049BA62F31F415E91627A5F9230F8AB
:10822000061D94F80C90408849BA40BA61F31F408B
:108230008246F748F649007840F001000870F54D95
:108240000DF1E6015D91491C05F5887065915A9024
:108250003AA96491491C6091491C481CCDE962010E
:10826000DFF8B48305F1FC004FF0010B61900C2A9C
:1082700081F02F86DFE812F035060C001800550358
:1082800035062905B405580A3506350635061F0E8C
:108290008DF8089088F800B0CDE900BA594602ABD5
:1082A0000A465E9801F004BE98F80000002801F02C
:1082B000108601205B90194602A80BF008FAA9F17C
:1082C0008E003B2830D200E0F0E3DFE800F01E250E
:1082D0002E353C434A51585F666D747B82898E957A
:1082E0009CA3AAB1B8BFC6CDF2F9EFEEEDECEBEA74
:1082F000E9E8E7E6E5E4E32DE2E1E0DFDE2DDDDCC1
:10830000DB2DDAD9D8D7D6D5D400B4F80D0040BAD1
:10831000A5F898000A2005E0B4F80D0040BAA5F8C9
:108320009A000B2002F0B3FFA4E2B4F80D0040BAAB
:10833000A5F89C000C20F5E7B4F80D0040BAA5F8AC
:108340009E000D20EEE7B4F80D0040BAA5F8A0009D
:108350000E20E7E7B4F80D0040BAA5F8A2000F2000
:10836000E0E7B4F80D0040BAA5F8A4001020D9E762
:10837000B4F80D0040BAA5F8A6001120D2E7B4F871
:108380000D0040BAA5F8A8001220CBE7B4F80D0004
:1083900040BAA5F8AA001320C4E7B4F80D0040BA0B
:1083A000A5F8AC001420BDE7B4F80D0040BAA5F85C
:1083B000AE001520B6E7B4F80D0040BAA5F8B0003D
:1083C0001620AFE7B4F80D0040BAA5F8B2001720A8
:1083D000A8E7B4F80D0040BAA5F8B4001820A1E74A
:1083E000607B85F8B60019209CE7B4F80D0040BA10
:1083F000A5F8B8001A2095E7B4F80D0040BAA5F822
:10840000BA001B208EE7B4F80D0040BAA5F8BC00F6
:108410001C2087E7B4F80D0040BAA5F8BE001D2067
:1084200080E7B4F80D0040BAA5F8C0001E2079E737
:10843000B4F80D0040BAA5F8C2001F2072E7B4F8E6
:108440000D0040BAA5F8C60020206BE7B4F80D0077
:1084500040BAA5F8CA00212064E7B4F80D0040BA7C
:10846000A5F8CC0022205DE7B4F80D0040BAA5F8CD
:10847000CE00232056E746E23EE236E22EE226E236
:1084800020E21AE214E20CE204E2ECE1DCE1CAE1EF
:10849000BDE1B8E1ABE1A4E19AE189E17BE175E1FD
:1084A00068E1E8E0E2E0DAE0A3E086E064E007E02B
:1084B000FFE7B4F80D0040BAA5F8D000242031E75A
:1084C000564F78680168BA681143016088F8046003
:1084D000607B00F00F0188F803101420FEF756FDB2
:1084E0004F4898F803104C4A807E121D00F0F000AF
:1084F000084388F8040001210020FFF729F9786873
:108500000168BA6891430160FFF7F5F895F8D21059
:10851000607B814227D00BF060FB0746B5F89C00DA
:108520008B4698350BF059FB00223E4B0BF0C7FAF7
:108530003A465B460BF051FA0BF089FB2880607BD2
:108540000BF04BFB07468B4668890BF046FB00227D
:10855000344B0BF0B4FA3A465B460BF03EFA0BF0A4
:1085600076FB6880983D607B85F8D200252002F07C
:108570008EFE03F0F6FF7DE1B4F80D00B4F80F10A5
:1085800043BA4ABA63F31F42D5F8D4309A4203D0B3
:10859000254A1670254A167042BA48BA62F31F403F
:1085A00045F8D40F262002F072FEA96B55F8D409C5
:1085B0008142E0D9C5F80C015CE1607B85F8D80008
:1085C000012809D01A485D4680F800B0FAF732FE5B
:1085D000184805702720A5E61548164D067028781E
:1085E00018B1154800780028F4D1FAF73AFE2E7039
:1085F000F0E7607B85F8D900012823D00F485D465D
:1086000080F800B0FAF79EFD0D480570282089E635
:1086100081000020E00E0020D40200207C0A00200F
:10862000300B00200000244076000020770000205E
:108630006600002073000020640000206700002016
:1086400074000020FB48FC4D0670287818B1FB48E8
:1086500000780028DAD1FAF793FD2E70D6E7B4F847
:108660000D0040BAA5F8DA0029205BE6607B85F8AA
:10867000DC002A2056E695F8DD10607B814270D040
:10868000EF490E7020B1012824D0022845D068E0BF
:1086900040F6426025F89C0F0420A8804FF46161E9
:1086A00069804FF42F61E980688140F65431298157
:1086B000142169824021A9823C21E981298250212B
:1086C000A5F89A10A5F89C004FF47A70A88140F69E
:1086D000E4401FE041F2680025F89C0F0420A880C8
:1086E00041F2040169804FF42F61E980688140F60E
:1086F00054312981142169824021A9823C21E981D8
:1087000029825021A5F89A10A5F89C004FF47A70A0
:10871000A8818000E8820A2021E040F6FC0025F8CC
:108720009C0F0420A88040F6CA01698040F2DC5109
:10873000E98068814FF4C861298114216982402150
:10874000A9823C21E98129825021A5F89A10A5F837
:108750009C004FF47A70A8814000E88205202883AD
:108760009C3D607B85F8DD002B2002F090FD03F03E
:108770006DFE7FE0B4F80D0040BA25F8DE0F2C2026
:1087800002F085FDAF482988018073E0607B85F8A1
:10879000E0002D20C6E5AC48D4F80D1040F82D1FA0
:1087A000D4F811104160B4F8151001812E20B9E5FC
:1087B000607B85F8EB0018B1A44981F800B005E0B2
:1087C000A3480670A3480680A04806702F20A9E59C
:1087D0009D48D4F80D108163D4F81110C163302086
:1087E000A0E59948D4F80D10016431209AE5B4F859
:1087F0000D0041BAB4F80F0040BA61F31F40C5F84C
:10880000F80032208EE5607B85F80B0132E0B4F889
:108810000D0041BAB4F80F0040BA61F31F40C5F82B
:108820000C0134207EE5182204F10D015A980AF05B
:1088300035FF352002F02BFD362002F028FD3720D1
:1088400002F025FD38206DE5607B85F828010128C0
:1088500010D15C4688F802B0FEF74DFFFFF7EEF846
:1088600084F310885BE0607B85F82901012801D141
:1088700003F09AFE0120CDE9000ADDE95E018DF8E2
:10888000089002AB5B9AFFF715FC98F802100129DB
:1088900040D026E3B4F80D0040BAA5F82A013B20E9
:1088A00040E5B4F80D0040BAA5F82C013C2039E5AC
:1088B000607B85F82E013D2034E5607B85F8300132
:1088C0003F202FE5607B85F8310140202AE5B4F890
:1088D0000D0040BAA5F83201412023E5B4F80D009F
:1088E00040BAA5F8340142201CE5B4F80D0040BAA6
:1088F000A5F83601432015E5B4F80D0040BAA5F8F7
:10890000380144200EE5B4F80D0040BAA5F83A014C
:10891000452007E588F80260012080F3108801F007
:108920001FFB98F800000028B3D04FF0010819464B
:1089300002A80AF0CCFEA9F17900502840D2DFE865
:1089400000F0283F3F3F3F3F3F404346494C4F5296
:10895000585B5E65689194979A9DA0A3A6A9ACAF59
:10896000B2B6B9BCBFC2C5F0F3F6F9FCFFE9E8E75F
:10897000E6E5E4E3E2E1E0DFDEDDDCDBDAD9D8D70F
:10898000D6D5D4D33F3F3FD2D1D0CFCECDCCCBCA9A
:10899000C9C8002002AEB5F890300BE000EB4002F1
:1089A000511932448F7E5770CF7E9770097F401CDB
:1089B000D170C0B28342F1D803EB4300401C87B2B0
:1089C0003BE1B5F87A007AE1B5F87C0077E1B5F8DB
:1089D0007E0074E1B5F8800071E1B5F882006EE1C7
:1089E00095F8840001E095F885008DF809000227CC
:1089F00023E1B5F8860062E1B5F888005FE116482A
:108A00008DF809608DF80A600088B1E0B5F8900033
:108A100055E112490878012802D0B5F892004EE1DC
:108A20000F480088020A8DF809208DF80A000E70A0
:108A3000032702E167000020740000206500002089
:108A40007700002042000020940F0020000000204A
:108A50007D000020A00000202E03002078000020D0
:108A60009E000020B5F8940029E1B5F8960026E1B3
:108A7000B5F8980023E1B5F89A0020E1B5F89C001C
:108A80001DE1B5F89E001AE1B5F8A00017E1B5F8B0
:108A9000A20014E1B5F8A40011E1B5F8A6000EE1BA
:108AA000B5F8A8000BE1B5F8AA0008E1FEE3B5F8B7
:108AB000AC0004E1B5F8AE0001E1B5F8B000FEE0AD
:108AC000B5F8B200FBE0B5F8B400F8E095F8B600F0
:108AD0008BE7F2E0EEE0EAE0E6E0E2E0DEE0DAE0BA
:108AE000D6E0D2E0C0E0AFE0A0E096E092E084E023
:108AF00080E073E069E065E057E053E04FE04BE071
:108B000047E043E03FE03BE02FE02BE027E023E0BD
:108B10001FE01BE017E013E00FE00BE007E003E0CD
:108B2000FFE7B5F8B800CAE0B5F8BA00C7E0B5F895
:108B3000BC00C4E0B5F8BE00C1E0B5F8C000BEE0BE
:108B4000B5F8C200BBE0B5F8C600B8E0B5F8CA0099
:108B5000B5E0B5F8CC00B2E0B5F8CE00AFE0B5F8BE
:108B6000D000ACE095F8D2003FE7D5F8D40056E04D
:108B7000010A8DF80B1000BF8DF80C0005275CE092
:108B800095F8D80031E795F8D9002EE7B5F8DA0066
:108B900095E095F8DC0028E795F8DD0025E7B5F8C5
:108BA000DE008CE095F8E0001FE7FE480B2750F848
:108BB0002D1FCDF809104168CDF80D100089ADF8D2
:108BC00011003AE095F8EB000FE7F6480927816BB2
:108BD000CDF80910C06BCDF80D002EE015F8F40F9C
:108BE0008DF8090068788DF80A00A8788DF80B00D8
:108BF000E878C1E7D5F8F80011E00F22EA4961985A
:108C00000AF04CFD0F220DF1090061990AF046FDB2
:108C1000102712E095F80B01E7E6D5F80C01010EDC
:108C20008DF80910010C8DF80A10A1E718220DF13A
:108C300009005A990AF032FD1927CDE9007A8DF81A
:108C4000089002AB4246FDE39DF809205D98BE21E5
:108C50001154B5F82A019DF809306599020A5A5451
:108C60009DF8092064990EE09DF809206098BF21C5
:108C70001154B5F82C019DF809306399020A5A5431
:108C80009DF8092062995054D2E695F82E01ACE681
:108C900095F82F01A9E695F83001A6E695F831017F
:108CA000A3E6B5F832010AE0B5F8340107E0B5F8FB
:108CB000360104E0B5F8380101E0B5F83A01010ADF
:108CC0008DF809108DF80A00B2E6B8484946B9F1A6
:108CD000E00F05D0E1293ED0B9F1E20F6AD15AE0A8
:108CE0000178627B914216D14178A27B914212D1E8
:108CF0008178E27B91420ED1C178227C91420AD1E7
:108D00000179627C914206D14079A17C884202D1EE
:108D10008DF809B01CE0A5488DF809600E30627B23
:108D20000178914234D14178A27B914230D181784F
:108D3000E27B91422CD1C178227C914228D10179E9
:108D4000627C914224D14079A17C8842E0D01FE02E
:108D500088F805602EE00178627B914218D1417855
:108D6000A27B914214D18178E27B914210D1C178EB
:108D7000227C91420CD10179627C914208D14079E8
:108D8000A17C884204D18DF809B088F805B011E0C3
:108D90008DF80960DCE7D4F80D20C8F81720B4F886
:108DA0001120A8F81B2098F805200021012A07D0DF
:108DB0008DF8096001228DF80890022002ABFDE3D6
:108DC0007A4AD21D535C4354491CC9B20629F9D3CF
:108DD0003A2002F05CFA88F805608DF809B0E9E7FE
:108DE00098F8000000287CD04FF00108194602A82E
:108DF0000AF06DFC79208DF80800B5F8901002AFEC
:108E000001EB41008DF8090000200FE000EB40036A
:108E10005A193B4492F81AC083F802C092F81BC05A
:108E200083F803C0127F401C1A71C0B28142EDD892
:108E30009DF80930B81C80221A54B5F87A009DF8C4
:108E400009700DF10B02030ABB549DF8093003AA07
:108E500098549DF809300DF10D0081221A54B5F88F
:108E60007C009DF809700DF10E02030ABB549DF8B9
:108E70000930521C98549DF8093004A882221A54D3
:108E8000B5F87E009DF809700DF11102030ABB547C
:108E90009DF80930521C98549DF809300DF11300CB
:108EA00083221A54B5F880009DF8097005AA030AB8
:108EB000BB549DF80930521C98549DF809300DF1AF
:108EC000160084221A54B5F882009DF809700DF13D
:108ED0001702030ABB549DF8093006AA985485224C
:108EE00000E0FCE39DF809300DF119001A549DF8DB
:108EF0000930401C95F884201A549DF80930401C14
:108F000086221A549DF8093007A895F885201A542E
:108F10009DF80930401C87221A54B5F886009DF848
:108F200009700DF11E02030ABB549DF80930521C52
:108F300098549DF8093008A889221A549DF80920F0
:108F4000401C16549DF80920401C165418489DF8E2
:108F500009700DF123020088030ABB549DF8093003
:108F600009AA98549DF809300DF125008A221A5457
:108F70009DF80930401C0A0A1A549DF80920401C2B
:108F80000C4B11549DF809200AA88B2111541A7812
:108F9000411C801C012A7DD0B5F892209DF8096003
:108FA000130A09E0940F002044000020E40200208E
:108FB0002E0300207800002073549DF809100A54F5
:108FC0009DF809200DF12B008C21115435F8940FD8
:108FD0009DF809300BA9020A5A549DF80920491C32
:108FE00050549DF809200DF12E008E211154A888AF
:108FF0009DF809300DF12F01020A5A549DF80920FD
:109000000CA950549DF809200DF131008F21115405
:10901000E8889DF809300DF13201020A5A549DF892
:109020000920491C50549DF809200DA89021115485
:1090300028899DF809300DF13501020A5A549DF82E
:109040000920491C50549DF809200DF13700912149
:10905000115468899DF809300EA9020A5A549DF8E6
:109060000920491C50549DF809200DF13A00922125
:109070001154A8899DF809300DF13B01020A5A5498
:109080009DF809200FA950549DF8092093210DF156
:109090003D0000E03CE31154E8899DF809300DF1F2
:1090A0003E01020A5A549DF80920491C50549DF86B
:1090B000092010A894211154288A9DF809300DF137
:1090C0004101020A5A549DF80920491C50549DF848
:1090D00009200DF1430095211154688A9DF809304B
:1090E00011A9020A5A549DF80920491C50549DF8B0
:1090F00009200DF1460096211154A88A9DF80930E7
:109100000DF14701020A5A549DF8092012A9505442
:109110009DF809200DF1490097211154E88A9DF826
:1091200009300DF14A01020A5A549DF80920491CE0
:1091300050549DF8092013A898211154288B9DF8AC
:1091400009300DF14D01020A5A549DF80920491CBD
:1091500050549DF809200DF14F0099211154688B4E
:10916000020A9DF8093014A95A549DF80920491C97
:1091700050549DF809200DF152009A211154A88BEA
:109180009DF809300DF15301020A5A549DF8092047
:1091900015A950549DF809200DF155009B2111543B
:1091A000E88B9DF809300DF15601020A5A549DF8DA
:1091B0000920491C50549DF8092016A89C211154DF
:1091C000288C9DF809300DF15901020A5A549DF876
:1091D0000920491C50549DF809200DF15B009D2188
:1091E00011549DF8092017A895F8221011549DF8E4
:1091F0000920401C9E211154A88C9DF809300DF1C6
:109200005E01020A5A549DF80920491C50549DF8E9
:10921000092018A89F211154E88C9DF809300DF100
:109220006101020A5A549DF80920491C5054A0219A
:109230009DF809200DF163001154288D9DF8093027
:1092400019A9020A5A549DF80920491C50549DF846
:1092500009200DF16600A1211154688D9DF8093097
:109260000DF16701020A5A549DF809201AA95054B9
:109270009DF809200DF16900A2211154A88D9DF8D7
:1092800009300DF16A01020A5A549DF80920491C5F
:1092900050549DF809201BA8A3211154E88D9DF876
:1092A00009300DF16D01020A5A5400E0F7E39DF810
:1092B0000920491C50549DF809200DF16F00A4218C
:1092C0001154688E9DF809301CA9020A5A549DF861
:1092D0000920491C50549DF809200DF17200A52168
:1092E0001154E88E9DF809300DF17301020A5A54A9
:1092F0009DF809201DA950549DF809200DF1750015
:10930000A6211154288F9DF809300DF17601020A2B
:109310005A549DF80920491C50549DF809201EA854
:10932000A7211154688F9DF809300DF17901020AC7
:109330005A549DF80920491C50549DF809200DF1FC
:109340007B00A8211154A88F9DF809301FA9020A9B
:109350005A549DF80920491C50549DF809200DF1DC
:109360007E00A92111549DF80920401C95F83E105B
:1093700011549DF8092020A8AA211154286C9DF8A9
:1093800009300DF18101020E5A549DF80930491C33
:10939000020C5A549DF80930491C020A5A549DF88F
:1093A000092021A950549DF809200DF18500AB2119
:1093B00011549DF80920401C95F8441011549DF853
:1093C0000920401CAC2111549DF8092022A895F8D1
:1093D000451011549DF80920401CAD211154B5F8D9
:1093E00046009DF809300DF18A01020A5A549DF891
:1093F0000920491C50549DF8092023A8AE2111547E
:109400009DF80920401C95F8481011549DF809203A
:10941000401CAF2111549DF80920401C95F84910BB
:1094200011549DF8092024A8B0211154B5F84A0020
:109430009DF809300DF19101020A5A549DF8092056
:10944000491C00E0FDE350549DF809200DF1930004
:10945000B12111549DF8092025A895F84C101154FC
:109460009DF80920401CB22111549DF80910401CA0
:109470000144FE48D0F82D200A60D0F831204A601F
:10948000B0F835200A819DF8093028A9B3225A5432
:109490009DF80930491C95F857205A549DF8093019
:1094A000491CB4225A549DF80920491C1144826B6E
:1094B0000A60C06B48609DF809200DF1AB00B52132
:1094C00011549DF809202BA895F8601011549DF8AF
:1094D0000920401C95F8611011549DF80920401C8A
:1094E00095F8621011549DF80920401C95F86310FE
:1094F00011549DF809202CA8B6211154686E9DF8CE
:1095000009300DF1B101020E5A54020C9DF80930D8
:10951000491C5A549DF80930491C020A5A549DF8B6
:1095200009202DA950549DF809200DF1B500B7214F
:1095300011540F22CE4961980AF0B0F89DF8091035
:109540000DF1B60008440F2261990AF0A7F89DF8C2
:1095500009200DF1C500B82111549DF80920401CC7
:1095600095F8771011549DF80920401CB921115429
:10957000A86F9DF8093032A9020E5A549DF809309F
:10958000491C020C5A549DF80930491C020A5A54CD
:109590009DF80920491C50549DF8092033A8BA2190
:1095A00011549DF80910401C084418225A990AF0D9
:1095B00075F89DF80900BE225D9900E0A5E04254CF
:1095C000B5F896009DF809306599020A5A549DF83D
:1095D0000920649950549DF809206098BF211154C6
:1095E000B5F898009DF809306399020A5A549DF81D
:1095F0000920629950549DF809203BA8C0211154BC
:109600009DF80920401C95F89A1011549DF80920E6
:10961000401CC12111549DF80920401C95F89B1055
:1096200011549DF809203CA8C22111549DF809202D
:10963000401C95F89C1011549DF80920401CC32132
:1096400011549DF80920401C95F89D1011549DF867
:1096500009203DA8C4211154B5F89E009DF8093099
:109660000DF1F501020A5A549DF80920491C505485
:109670009DF809200DF1F700C5211154B5F8A0009F
:109680009DF809303EA9020A5A549DF80920491C48
:1096900050549DF809200DF1FA00C6211154B5F877
:1096A000A2009DF809300DF1FB01020A5A549DF801
:1096B00009203FA950549DF809200DF1FD00C72154
:1096C0001154B5F8A4009DF809300DF1FE01020A0D
:1096D0005A549DF80920491C5054C82100E0A4E0C8
:1096E0009DF8092040A81154B5F8A6009DF809304E
:1096F0000DF20111020A5A549DF80920491C02ABCF
:1097000050549DF809004246FB30CDE9000ACDE3F4
:10971000584A9DF809C01288170A0CF801709DF884
:1097200009100A541E704BE45348007800287CD07E
:109730004FF0000801205B90C1464746194602A839
:1097400009F0C5FF207B8E2805D1B4F80D00032752
:1097500040BAA5F89800E019017B8F2905D1B0F82F
:109760000D00FF1C40BAA5F89A00E01940F6C4119C
:10977000027B902A0BD1B0F80D003F4A40BA10810D
:10978000A0F5FA628A4250D8A5F89C00FF1CE019A7
:10979000027B912A0BD1B0F80D00374A40BA5081B4
:1097A000A0F5FA628A42EED8A5F89E00FF1CE019E7
:1097B000017B922905D1B0F80D00FF1C40BAA5F835
:1097C000A000E01940F62821027B932A0BD1B0F8C3
:1097D0000D00294A40BA9081A0F57A728A42D2D807
:1097E000A5F8A200FF1CE019027B942A0BD1B0F867
:1097F0000D00214A40BAD081A0F57A728A42C2D8BF
:10980000A5F8A400FF1CE019017B952905D1B0F84B
:109810000D00FF1C40BAA5F8A600E019017B9629AF
:1098200007D1B0F80D0040BA00E043E3A5F8A80066
:10983000FF1CE019017B972905D1B0F80D00FF1C32
:1098400040BAA5F8AA00E019017B982905D1B0F823
:109850000D00FF1C40BAA5F8AC00E019017B992966
:109860000FD1B0F80D0040BA08E00000940F0020BE
:10987000440000209E000020D4020020A5F8AE0085
:10988000FF1CE019017B9A2905D1B0F80D00FF1CDF
:1098900040BAA5F8B000E019017B9B2905D1B0F8CA
:1098A0000D00FF1C40BAA5F8B200E019017B9C290D
:1098B00005D1B0F80D00FF1C40BAA5F8B400E019BE
:1098C000017B9D2904D1407BBF1C85F8B600BFB247
:1098D000E019017B9E2906D1B0F80D00FF1C40BAAB
:1098E000A5F8B800BFB2E019017B9F2906D1B0F8F6
:1098F0000D00FF1C40BAA5F8BA00BFB2E019017B09
:10990000A02906D1B0F80D00FF1C40BAA5F8BC0094
:10991000BFB2E019017BA12906D1B0F80D00FF1CF0
:1099200040BAA5F8BE00BFB2E019017BA22906D15A
:10993000B0F80D00FF1C40BAA5F8C000BFB2E01996
:10994000017BA32906D1B0F80D00FF1C40BAA5F891
:10995000C200BFB2E019017BA42906D1B0F80D0006
:10996000FF1C40BAA5F8C600BFB2E019017BA529CB
:1099700006D1B0F80D00FF1C40BAA5F8CA00BFB26E
:10998000E019017BA62906D1B0F80D00FF1C40BAF2
:10999000A5F8CC00BFB2E019017BA72906D1B0F829
:1099A0000D00FF1C40BAA5F8CE00BFB2E019017B44
:1099B000A82906D1B0F80D00FF1C40BAA5F8D000C8
:1099C000BFB2E019017BA9292CD1FA4990F80D907A
:1099D00049680A68F74B9B681A430A60F649CE70DB
:1099E0000E71407B00F00F01F348C1701420FDF7A9
:1099F000CDFAF248F049807EC97800F0F0000843C3
:109A0000ED490A1D087101210020FDF7A1FEE9487A
:109A100040680168E74A926891430160FDF76BFE78
:109A2000BF1CBFB2E019017BAA2920D1B0F80D10EC
:109A30004ABAB0F80F1049BA62F31F41D5F8D420E2
:109A4000914203D0DE490E70DE490E7030F80D1FD2
:109A50007F1D408849BA40BA61F31F40C5F8D40061
:109A6000D5F80C11BFB2814201D9C5F80C01E0193B
:109A7000017BAB290ED1407B85F8D80001280FD09F
:109A8000D14981F800B0F9F7D5FBD04981F800B091
:109A9000BF1CBFB2E019017BAC290FD01DE01DE255
:109AA000C9480670C948007818B1C948007800282C
:109AB000EED1F9F7D6FBC5480670E9E7407B85F89B
:109AC000D90001280ED0C34981F800B0F9F73AFB5C
:109AD000C14981F800B0BF1CBFB2E019017BAD29BC
:109AE0000ED014E0BB480670BB48007818B1BB48E4
:109AF00000780028EFD1F9F743FBB7480670EAE792
:109B0000B0F80D00FF1C40BAA5F8DA00BFB2E019AA
:109B1000017BAE2904D1407BBF1C85F8DC00BFB2BD
:109B2000E019017BAF2903D190F80D80BF1CBFB2B3
:109B3000E019017BB02908D1B0F80D00A84940BA5E
:109B4000A5F8DE00FF1CBFB20880E019017BB12937
:109B500004D1407BBF1C85F8E000BFB2E019017B57
:109B6000B2290AD19F4950F80D2F0B3741F82D2FFC
:109B700042684A6000890881BFB2E019017BB329BD
:109B800012D1407BBF1C85F8EB00BFB218B19649DB
:109B900081F800B005E09448067094480670944837
:109BA00006802F2001F073FBE019017BB42907D157
:109BB0008C4950F80D2F09378A634068BFB2C863DB
:109BC000E019017BB52905D18649D0F80D007F1D2C
:109BD000BFB20864E019017BB6290AD130F80D1F25
:109BE0007F1D408849BA40BA61F31F40BFB2C5F833
:109BF000F800E019017BB82904D1407BBF1C85F82F
:109C00000B01BFB2E019017BB9290AD130F80D1F51
:109C10007F1D408849BA40BA61F31F40BFB2C5F802
:109C20000C01E119087BBA2806D118220D315A9887
:109C300009F034FD1937BFB2E019017BBE2908D104
:109C400000E033E1B0F80D00FF1C40BAA5F82A018E
:109C5000BFB2E019017BBF2906D1B0F80D00FF1C8F
:109C600040BAA5F82C01BFB2E019017BC02904D18C
:109C7000407BBF1C85F82E01BFB2E019017BC229D1
:109C800004D1407BBF1C85F83001BFB2E019017BD5
:109C9000C32904D1407BBF1C85F83101BFB2E01954
:109CA000017BC42906D1B0F80D00FF1C40BAA5F80D
:109CB0003201BFB2E019017BC52906D1B0F80D0011
:109CC000FF1C40BAA5F83401BFB2E019017BC629D8
:109CD00006D1B0F80D00FF1C40BAA5F83601BFB29E
:109CE000E019017BC72906D1B0F80D00FF1C40BA6E
:109CF000A5F83801BFB2E019017BC82904D1B0F83A
:109D00000D0040BAA5F83A0195F8DD1041450AD09A
:109D10002C48B8F1000F067006D0B8F1010F25D01D
:109D2000B8F1020F66D089E040F6426025F89C0F3A
:109D30000420A8804FF4616169804FF42F61E980AD
:109D4000688140F654312981142169824021A98219
:109D50003C21E98129825021A5F89A10A5F89C00A0
:109D60004FF47A70A88140F6E4401FE041F26800A9
:109D700025F89C0F0420A88041F2040169804FF46B
:109D80002F61E980688140F654312981142169826C
:109D90004021A9823C21E98129825021A5F89A100D
:109DA000A5F89C004FF47A70A8818000E8820A2010
:109DB00042E01FE07C0A0020D4020020300B00208B
:109DC000760000207700002066000020730000204D
:109DD000640000206700002074000020650000205F
:109DE00042000020940F0020000000207D00002091
:109DF000A000002040F6FC0025F89C0F0420A8805D
:109E000040F6CA01698040F2DC51E98068814FF474
:109E1000C8612981142169824021A9823C21E981FC
:109E200029825021A5F89A10A5F89C004FF47A7069
:109E3000A8814000E882052028839C3D484695F88B
:109E4000D210494524D009F0C8FE0646B5F89C005A
:109E50000F46983509F0C1FEDFF818B100225B46C5
:109E600009F02DFE32463B4609F0B7FD09F0EFFE42
:109E70002880688909F0B1FE00225B4609F01FFEC8
:109E80003B46324609F0A9FD09F0E1FE6880983DA5
:109E900085F8DD8085F8D29002F073F8FF208DF808
:109EA00008000120CDE9000A5B9A02ABDDE95E0102
:109EB000FEF700F90DE098F8000050B1B9F1010F7C
:109EC00007D1607B88F80100012800D00020FCF752
:109ED00006FF40F26311601C09F0F9FB69B0BDE8B0
:109EE000F08F254810B5007801280ED12248FEF7E2
:109EF00069F922490020244A8871214908702149C2
:109F0000B1F8DE1011802149088010BD204810B53D
:109F1000007801280AD11E48FEF754F91D49002097
:109F2000087018481849B0F8DE00088010BD10B558
:109F3000194C94F82300012811D1002084F8230043
:109F400084F82200201DFDF77BF81E21201D09F05A
:109F5000BEFBBDE810404FF4FA70FDF717B810BD16
:109F60000E4801680E4A01F4E06111430160BFF33D
:109F70004F8FFEE700002440140C0020D402002084
:109F800040010020E00E00204200002012000020CE
:109F90007A0D002042010020101A00200CED00E094
:109FA0000400FA05204810B50178012928D10021C4
:109FB00001700A4608461D490B5C401C1A44C0B299
:109FC000D2B21B28F8D3C87E904219D11648182265
:109FD000401CC91C09F062FB13491822491C144893
:109FE00009F05CFB352001F052F9362001F04FF901
:109FF000372001F04CF9BDE81040382001F047B996
:10A0000010BD0C4810B5007801280CD10948FEF7A6
:10A01000D9F8094900200A4A08700849B1F8DE1049
:10A0200011800849088010BD13030020DE140020B1
:10A03000F00F00201C10002041010020E00E002045
:10A0400042000020120000202DE9F04F87B04FF4AD
:10A05000FA62F849F84805F037FFF748F749322720
:10A06000027800250126AA2A02D14278552A07D073
:10A070000D70F3490F70827AF249AA2A05D007E0E1
:10A080000E70EF4982780A70F5E7C27A552A0BD034
:10A09000A1F8005090F814C0EB496422EB4BEC4C53
:10A0A000BCF1AA0F04D008E0828952BA0A80F1E715
:10A0B00090F815C0BCF1550F06D00D601A80827F54
:10A0C000E449AA2A0FD011E0B0F816C0B0F8188001
:10A0D0009CFA9CFC98FA98F86CF31F48C1F8008031
:10A0E000C4F88C80EAE7C27F552A07D081F8006067
:10A0F00090F82820D849AA2A04D007E090F8202018
:10A100000A70F5E790F82920552A07D081F80060F9
:10A1100090F83220D149AA2A04D007E090F82A20EA
:10A120000A70F5E790F83320552A07D081F80060CF
:10A1300090F83C20CA49AA2A04D007E090F83420BD
:10A140000A70F5E790F83D20552A07D081F80060A5
:10A1500090F84620C349AA2A04D007E090F83E2090
:10A160000A70F5E790F84720552A07D081F800607B
:10A1700090F85020BC49AA2A04D007E090F8482063
:10A180000A70F5E790F85120552A07D081F8006051
:10A1900090F85A20B549AA2A04D007E090F8522036
:10A1A0000A70F5E790F85B20552A06D081F8006028
:10A1B00090F87810AA2904D007E090F85C200A7083
:10A1C000F6E790F87910552909D041F2680100BFEF
:10A1D000A4F89C1090F88210AA2904D007E0B0F8E7
:10A1E0007A1049BAF4E790F88310552909D041F262
:10A1F000040100BFA4F89E1090F88C10AA2904D086
:10A2000007E0B0F8841049BAF4E790F88D105529AA
:10A2100007D00421A4F8A01090F89610AA2904D021
:10A2200007E0B0F88E1049BAF4E790F89710552976
:10A2300009D04FF42F6100BFA4F8A21090F8A0102D
:10A24000AA2904D007E0B0F8981049BAF4E790F8CA
:10A25000A110552909D040F6543100BFA4F8A4102C
:10A2600090F8AA10AA2904D007E0B0F8A21049BAC1
:10A27000F4E790F8AB10552907D00421A4F8A610F4
:10A2800090F8B410AA2904D007E0B0F8AC1049BA8D
:10A29000F4E790F8B51055290AD04FF47A7100BF51
:10A2A000A4F8A81090F8BE203C21AA2A04D007E008
:10A2B000B0F8B61049BAF3E790F8BF20552A06D097
:10A2C000A4F8AA1090F8C820AA2A06D009E0B0F88D
:10A2D000C02052BAA4F8AA20F4E790F8C920552A61
:10A2E00009D0A4F8AC1000BF90F8D2204FF0140BA6
:10A2F000AA2A06D009E0B0F8CA2052BAA4F8AC20C5
:10A30000F2E790F8D320552A07D0A4F8AEB000BFEA
:10A3100090F8DC20AA2A06D009E0B0F8D42052BA7E
:10A32000A4F8AE20F4E790F8DD20552A09D04022A9
:10A33000A4F8B02090F8E6204FF47A6AAA2A04D054
:10A3400007E0B0F8DE2052BAF2E790F8E720552A8D
:10A3500009D0A4F8B2A000BF90F8F0204FF00A098D
:10A36000AA2A06D009E0B0F8E82052BAA4F8B22030
:10A37000F2E790F8F120552A07D0A4F8B49000BF76
:10A3800090F8FA20AA2A06D009E0B0F8F22052BAD2
:10A39000A4F8B420F4E790F8FB20552A07D084F8FD
:10A3A000B66000BF90F80421AA2A05D008E090F812
:10A3B000FC2084F8B620F5E790F80521552A08D04E
:10A3C0005FF04B02A4F8B82090F80E21AA2A04D01E
:10A3D0000AE0B0F8062152BAF4E790F80F21552AA6
:10A3E00002D1B0F8101149BAA4F8BA1090F81821A7
:10A3F0004121AA2A03D190F81921552A07D0A4F89F
:10A40000BC1000BF90F82221AA2A06D009E0B0F8BB
:10A410001A2152BAA4F8BC20F4E790F82321552A57
:10A4200026D03722A4F8BE2090F82C21AA2A23D0C7
:10A4300026E0000000F00108FA1400207600002059
:10A440006A00002010010020D40000202E0300200C
:10A45000E00E00206C0000206D0000206E00002047
:10A460006F000020700000207100002072000020AA
:10A47000B0F8242152BAD5E790F82D21552A06D0FC
:10A48000A4F8C0B090F83621AA2A06D009E0B0F8A6
:10A490002E2152BAA4F8C020F4E790F83721552AAB
:10A4A00007D0A4F8C21000BF90F84021AA2A06D015
:10A4B0000CE0B0F8382152BAA4F8C220F4E790F8C2
:10A4C0004121552A02D1B0F8421149BAA4F8C61068
:10A4D00090F84A116FF02702AA2903D190F84B1186
:10A4E000552908D0A4F8CA2090F854316FF0220101
:10A4F000AA2B06D009E0B0F84C1149BAA4F8CA104A
:10A50000F2E790F85531552B07D0A4F8CC1000BFD6
:10A5100090F85E31AA2B06D00CE0B0F856315BBA49
:10A52000A4F8CC30F4E790F85F31552B02D1B0F8A5
:10A53000602152BAA4F8CE2090F86821AA2A06D148
:10A5400090F86921552A02D1B0F86A1149BAA4F8E5
:10A55000D01090F87211AA2903D190F873115529DF
:10A5600008D0102184F8D210804690F86400AA2800
:10A5700003D006E090F87411F4E798F865105529B7
:10A580001BD094F8D20009F028FB00910290B4F897
:10A590009C0009F022FB0022FD4B09F090FA009B81
:10A5A000029A09F01AFA09F052FB00BFA4F89800C9
:10A5B00098F86E00AA2804D007E0B8F8660040BA00
:10A5C000F4E798F86F1055291BD094F8D20009F0E1
:10A5D00004FBCDE90001B4F8A20009F0FEFA002264
:10A5E000EB4B09F06CFADDE9002309F0F6F909F00C
:10A5F0002EFB00BFA4F89A0098F87C01AA2804D08A
:10A6000007E0B8F8700040BAF4E798F87D015528E3
:10A6100007D02820C4F8D40098F88601AA2809D0C9
:10A620000CE0B8F87E0141BAB8F8800140BA61F395
:10A630001F40EFE798F88701552804D0D5480570EA
:10A6400084F8D86007E0D34998F88801087000289A
:10A65000F6D084F8D85098F89001AA2803D198F839
:10A660009101552805D0CC4880F8005084F8D96075
:10A6700007E0C94998F8920108700028F6D084F8DC
:10A68000D95098F89A0142F2107EAA2803D198F87E
:10A690009B01552807D0A4F8DAE000BF98F8A40180
:10A6A000AA2806D009E0B8F89C0140BAA4F8DA005C
:10A6B000F4E798F8A501552807D084F8DC6000BFBE
:10A6C00098F8AE01AA2805D008E098F8A60184F809
:10A6D000DC00F5E798F8AF01552806D084F8DD6076
:10A6E00098F8B801AA2805D008E098F8B00184F8D5
:10A6F000DD00F5E798F8B901552808D05FF00F00A4
:10A70000A4F8DE0098F8C201AA2804D007E0B8F83F
:10A71000BA0140BAF4E798F8C301552809D084F883
:10A72000E09000BF98F8CC019C499D4AAA2805D02A
:10A7300008E098F8C40184F8E000F3E798F8CD0148
:10A7400055280AD09648803840F8E15FC0F8045098
:10A7500098F8D601AA280AD00DE09148D1F84E30D9
:10A76000803840F8E13FD1F852304360F0E798F884
:10A77000D701552808D084F8EB5000BF98F8E03195
:10A780008848AA2B0AD00DE098F8D801864B84F8A7
:10A79000EB0008B11E70F1E71D70EFE798F8E131AA
:10A7A000552B14D07E4BB0F802C0803BA3F8ECC010
:10A7B00090F804C083F8EEC0D0F8093042F86F3F3B
:10A7C000437B137198F8EA21AA2A0AD00DE0744A53
:10A7D000D1F86230803A42F8EC3FD1F866305360ED
:10A7E000F0E798F8EB21552A0BD06D49D0F8050019
:10A7F0008039C1F8F40000BF98F8F401AA2806D007
:10A8000009E06748C96E8038C0F8F410F4E798F89A
:10A81000F501552808D0C4F8F85000BF98F8FE019B
:10A820006249AA280BD00EE0B8F8F60141BAB8F890
:10A83000F80140BA61F31F40C4F8F800EEE798F859
:10A84000FF01552806D05A48086098F80802AA283F
:10A8500009D00CE0B8F8000242BAB8F8020240BAD7
:10A8600062F31F40F0E798F80902552812D0D4F897
:10A87000D400C4F80C010146D4F8D400814201D9B7
:10A88000C4F80C01454998F812324A4A8031AA2B83
:10A8900009D00CE0B8F80A0241BAB8F80C0240BA84
:10A8A00061F31F40E5E798F81332552B13D03C4B6A
:10A8B000D2F800C0803BC3F810C1D2F804C0C3F87E
:10A8C00014C192F808C083F818C100BF98F81C3270
:10A8D000AA2B0BD00EE0324BD1F814C0803BC3F84A
:10A8E00010C1D1F818C0C3F814C1EFE798F81D32B1
:10A8F000552B0ED02A4BD2F809C0803BC3F819C1A2
:10A90000B2F80DC0A3F81DC198F82632AA2B0FD0BB
:10A9100012E0234BD1F81EC0803BC3F818C1B1F838
:10A9200022C0A3F81CC191F824C083F81EC1EBE734
:10A9300098F82732552B0ED0194BD2F80FC0803B18
:10A94000C3F81FC1B2F813C0A3F823C198F830327E
:10A95000AA2B09D00CE0124BD1F828C0803BC3F8D9
:10A960001FC1B1F82CC0EFE798F83132552B23D036
:10A970000B4BB2F815C0803BA3F825C1D27D83F8FC
:10A98000272100BF98F84422AA2A1ED027E0000001
:10A990000000244066000020670000207A16002096
:10A9A000600F0020F902002000000020D8000020E5
:10A9B0009738F23914030020F94A4B8EA2F825315A
:10A9C00091F8343082F82731DCE798F84522552A8F
:10A9D00005D1F44A51F8463F13608988918098F870
:10A9E0004E12AA2903D198F84F12552909D094F88C
:10A9F000DD1040F6BE2251B1012908D0022906D04F
:10AA000007E0B8F8501249BAA4F82A1101E0A4F8F6
:10AA10002A2198F85812AA2903D198F859125529D1
:10AA200009D094F8DD1040F6223251B1012908D046
:10AA3000022906D007E0B8F85A1249BAA4F82C1136
:10AA400001E0A4F82C2198F86212AA2903D198F801
:10AA50006312552907D084F82E5100BF98F86C1264
:10AA6000AA2905D00CE098F8641284F82E11F5E7B5
:10AA700098F86D12552903D198F86E1284F82F11A9
:10AA800098F87612AA2903D198F87712552908D098
:10AA90005FF05A0184F8301198F88012AA2903D087
:10AAA00006E098F87812F5E798F88112552908D051
:10AAB0005FF0260184F8311198F88A12AA2903D090
:10AAC00006E098F88212F5E798F88B12552908D01D
:10AAD0004FF4C871A4F8321198F89412AA2904D03E
:10AAE00007E0B8F88C1249BAF4E798F8951255299E
:10AAF00007D0A4F8345100BF98F89E12AA2906D0B6
:10AB000009E0B8F8961249BAA4F83411F4E798F8B5
:10AB10009F12552907D05021A4F8361198F8A81291
:10AB2000AA2904D007E0B8F8A01249BAF4E798F8C7
:10AB3000A912552907D00421A4F8381198F8B212A7
:10AB4000AA2904D007E0B8F8AA1249BAF4E798F89D
:10AB5000B31255290AD040F6165100BFA4F83A1195
:10AB600098F8BC229049AA2A04D007E0B8F8B41299
:10AB700049BAF3E798F8BD22552A07D041F2883246
:10AB80000A8098F8C622AA2A04D007E0B8F8BE22A4
:10AB900052BAF5E798F8C722552A07D041F2941225
:10ABA0004A8098F8D022AA2A04D007E0B8F8C82230
:10ABB00052BAF5E798F8D122552A06D0A1F804A098
:10ABC00098F8DA22AA2A05D008E0B8F8D22252BAB8
:10ABD0008A80F5E798F8DB22552A07D041F2CC02AB
:10ABE000CA8098F8E422AA2A04D007E0B8F8DC2248
:10ABF00052BAF5E798F8E522552A07D041F26802E3
:10AC00000A8198F8EE22AA2A04D007E0B8F8E622D2
:10AC100052BAF5E798F8EF22552A06D0A1F80AA013
:10AC200098F8F822AA2A05D008E0B8F8F02252BA1B
:10AC30004A81F5E798F8F922552A07D040F6B8324C
:10AC40008A8198F80223AA2A04D007E0B8F8FA22E9
:10AC500052BAF5E798F80323552A0AD040F6AC52C9
:10AC6000CA8198F80C3342464FF44878AA2B04D096
:10AC700007E0B8F8042352BAF2E792F80D33552BE7
:10AC800007D0A1F8108000BF92F81633AA2B05D088
:10AC900008E0B2F80E335BBA0B82F5E792F817338F
:10ACA000552B07D04FF416734B8292F82033AA2B02
:10ACB00004D007E0B2F818335BBAF5E792F8213315
:10ACC000552B06D0A1F814E092F82A33AA2B05D010
:10ACD00008E0B2F822335BBA8B82F5E792F82B33A7
:10ACE000552B07D04FF4FA53CB8292F83433AA2B6A
:10ACF00004D007E0B2F82C335BBAF5E792F83533AD
:10AD0000552B07D044F620630B8392F83E33AA2BD1
:10AD100004D007E0B2F836335BBAF5E792F83F3378
:10AD2000552B07D044F250634B8392F84833AA2B3B
:10AD300004D007E0B2F840335BBAF5E792F8493344
:10AD4000552B08D0A1F81C7092F852C32D23BCF1EA
:10AD5000AA0F05D009E0B2F84A335BBA8B83F3E758
:10AD600092F853C3BCF1550F06D0CB8392F85CC365
:10AD7000BCF1AA0F07D00BE0B2F854C39CFA9CFCBC
:10AD8000A1F81EC0F2E792F85DC3BCF1550F0DD0DB
:10AD9000A1F8207092F866C3BCF1AA0F0DD011E0A3
:10ADA000E00E0020E40200206E130020B2F85EC323
:10ADB0009CFA9CFCA1F820C0ECE792F867C3BCF1B8
:10ADC000550F07D0A1F8223092F870C3BCF1AA0F3A
:10ADD00007D00BE0B2F868C39CFA9CFCA1F822C033
:10ADE000F2E792F871C3BCF1550F07D0A1F824B077
:10ADF00092F87AC3BCF1AA0F07D00BE0B2F872C385
:10AE00009CFA9CFCA1F824C0F2E792F87BC3BCF149
:10AE1000550F09D04FF00F0CA1F826C092F884C34B
:10AE2000BCF1AA0F05D009E0B2F87CC39CFA9CFCE7
:10AE3000F2E792F885C3BCF1550F07D0A1F828704E
:10AE400092F88EC3BCF1AA0F07D00BE0B2F886C30C
:10AE50009CFA9CFCA1F828C0F2E792F88FC3BCF1E1
:10AE6000550F07D0A1F82A3092F898C3BCF1AA0F69
:10AE700007D00EE0B2F890C39CFA9CFCA1F82AC05F
:10AE8000F2E792F899C3BCF1550F02D1B2F89A7368
:10AE90007FBA8F8592F8A273AA2F06D192F8A37376
:10AEA000552F02D1B2F8A4335BBACB8592F8AC33FC
:10AEB000AA2B03D192F8AD33552B06D0A1F8305010
:10AEC00092F8B633AA2B05D008E0B2F8AE335BBADD
:10AED0000B86F5E792F8B733552B06D0A1F83290E0
:10AEE00092F8C033AA2B05D008E0B2F8B8335BBAA9
:10AEF0004B86F5E792F8C133552B06D0A1F83450B4
:10AF000092F8CA33AA2B05D008E0B2F8C2335BBA74
:10AF10008B86F5E792F8CB33552B06D0A1F8369007
:10AF200092F8D433AA2B05D008E0B2F8CC335BBA40
:10AF3000CB86F5E792F8D533552B07D081F838B09A
:10AF400092F8DE33DD49AA2B06D009E0B2F8D633F9
:10AF50005BBA81F83830F3E792F8DF33552B07D02E
:10AF600041F27C530B8092F8E833AA2B04D007E01F
:10AF7000B2F8E0335BBAF5E792F8E933552B06D027
:10AF8000A1F802A092F8F233AA2B05D008E0B2F89B
:10AF9000EA335BBA4B80F5E792F8F333552B07D0D1
:10AFA00041F2CC038B8092F8FC33AA2B04D007E04B
:10AFB000B2F8F4335BBAF5E792F8FD33552B08D0BD
:10AFC00041F26803CB8092F806740323AA2F04D0C1
:10AFD00007E0B2F8FE335BBAF4E792F80774552F36
:10AFE00005D00B8192F81074AA2F05D008E0B2F8B2
:10AFF00008747FBA0F81F5E792F81174552F07D0C6
:10B0000040F6B8374F8192F81A74AA2F04D007E09F
:10B01000B2F812747FBAF5E792F81B74552F07D077
:10B020004FF448678F8192F82474AA2F04D00AE065
:10B03000B2F81C747FBAF5E792F82574552F02D147
:10B04000B2F826345BBACB8192F82E34AA2B03D106
:10B0500092F82F34552B06D0A1F8108092F838348E
:10B06000AA2B05D008E0B2F830345BBA0B82F5E7C2
:10B0700092F83934552B07D04FF4FA434B8292F8AB
:10B080004234AA2B04D007E0B2F83A345BBAF5E7B1
:10B0900092F84334552B06D0A1F8146092F84C3442
:10B0A000AA2B05D008E0B2F844345BBA8B82F5E7EE
:10B0B00092F84D34552B07D0A1F8169092F85634DB
:10B0C0007F4FAA2B05D008E0B2F84E345BBACB8292
:10B0D000F4E792F85734552B06D07A4B3B6092F840
:10B0E0006034AA2B0AD00DE0B2F8583493FA93FCDE
:10B0F000B2F85A345BBA6CF31F43EFE792F861344D
:10B10000552B07D0C1F818E092F86A346E49AA2B83
:10B110000AD00DE0B2F862345FBAB2F864345BBAB8
:10B1200067F31F438B61EFE792F86B34552B11D017
:10B130004FF4FD630B8005238B701A23CB70102313
:10B140004B718B71CB7107230B7192F87414AA2980
:10B1500016D019E0B2F86C345BBA0B8092F86E34FA
:10B160008B7092F86F34CB7092F870344B7192F808
:10B1700071348B7192F87234CB7192F87334E3E7C7
:10B1800092F87514552908D05FF03701A4F8C4105F
:10B1900092F87E14AA2904D007E0B2F8761449BACE
:10B1A000F4E792F87F14552908D03721A4F8C81085
:10B1B00092F888344549AA2B04D007E0B2F88014ED
:10B1C00049BAF3E792F88934552B07D081F88350B8
:10B1D00092F892343E49AA2B05D008E092F88A34BE
:10B1E00081F88330F4E792F89334552B2ED00D700C
:10B1F000A04608F0F2FC044636480F46007808F0F6
:10B20000ECFC0022344B08F05AFC22463B4608F086
:10B21000E4FB08F048FD31490860D8F80C0108F05B
:10B22000DCFC0B4602462046394608F048FC08F094
:10B230003AFD2B492C4A086098F8DD3029482B4903
:10B2400043B1012B06D0022B04D005E092F89424E0
:10B250000A70CDE71060086025480178254861B183
:10B260000670F7F7E7FF24480178244849B10670D3
:10B2700007B0BDE8F04FF7F765BF0570F7F7F1FFCE
:10B28000F1E7057007B0BDE8F04FF7F779BF2DE99A
:10B29000F047DFF86C9004464FF4FA652A464946B9
:10B2A000184804F011FE1849184B0448154A552651
:10B2B000AA274FF0000C762C2AD22AE0AC130020EB
:10B2C000DC00002087C0113A7C030020D01300204E
:10B2D000070000206A00002000005940C000002044
:10B2E000D0000020713D8A3FC4000020C80000202B
:10B2F000660000207300002067000020740000201A
:10B3000000F00108FA140020E00E00206E13002067
:10B310003FE0DFE804F03B3F4953595F656B7177CD
:10B320007DF2FCEFEEEDECEBEAE9E8E7E6E5E4E3DD
:10B33000E2E1E0DFDEDDDCDBDAD9D8D7D6D5D4D365
:10B34000D2D1D0CFCECDCCCBCAC9C8C7C6C5C43EDA
:10B35000C3C2C1C0BFBEBDBCBBBAB9B8B7B6B5B435
:10B36000B3B2B1B0AFAEADACABAAA9A8A7A6A5A425
:10B37000A3A2A1A09F9E9D9C9B9A99989796959415
:10B38000939291908F8E8D8C8B8A8988FB48007860
:10B39000907010E2FA48FB4B008803F10A014FEA73
:10B3A000102C83F80CC03CE0D1F88C00F54B4FEA30
:10B3B000106C03F1140183F816C0ADE1F248F149B5
:10B3C000007881F82000F6E1F048EE49007881F835
:10B3D0002A00F0E1EE48EB49007881F83400EAE118
:10B3E000EC48E849007881F83E00E4E1EA48E549A4
:10B3F000007881F84800DEE1E848E249007881F809
:10B400005200D8E1E648DF49007881F85C00D2E1DB
:10B41000B1F89800DB4B4FEA102C03F1640183F87C
:10B4200066C0C870C7E1EEE3EEE3EEE3EEE3EEE301
:10B43000EEE3EEE3EEE3EEE3EEE3EEE3EEE3EEE384
:10B44000EEE3EEE3EEE3EEE3D4E3CAE3C0E3B6E318
:10B45000ACE39AE390E386E37CE372E368E35EE3C4
:10B4600054E34AE340E336E32CE322E318E30EE33C
:10B4700004E3FAE2F0E2E6E2DCE2D2E2C8E2BEE2B3
:10B48000B4E2AAE2A0E295E28AE27FE274E269E233
:10B4900062E25BE254E24DE242E237E22DE21EE27A
:10B4A00006E2ECE1CEE1C3E1B8E1ADE19EE193E17A
:10B4B0008CE181E17AE157E150E149E13EE137E198
:10B4C00030E120E119E10EE103E1F8E0EDE0E2E036
:10B4D000D7E0CCE0C1E0B6E0ABE0A0E099E08EE0E0
:10B4E00083E078E06DE062E057E04CE041E036E078
:10B4F0002BE020E015E00AE0FFE7B1F89A00A14B4D
:10B500004FEA102C03F16E0183F870C089E7B1F89F
:10B510009C009C4B4FEA102C03F1780183F87AC011
:10B520007FE7B1F89E00974B4FEA102C03F18201A0
:10B5300083F884C075E7B1F8A000924B4FEA102C55
:10B5400003F18C0183F88EC06BE7B1F8A2008D4B3C
:10B550004FEA102C03F1960183F898C061E7B1F827
:10B56000A400884B4FEA102C03F1A00183F8A2C07D
:10B5700057E7B1F8A600834B4FEA102C03F1AA015C
:10B5800083F8ACC04DE7B1F8A8007E4B4FEA102C11
:10B5900003F1B40183F8B6C043E7B1F8AA00794BD0
:10B5A0004FEA102C03F1BE0183F8C0C039E7B1F8AF
:10B5B000AC00744B4FEA102C03F1C80183F8CAC0E9
:10B5C0002FE7B1F8AE006F4B4FEA102C03F1D20118
:10B5D00083F8D4C025E7B1F8B0006A4B4FEA102CCD
:10B5E00003F1DC0183F8DEC01BE7B1F8B200654B64
:10B5F0004FEA102C03F1E60183F8E8C011E7B1F837
:10B60000B400604B4FEA102C03F1F00183F8F2C054
:10B6100007E791F8B6005B4981F8FC00A7E3B1F8B1
:10B62000B800584B4FEA102C03F5827183F806C11D
:10B63000F7E6B1F8BA00534B4FEA102C03F58771C7
:10B6400083F810C1EDE6B1F8BC004E4B4FEA102C68
:10B6500003F58C7183F81AC1E3E6B1F8BE00494BDB
:10B660004FEA102C03F5917183F824C1D9E6B1F8A3
:10B67000C000444B4FEA102C03F5967183F82EC19D
:10B68000CFE6B1F8C2003F4B4FEA102C03F59B7197
:10B6900083F838C1C5E6B1F8C6003A4B4FEA102C22
:10B6A00003F5A07183F842C1BBE6B1F8CA00354B7F
:10B6B0004FEA102C03F5A57183F84CC1B1E6B1F83F
:10B6C000CC00304B4FEA102C03F5AA7183F856C119
:10B6D000A7E6B1F8CE002B4B4FEA102C03F5AF7163
:10B6E00083F860C19DE6B1F8D000264B4FEA102CDC
:10B6F00003F5B47183F86AC193E691F8D200214949
:10B7000081F8740133E3D1F8D4001E4B4FEA106C7A
:10B7100003F5BE7183F87EC1030CCB70030A0B7175
:10B72000487124E31F481749007881F888011EE317
:10B730001D481449007881F8920118E3B1F8DA0045
:10B74000104B4FEA102C03F5CD7183F89CC168E6CD
:10B7500091F8DC000B4981F8A60108E391F8DD00BF
:10B76000084981F8B00102E3B1F8DE00054B4FEA69
:10B77000102C03F5DC7183F8BAC152E66A00002090
:10B7800010010020FA1400206C0000206D00002041
:10B790006E0000206F00002070000020710000206B
:10B7A00072000020660000206700002091F8E00091
:10B7B000FA4981F8C401DAE2F949F84851F8E13F61
:10B7C000C0F8CE314968C0F8D211D0E291F8EB0050
:10B7D000F24981F8D801CAE2F149F04851F8EC3F4A
:10B7E000C0F8E2314968C0F8E611C0E2EB4B11F84D
:10B7F000F4CF03F5F57083F8ECC14B78C3708B7808
:10B800000371C9784171B2E2D1F8F800E34B4FEA15
:10B81000106C03F5FA7183F8F6C17DE7E148DF4B60
:10B82000006803F5FF714FEA106C83F800C273E7FC
:10B83000D1F80C01D94B4FEA106C03F5027183F873
:10B840000AC269E7D54B91F810C103F2122083F8C0
:10B8500014C291F81131C37091F81231037191F84B
:10B860001331437191F81431837191F81531C3711B
:10B8700091F81631037291F81711417277E2C74BB4
:10B8800091F818C103F5077083F81EC291F81931B9
:10B89000C37091F81A31037191F81B31437191F81B
:10B8A0001C31837191F81D31C37191F81E113CE276
:10B8B000BA4B91F81FC103F2262083F828C291F8F1
:10B8C0002031C37091F82131037191F82231437115
:10B8D00091F82331837191F82411C17147E2AF4B84
:10B8E00091F825C103F50C7083F832C291F8263126
:10B8F000C37091F82711017139E2AB49A7480B6871
:10B90000C0F846328988A0F84A1230E2B1F82A011C
:10B91000A24B4FEA102C03F24E2183F850C280E56F
:10B92000B1F82C019D4B4FEA102C03F5167183F8EA
:10B930005AC276E591F82E01984981F8640216E220
:10B9400091F82F01954981F86E0210E291F83001CB
:10B95000924981F878020AE291F831018F4981F821
:10B96000820204E2B1F832018C4B4FEA102C03F250
:10B970008A2183F88CC254E5B1F83401874B4FEA31
:10B98000102C03F5257183F896C24AE5B1F836010B
:10B99000824B4FEA102C03F29E2183F8A0C240E5AF
:10B9A000B1F838017D4B4FEA102C03F52A7183F86A
:10B9B000AAC236E5B1F83A01784B4FEA102C03F2EF
:10B9C000B22183F8B4C22CE51888744B4FEA102CCE
:10B9D00003F52F7183F8BEC223E558886F4B4FEAF9
:10B9E000102C03F2C62183F8C8C21AE598886B4B65
:10B9F0004FEA102C03F5347183F8D2C211E5D888D0
:10BA0000664B4FEA102C03F2DA2183F8DCC208E51A
:10BA10001889624B4FEA102C03F5397183F8E6C29E
:10BA2000FFE458895D4B4FEA102C03F2EE2183F8B6
:10BA3000F0C2F6E49889594B4FEA102C03F53E7199
:10BA400083F8FAC2EDE4D889544B4FEA102C03F284
:10BA5000023183F804C3E4E4188A504B4FEA102CF7
:10BA600003F5437183F80EC3DBE4588A4B4B4FEA6E
:10BA7000102C03F2163183F818C3D2E4988A474B8E
:10BA80004FEA102C03F5487183F822C3C9E4D88A21
:10BA9000424B4FEA102C03F22A3183F82CC3C0E446
:10BAA000188B3E4B4FEA102C03F54D7183F836C3CB
:10BAB000B7E4588B394B4FEA102C03F23E3183F830
:10BAC00040C3AEE4988B354B4FEA102C03F552710E
:10BAD00083F84AC3A5E4D88B304B4FEA102C03F20D
:10BAE000523183F854C39CE4188C2C4B4FEA102C31
:10BAF00003F5577183F85EC393E4588C274B4FEAE4
:10BB0000102C03F2663183F868C38AE4988C234BC7
:10BB10004FEA102C03F55C7183F872C381E4D88C72
:10BB20001E4B4FEA102C03F27A3183F87CC378E481
:10BB3000188D1A4B4FEA102C03F5617183F886C3F8
:10BB40006FE4588D154B4FEA102C03F28E3183F8B9
:10BB500090C366E4988D114B4FEA102C03F5667183
:10BB600083F89AC35DE4D88D0C4B4FEA102C03F296
:10BB7000A23183F8A4C354E4188E084B4FEA102C6A
:10BB800003F56B7183F8AEC34BE4588E034B4FEA59
:10BB9000102C03F2B63183F8B8C342E4FA14002043
:10BBA000E00E0020D8000020E4020020988EFF4B19
:10BBB0004FEA102C03F5707183F8C2C331E4D88EBC
:10BBC000FA4B4FEA102C03F2CA3183F8CCC328E4B5
:10BBD000F64901F5757081F8D6C393F83810C17035
:10BBE000C5E00088F14B4FEA102C03F2DE3183F8F8
:10BBF000E0C316E44088ED4B4FEA102C03F57A7150
:10BC000083F8EAC30DE4ADE0A5E09AE08FE078E0C8
:10BC10006EE063E059E04FE045E03BE031E027E0D3
:10BC20001DE013E009E0FFE78088E04B4FEA102CAD
:10BC300003F2F23183F8F4C368E4C088DB4B4FEAC7
:10BC4000102C03F57F7183F8FEC35FE40089D74BA6
:10BC50004FEA102C03F2064183F808C456E44089E9
:10BC6000D24B4FEA102C03F5826183F812C44DE4E5
:10BC70008089CE4B4FEA102C03F21A4183F81CC482
:10BC800044E4C089C94B4FEA102C03F2244183F8E5
:10BC900026C43BE4008AC54B4FEA102C03F22E4128
:10BCA00083F830C432E4408AC04B4FEA102C03F5CD
:10BCB000876183F83AC429E4808ABC4B4FEA102C90
:10BCC00003F2424183F844C420E4C08AB74B4FEAF0
:10BCD000102C03F24C4183F84EC417E4B448B34B24
:10BCE000006803F256414FEA106C83F858C413E51C
:10BCF0008069AE4B4FEA106C03F58C6183F862C427
:10BD00000AE5AC49DFF8A4C20B880CF26A404FEA9E
:10BD100013288CF86C84C3708B780371CB784371D3
:10BD20004B7983718B79C371C97901721FE0B1F8C6
:10BD3000C4009E4B4FEA102C03F2744183F876C482
:10BD40000CE4B1F8C800994B4FEA102C03F27E4185
:10BD500083F880C40CE49848944990F8830081F8F3
:10BD60008A0404E095489149007881F8940404EB32
:10BD70008400494602F8107002EB40002A464670E3
:10BD8000BDE8F047894804F0C7B82DE9F047874A75
:10BD900000EB80033321DFF8209202F8131002EB4E
:10BDA000430499F88200864D60700021002001EB69
:10BDB00041077E1907EB000806EB000C08EB43086F
:10BDC0009044401C9CF81AC0C0B288F802C00328F6
:10BDD000F0D3491CC9B22029E8D37A480088010A67
:10BDE00004F8621F607078480088010AA170E07052
:10BDF0000120FBF7CBF835F87C0F010A2171607147
:10BE000072480088010AA171E07171480088010A36
:10BE1000217260722720A0720F21E172207361737A
:10BE2000A073E17320746174A074E174207561756E
:10BE3000A888010AA175E075E888010A2176607674
:10BE4000287A4946A07631F87E0F020AE2762077FA
:10BE500048886049020A6277A07756480288130A28
:10BE6000E37704F8202F82786270C278A27042795A
:10BE7000E27082792271C07960716620A07199F8B0
:10BE80008200BDE8F04701EB80214FF4FA62474899
:10BE900004F042B82DE9F041444C064633202070AE
:10BEA000474D66700020002100EB400253195F18D7
:10BEB00002EB010CA444491CBF7EC9B28CF802708D
:10BEC0000329F4D3401CC0B22028ECD33D4800889D
:10BED000010A04F8621F60703B480088010AA170E3
:10BEE000E0700120FBF752F835F87C0F010A217150
:10BEF000607136480088010AA171E07134480088F9
:10BF0000010A217260722720A0720F21E172207352
:10BF10006173A073E17320746174A074E17420757F
:10BF20006175A888010AA175E075E888010A217683
:10BF300060762149287AA07631F87E0F020AE276EF
:10BF400020774888010A6177A0771A4801880A0A91
:10BF5000E27704F8201F81786170C178A17041797F
:10BF6000E17081792171C07960716620A0711948F2
:10BF70004FF4C87200EB8621BDE8F0410B4803F096
:10BF8000CBBF2DE9F041144D4FF4FA642246294607
:10BF9000064803F099FF0548AA21094B00F8641FE1
:10BFA0005522427033F8986F370A17E0FA140020D0
:10BFB000DC0000207C030020D013002007000020BC
:10BFC000E00E0020BE000020BC000020B6000020D3
:10BFD000B80000200078010800F001088770C670E2
:10BFE0008172C2725E88370A0773467301754275A3
:10BFF0009E88370A8775C6758177C277DE88370ACB
:10C0000080F8207080F8216080F8281080F82920BE
:10C010001E89370A80F82A7080F82B6080F8321069
:10C0200080F833205E89370A80F8347080F83560F4
:10C0300080F83C1080F83D209E89370A80F83E70D9
:10C0400080F83F6080F8461080F84720DE89370A84
:10C0500080F8487080F8496080F8501080F85120CE
:10C060001E8A370A80F8527080F8536080F85A10A0
:10C0700080F85B205E8A370A80F85C7080F85D602B
:10C0800080F8641080F865209E8A370A80F8667010
:10C0900080F8676080F86E1080F86F20DE8A370ABB
:10C0A00080F8707080F8716080F8781080F87920DE
:10C0B0001E8B370A80F87A7080F87B6080F88210D7
:10C0C00080F883205E8B370A80F8847080F8856062
:10C0D00080F88C1080F88D209E8B370A80F88E7047
:10C0E00080F88F6080F8961080F897209E7F80F807
:10C0F000986080F8A01080F8A12033F8206F370AEC
:10C1000080F8A27080F8A36080F8AA1080F8AB20B5
:10C110005E88370A80F8AC7080F8AD6080F8B410A3
:10C1200080F8B5209E88370A80F8B67080F8B7602E
:10C1300080F8BE1080F8BF20DE88370A80F8C07013
:10C1400080F8C16080F8C81080F8C9201E89370ABD
:10C1500080F8CA7080F8CB6080F8D21080F8D320C5
:10C160005E89370A80F8D47080F8D56080F8DC10DA
:10C1700080F8DD20DE89370A80F8DE7080F8DF6025
:10C1800080F8E61080F8E7205E8A370A80F8E870C9
:10C1900080F8E96080F8F01080F8F1209E8A370A74
:10C1A00080F8F27080F8F36080F8FA1080F8FB20D5
:10C1B000DE8A370A80F8FC7000F8FD6FDFF834C4BF
:10C1C000C17102721E8B370A477286724174827483
:10C1D0009E7EC674C1760277DE69370E4777370CCC
:10C1E0008777370AC77780F82060FF4E80F82510E0
:10C1F00080F82620367880F82760FC4E80F82F10D3
:10C2000080F83020367880F8316080F8391080F876
:10C210003A205E8C370A80F83B7080F83C6080F8EA
:10C22000431080F8442093F8246080F8456080F83B
:10C230004D1080F84E2093F8256080F84F6080F80C
:10C24000571080F85820DE8C370A80F8597080F833
:10C250005A6080F8611080F8622093F8286080F8B6
:10C26000636080F86B10E24F80F86C20DCF8E1E04E
:10C270000CF18006C7F84EE0DCF8E5C0C7F852C004
:10C2800080F8751080F8762093F833C080F877C076
:10C2900080F87F1080F88020D6F86CC0C7F862C0A4
:10C2A000366FC7F8666080F8891080F88A2093F8A6
:10C2B0003C6080F88B6093F83D6080F88C6093F868
:10C2C0003E6080F88D6093F83F6080F88E6080F863
:10C2D000931080F894201E6C370E80F89570370C00
:10C2E00080F89670370A80F8977080F8986080F828
:10C2F000A71080F8A8205E6D370E80F8A970370C63
:10C3000080F8AA70370A80F8AB7080F8AC6080F8CB
:10C31000B11000F8B22F93F85860467093F8596046
:10C32000867093F85A60C67093F85B60067193F854
:10C330005C60467193F85D60867193F85E60C671CB
:10C3400093F85F600672417200F80A2F93F86060FC
:10C35000467093F86160867093F86260C67093F8D7
:10C360006360067193F86460467193F86560867146
:10C3700013F8666FC671417200F80A2F5E78467036
:10C3800013F8026F86705E78C6709E780671DE784C
:10C3900046711E79867100F8271F42705E89370A40
:10C3A00000F8027F4670017242729E89370A8772D6
:10C3B00000F80B6F00F82B1C00F82A2C5E7900F8AF
:10C3C000296C9E7900F8286CDE7900F8276CC17121
:10C3D00002729E7B467241748274DE7BC674C176A3
:10C3E00002771E7C467780F8251080F826205E7C38
:10C3F00080F8276000F82F1F427033F8126F370A59
:10C400008770C6708172C2725E88370A077346737E
:10C41000017542759E88370A8775C6758177C27720
:10C42000DE88370A80F8207080F8216080F82810B4
:10C4300080F8292019890A0A00F82A2F224641701B
:10C440002946BDE8F0416C4803F066BD2DE9F04196
:10C450006A4D4FF4FA6422462946674803F034FDDA
:10C460006548AA23634A00F8783F5521417032F8A5
:10C470009C6F370A8770C6708372C1725688370AFC
:10C4800007734673037541759688370A8775C675B5
:10C490008377C177D688370A80F8207080F82160CA
:10C4A00080F8283080F829101689370A80F82A7019
:10C4B00080F82B6080F8323080F833105689370AC4
:10C4C00080F8347080F8356080F83C3080F83D109A
:10C4D0009689370A80F83E7080F83F6080F84630D1
:10C4E00080F84710D689370A80F8487080F849608C
:10C4F00080F8503080F85110168A370A80F8527050
:10C5000080F8536080F85A3080F85B10568A370AFA
:10C5100080F85C7080F85D6080F8643080F86510A9
:10C52000968A370A80F8667080F8676080F86E3007
:10C5300080F86F10D68A370A80F8707080F87160C2
:10C5400080F8783080F87910118B0A0A80F87A2008
:10C5500080F87B1022462946BDE8F041264803F0CA
:10C56000DBBC2DE9F041254D4FF4FA642246294603
:10C57000214803F0A9FC2048AA211E4E00F8641FA0
:10C580005522427036F8983F1F0A8770C370817237
:10C59000C27271880A0A0273417322462946BDE8B5
:10C5A000F041154803F0B8BC2DE9F05F4FF4FA6292
:10C5B0001249114803F088FC11480023AA24038083
:10C5C0000D4855220F4900F80A4F42708370C3701E
:10C5D0000B600849C1F88C308472C27203734373D4
:10C5E0008373C37310E00000660000206700002022
:10C5F0007A160020E00E0020FA14002000F0010856
:10C6000010010020D400002041F26805A1F89C50E0
:10C6100080F86E4080F86F204FF0100880F870802E
:10C62000682580F8715041F20405A1F89E5080F809
:10C63000784080F8792080F87A804FF0040E80F8F6
:10C640007BE0A1F8A0E080F8824080F8832080F8A9
:10C65000843080F885E04FF42F65A1F8A25080F86F
:10C660008C4080F88D204FF00A0A80F88EA0F025CB
:10C6700080F88F5040F65435A1F8A45000F8964F3A
:10C680000B25427085705425C5700425A1F8A6506D
:10C690008472C272037345734FF47A75A1F8A8507F
:10C6A0000475427503258575E825C5753C25A1F8F7
:10C6B000AA508477C27780F8203080F82150A1F802
:10C6C000AC5080F8284080F8292080F82A3080F883
:10C6D0002B501425A1F8AE5080F8324080F833205A
:10C6E00080F8343080F835504FF0400CA1F8B0C0DD
:10C6F00080F83C4080F83D2080F83E3080F83FC014
:10C700004FF47A65A1F8B25080F8464080F847208F
:10C710004FF00F0B80F848B0A02580F849500A254B
:10C72000A1F8B45080F8504080F8512080F8523081
:10C7300080F853504FF0010981F8B69080F85A40C4
:10C7400080F85B2080F85C904B25A1F8B85080F809
:10C75000644080F8652080F8663080F867503C259A
:10C76000A1F8BA5080F86E4080F86F2080F87030E1
:10C7700080F871504125A1F8BC5080F8784080F8CD
:10C78000792080F87A3080F87B503725A1F8BE50A8
:10C7900080F8824080F8832080F8843080F88550CB
:10C7A0001426A1F8C06080F88C4080F88D2080F8B5
:10C7B0008E3080F88F604126A1F8C260A1F8C45085
:10C7C00080F8964080F8972080F8983080F899603B
:10C7D000A1F8C660A1F8C85080F8A04080F8A12058
:10C7E00080F8A23080F8A3606FF02705A1F8CA5046
:10C7F000AA23FE48FF24D82680F84A3180F84B212E
:10C8000080F84C4180F84D616E1DA1F8CC6080F835
:10C81000543180F8552180F85641DD2780F8577152
:10C82000A1F8CE5080F85E3180F85F2180F8604139
:10C83000D82580F86151A1F8D06080F8683180F87F
:10C84000692180F86A4180F86B7181F8D28080F8A4
:10C85000723180F8732180F874814FF4D254A1F8BA
:10C86000984080F8643080F865201A2480F866408B
:10C8700080F867C04FF48C54A1F89A4000F86E3FDE
:10C88000112442708470802400F8034F2826C1F8D8
:10C89000D46080F80B3180F80C21002480F80D4121
:10C8A00080F80E41D24D80F80F4180F810612C7055
:10C8B00080F81531CF4D80F8162180F817412C7083
:10C8C00080F81F3180F8202180F8214142F2107554
:10C8D000A1F8DA5080F8293180F82A21272580F83C
:10C8E0002B5180F82C8181F8DC9080F8333180F86E
:10C8F000342180F8359181F8DD9080F83D3180F861
:10C900003E2180F83F91A1F8DEB080F8473180F8F1
:10C91000482180F8494180F84AB181F8E0A080F8C8
:10C92000513180F852210A2580F853510F4607F102
:10C93000EC0547F8E14FDFF8C4827C60AE4F80F829
:10C940005B3180F85C2147F84E4F7C6081F8EB400A
:10C9500080F8653180F8662180F86741B8F8027088
:10C960002F8098F80470AF70D8F80970C5F803707C
:10C9700098F80D70EF7180F86F319F4F80F870213B
:10C98000D5F800C0C7F862C0D5F804C0C7F866C0C3
:10C99000D8F80570AF6080F8793180F87A2191F885
:10C9A000F45080F87B5191F8F55080F87C5191F863
:10C9B000F65080F87D5191F8F75080F87E51C1F81B
:10C9C000F84080F8833180F8842180F8854180F830
:10C9D00086418C4F80F8874180F88841884D3D60C2
:10C9E000392580F88F51F22580F89051382580F84C
:10C9F0009151972580F89251C1F80C6180F89731D8
:10CA000080F8982180F8994180F89A4180F89B41FC
:10CA10007D4D80F89C610E4655F8047BC6F8107178
:10CA200055F8047BC6F8147115F8017B06F2191449
:10CA300086F8187180F8A13180F8A22191F812616E
:10CA400080F8A36191F8136180F8A46191F81461F2
:10CA500080F8A56191F8156180F8A66191F81661DA
:10CA600080F8A76191F8176180F8A86180F8A97132
:10CA700055F8046B266035F80C69A68080F8AB3158
:10CA800080F8AC2191F8196180F8AD6191F81A61D4
:10CA900080F8AE6191F81B6180F8AF6191F81C617C
:10CAA00080F8B06191F81D6180F8B16191F81E6164
:10CAB00080F8B261D5F80E60C4F806606E8A6681AF
:10CAC00080F8B53180F8B62191F81F6180F8B76120
:10CAD00091F8206180F8B86191F8216180F8B9611E
:10CAE00091F8226180F8BA6191F8236180F8BB6106
:10CAF00091F8246180F8BC61AE8AA681AD7DA573F2
:10CB000080F8BF3180F8C02191F8253180F8C1311B
:10CB100091F8263180F8C23180F8C35140F6BE202A
:10CB2000A1F82A013148AA23BE2480F84E3280F8A9
:10CB30004F2280F850A280F8514240F62234A1F8EA
:10CB40002C4180F8583280F859220B2480F85A4240
:10CB5000222480F85B42002481F82E4180F8623262
:10CB600080F8632280F8644280F86C3280F86D228D
:10CB700091F82F5180F86E525A2581F8305180F883
:10CB8000763280F8772280F87852262581F8315164
:10CB900080F8803280F8812280F882524FF4C87584
:10CBA000A1F8325180F88A3280F88B2280F88C927A
:10CBB000902580F88D52A1F8344180F8943280F8A5
:10CBC000952280F8964280F897425025A1F8365178
:10CBD00080F89E3280F89F2280F8A04280F8A1520F
:10CBE000A1F838E180F8A83210E00000FA14002023
:10CBF00066000020670000207A160020F90200205D
:10CC00009738F239D80000201403002080F8A922B8
:10CC100080F8AA4280F8ABE240F61654A1F83A41F7
:10CC200080F8B23280F8B3220D2180F8B4121621B8
:10CC300080F8B512BDE8F05F4FF4FA62014903F0E5
:10CC40006BB9000000F0010838B50121042005F09F
:10CC50000BFB0121480605F014FB4FF48050ADF8A2
:10CC6000000003208DF8020018208DF803006946AB
:10CC7000FE4C204604F0B6FFE014ADF8000048205A
:10CC80008DF803006946204604F0ACFF38BD08B5B6
:10CC900014208DF8000000208DF801008DF80200AE
:10CCA00001208DF80300684603F0BBFA08BD30B5DB
:10CCB00087B0FFF7C9FFFFF7EAFFED4D284603F005
:10CCC000A3FD684603F0C4FE00248DF806408DF8ED
:10CCD000074008208DF8040007208DF802408DF8E9
:10CCE00005008DF803400420ADF800000294694669
:10CCF000284603F0A2FD6946284603F09EFD012167
:10CD00008DF816408DF818108DF81740ADF80C40CE
:10CD1000ADF810408DF819100A46ADF80E40ADF888
:10CD20001240ADF814400221284604F00FF903A880
:10CD300003F00DFE07B030BD00B585B0082A0FD84E
:10CD4000009000208DF808008DF809008DF80A2069
:10CD50000DF10B0006F0A2FC6946C54803F0E6FEA3
:10CD600005B000BD00B585B0082AF9D801900420AF
:10CD70008DF8080000208DF809008DF80A200DF1CB
:10CD80000B0006F08BFC6946B94803F0CFFEE7E7DD
:10CD90002DE9F0470646894600200721B2FBF1F352
:10CDA00001FB13239BB1B2FBF1F301FB1327B2FB91
:10CDB000F1F1491C5FFA81F505EB1661C6F3074CEA
:10CDC0006144C6F307242144F3B219440AE0B2FBDC
:10CDD000F1F1CDB20727EFE719F80080401C41447C
:10CDE00089B2C0B29042F7D3DFF888820022304681
:10CDF00088F8352188F83651320E88F8372188F8BE
:10CE000038C188F8394188F83A310A0A88F83B2154
:10CE100088F83C1108F2351108228A46FFF7A2FF74
:10CE2000012428E008EBC401C4EBC40202EB0900B2
:10CE300081F8354110F8072D81F83621427881F8C4
:10CE40003721827881F83821C27881F83921027936
:10CE500081F83A21427981F83B21807981F83C01BF
:10CE60000822304601F23511FFF77CFF1420FAF753
:10CE70008DF8641CE4B2AC42D4D3AC4227D108EBA9
:10CE8000C401C4EBC40202EB090081F8354110F87B
:10CE9000072D81F83621427881F83721827881F890
:10CEA0003821C27881F83921027981F83A21427912
:10CEB00081F83B21807981F83C017F1CFAB2304631
:10CEC00001F23511FFF74EFF1420FAF75FF8142036
:10CED000FAF75CF85046BDE8F0474FF4967106F05B
:10CEE000F6BB70B564480021654CC16001616348C0
:10CEF000B4F84010028860480C3022B141B9417842
:10CF000041F0010103E019B1417841F002014170A3
:10CF10005C4940F20443B1F892201A4203D04378AE
:10CF200043F00403437040F608031A4203D04378E9
:10CF300043F008034370930603D5437843F010038E
:10CF40004370530603D5437843F020034370D30660
:10CF500005D5437843F0400343F080034370B1F8B4
:10CF600094301D0703D4057845F0010505706479F8
:10CF7000012C03D1047844F002040470D40605D5D2
:10CF8000047844F0040444F008040470920703D5C4
:10CF9000027842F010020270DA0703D0027842F001
:10CFA000400202709A0703D5027842F080020270B4
:10CFB000B1F8822042F210739A1A0A2392FBF3F21C
:10CFC000140A8470C270B1F88010B1FBF3F2B1FBA7
:10CFD000F3F1120A027141712B490822097881711B
:10CFE0002A490978C17124494FF4C2600C31FFF716
:10CFF000A3FEBDE870400A20F9F7C8BF2DE9F04153
:10D000001D4E00201F4D7061B061F061306206F16D
:10D01000140415F8840F20701D4800786070E88CA7
:10D0200000EB80004000010AA170E070688D00EB09
:10D0300080004000010A21716071288B06F0CDFD4F
:10D040000022144B06F03BFD06F02DFEDFF8308089
:10D050000746B060B8F8380006F0A9FD394606F07A
:10D0600099FB06F0E0FD010AA17115E000080140FE
:10D07000006400402C1B0020300300209A00002098
:10D0800054140020E00E0020B0000020B200002068
:10D090002E03002000005940E0710822214640F292
:10D0A0000110FFF749FE0A20F9F770FF2A6D64218D
:10D0B00010464A4304F10801130A0B704A702A789B
:10D0C0005043F080020A8A70C8706A88130A0B7194
:10D0D0004A71B8F84020322A09D9012300EB8000B8
:10D0E00040048B71000CF080B0FBF2F0C871082294
:10D0F000FE4940F21260FFF71FFEBDE8F0410A2032
:10D10000F9F744BF704770B586B06A460021F84809
:10D1100003F001FEF74C009B04F114012360019819
:10D1200060609DF80A2022729DF8090060740198E1
:10D13000486014310198ED4D4860A1F11F000126AF
:10D140001C3D0DF10B01B3F5897F08D0A3F5807468
:10D15000113C02D12E7006F0A1FA06B070BD6E70BF
:10D1600006F09CFA617A0020012902D0022902D03F
:10D1700002E0AE7000E0A870A17A012903D0022974
:10D18000EBD1E870E9E7EE70E7E72DE9FF5F0025F6
:10D19000DFF864830095202401950295284640F22B
:10D1A00013160395471C009500EB40018DF80070A5
:10D1B00001EB080001958DF80170C17E8DF8021019
:10D1C000007F8DF80300082269463046FFF7B4FD62
:10D1D0000120F9F7DBFEF8B22028E3D3C748009519
:10D1E000641C01958DF8004000880822010A8DF822
:10D1F00001108DF80200694640F21310FFF79CFD04
:10D200000120F9F7C3FEBE480095641C01958DF816
:10D21000004000880822010A8DF801108DF80200F4
:10D22000694640F21310FFF787FD0120F9F7AEFEC3
:10D230000095641C8DF8004027268DF801600F27AB
:10D2400001958DF802700822694640F21310FFF72D
:10D2500073FD0120F9F79AFEDFF8A8B20095641C6F
:10D2600001958DF80040BBF800000822010A8DF8F6
:10D2700001108DF80200694640F21310FFF75CFDC3
:10D280000120F9F783FEDFF880920095641C019578
:10D290008DF80040B9F800000822010A8DF801104D
:10D2A0008DF80200694640F21310FFF745FD01209A
:10D2B000F9F76CFE0095641C01958DF80040B8F8F4
:10D2C0007C000822010A8DF801108DF802006946E1
:10D2D00040F21310FFF730FD0120F9F757FE8B489D
:10D2E0000095641C01958DF8004000880822010A11
:10D2F0008DF801108DF80200694640F21310FFF717
:10D300001BFD0120F9F742FE0095641C8DF80040DA
:10D310008DF8016001958DF802700822694640F28F
:10D320001310FFF709FD0120F9F730FE0095641C8A
:10D330008DF800408DF8016001958DF8027008228B
:10D34000694640F21310FFF7F7FC0120F9F71EFEC3
:10D350000095641C8DF800408DF8016001958DF8F2
:10D3600002700822694640F21310FFF7E5FC012025
:10D37000F9F70CFE0095641C8DF800408DF80160F3
:10D3800001958DF802700822694640F21310FFF7EC
:10D39000D3FC0120F9F7FAFD0095641C01958DF886
:10D3A0000040B8F880000822010A8DF801108DF8BD
:10D3B0000200694640F21310FFF7BEFC0120F9F7A6
:10D3C000E5FD0095641C01958DF80040B8F88200D9
:10D3D0000822010A8DF801108DF80200694640F21A
:10D3E0001310FFF7A9FC0120F9F7D0FD0095641C8C
:10D3F00001958DF8004098F884008DF8010008220E
:10D40000694640F21310FFF797FC0120F9F7BEFDC3
:10D410003F480095641C01958DF800400088082263
:10D42000010A8DF801108DF80200694640F21310D0
:10D43000FFF782FC0120F9F7A9FD0095641C019516
:10D440008DF80040B8F886000822010A8DF8011016
:10D450008DF80200694640F21310FFF76DFC0120C1
:10D46000F9F794FD0095641C01958DF8004098F83B
:10D4700085008DF801000822694640F21310FFF77D
:10D480005BFC0120F9F782FD0095641C01958DF885
:10D490000040B8F890000822010A8DF801108DF8BC
:10D4A0000200694640F21310FFF746FC0120F9F72D
:10D4B0006DFD641C0095E4B201958DF80040B8F84C
:10D4C0008000B8F89810134E884203D3318C41F095
:10D4D000010131843188884203D8318C21F0010167
:10D4E0003184B8F89A1088421AD815E04C0300200D
:10D4F00000640040041B0020E00E0020BE0000205D
:10D50000BC000020B6000020B8000020BA000020B7
:10D510002E030020AC130020318C41F00201318435
:10D520007188884203D3308C20F0020030840020C0
:10D53000FE4ADFF8FCA3B8F89C70B8F89E3098F863
:10D54000D210AE460EE000BF3AF81050BD4203D9EB
:10D550004FF0010C02F800C09D4201D202F800E039
:10D56000401CC0B28142EFD80023184604E0155C8D
:10D57000401C2B44DBB2C0B28142F8D8308C13B1CE
:10D5800040F0040001E020F004003084E74A00206D
:10D590002032B8F8A450B8F8A2300DE03AF8107074
:10D5A0009F4203D24FF0010C02F800C0AF4201D9F4
:10D5B00000271754401CC0B28142EFD80023184600
:10D5C00004E0155C401C2B44DBB2C0B28142F8D8A9
:10D5D000308C13B140F0080001E020F00800D5497C
:10D5E000D54A308408881388C01AB8F8A830984201
:10D5F00003DB338C43F010033384318A884203DC2D
:10D60000308C20F010003084B8F8AA00CB4A00EB30
:10D61000C00101EB00101188B1EB800F308C02D3F8
:10D6200040F0200001E020F020003084C448B8F829
:10D63000AE30B0F8405003EBC30707EB0313B5EB74
:10D64000830F338C02D343F0400301E023F0400307
:10D65000338498F8313103EB4305C5EBC313B1EBC9
:10D66000C30F318C02D341F0800101E021F0800131
:10D670003184B0F94610B8F8B820914203DB328CFF
:10D6800042F480723284B8F8BA20914203DC318CC3
:10D6900021F480713184B0F94210B8F8BC20914275
:10D6A00003DB328C42F400723284B8F8BE2091421F
:10D6B00003DC328C22F400723284A248ADF80810E8
:10D6C00000210088ADF80A009F4802AD0088ADF83F
:10D6D0000C009E480088ADF80E00084601E00020CE
:10D6E0000CE005EB400735F91020B7F902309A42FB
:10D6F00002DD25F810307A80401CC0B2C1F103026F
:10D700008242EEDC491CC9B20429E8D3BDF90E10EF
:10D71000BDF90800B8F8C0300A1A12B2934203DC0F
:10D72000338C43F480633384F38A934203DB328C7B
:10D7300022F480623284B8F8C620914203DB328C36
:10D7400042F400623284B8F8C820914203DC328C83
:10D7500022F400623284B8F9CE20904203DC328C8D
:10D7600042F480523284B8F9D020904203DB328CEC
:10D7700022F480523284B8F8C220914203DB328C0A
:10D7800042F400523284B8F8C420914203DC318C58
:10D7900021F400513184B8F9CA10884203DC318C7D
:10D7A00041F480413184B8F9CC10884203DB308CDD
:10D7B00020F480403084B8F89200C004308C02D548
:10D7C00040F4004001E0C0F30E00308480B2010A52
:10D7D0008DF801108DF802000822694640F21310FE
:10D7E000FFF7AAFA0120F9F7D1FB0027641C009784
:10D7F000E4B201978DF800404C4A38464032B6F802
:10D800000490B6F806C04FF0010E434698F8D210C7
:10D81000BB460BE03AF810704F4501D902F800E022
:10D82000674501D202F800B0401CC0B28142F1D875
:10D830000027384606E000BF12F800C0401C6744CD
:10D84000FFB2C0B28142F7D8708C17B140F004002B
:10D8500001E020F004007084344A00206032B6F801
:10D860000AC0B78999460DE03AF81030634503D2F3
:10D870004FF0010802F80080BB4201D90023135485
:10D88000401CC0B24B468142EED80027384605E026
:10D8900012F800C0401C6744FFB2C0B28142F7D802
:10D8A000708C17B140F0080001E020F0080070848F
:10D8B000B3F8361101EBC10000EB01111F480088DD
:10D8C000B0EB810F708C02D340F0200001E020F01B
:10D8D00020007084DFF868B0718ABBF8400001EB6B
:10D8E000C10202EB0111B0EB810F708C02D340F04A
:10D8F000400001E020F040007084B9F892004F46EB
:10D900008004708C02D540F4004001E0C0F30E00AA
:10D9100070840F48408C010A8DF801108DF80200C8
:10D920000822694640F2131014E00000841A002017
:10D9300000090020A2000020A40000209A0000207E
:10D9400054140020BA000020B6000020B8000020C7
:10D95000AC130020FFF7F0F90120F9F717FB0020C6
:10D96000641C0090E4B201908DF80040B7F880107C
:10D970003B46FE4E3288914203D3728F42F0010241
:10D9800072877288914203D8728F22F001027287E7
:10D99000B288914203D8728F42F002027287F288F5
:10D9A000914203D3718F21F0020171870022DFF8C9
:10D9B000C083B6F8089077894FF0010E93F8D21023
:10D9C0000DE000BF3AF81200484501D908F802E01E
:10D9D000B84202D2002008F80200521CD2B2914292
:10D9E000F0D800221046474606E000BF17F800C0F6
:10D9F000401C6244D2B2C0B28142F7D8708F12B1DB
:10DA000040F0040001E020F0040070870020D84AB4
:10DA1000F046D6462032B6F80CC0F78982469946C1
:10DA20000CE000BF3EF81030634501D202F80080E0
:10DA3000BB4201D902F800A0401CC0B28142F1D81B
:10DA40000027384604E0135C401C3B44DFB2C0B200
:10DA50008142F8D8708F17B140F0080001E020F043
:10DA600008007087C3480188C3480088081A318AB3
:10DA7000884203DB718F41F010017187718A8842FF
:10DA800003DC708F20F010007087B08A00EBC001BB
:10DA900001EB0011B9480088B0EB810F03D3718FFF
:10DAA00041F020017187F18A01EBC10202EB011103
:10DAB000B0EB810F03D8708F20F020007087328B7D
:10DAC000BBF8401002EBC20303EB02125846B1EB65
:10DAD000820F03D3728F42F040027287728B02EB87
:10DAE000C20303EB0212B1EB820F03D8718F21F056
:10DAF00040017187B0F94610B28B914203DB728FFF
:10DB000042F080027287F28B914203DC718F21F028
:10DB100080017187BBF94200318C884203DB718F31
:10DB200041F480717187718C884203DC718F21F41C
:10DB300080717187ADF80800914800210088ADF828
:10DB40000A0090480088ADF80C008F480088ADF8B6
:10DB50000E00084601E000200CE005EB400735F917
:10DB60001020B7F902309A4202DD25F810307A8091
:10DB7000401CC0B2C1F103028242EEDC491CC9B2B2
:10DB80000429E8D3BDF90E10BDF90800B38C0A1AB8
:10DB900012B2934203DC738F43F400737387F38CE8
:10DBA000934203DB728F22F400727287328D9142AE
:10DBB00003DB728F42F480627287728D914203DCC4
:10DBC000728F22F480627287B28D914203DB728F72
:10DBD00042F400627287F28D914203DC718F21F46E
:10DBE00000617187B6F93010884203DC718F41F40F
:10DBF00080517187B6F93210884203DB718F21F4AE
:10DC000080517187B6F93410884203DC718F41F47A
:10DC100000517187B6F93610884203DB708F20F40B
:10DC20000050708799F8841099F8E0209142728F23
:10DC300002D842F4804201E022F48042728796F8D2
:10DC400038004F46814290B202D840F4004001E0D3
:10DC5000C0F30E00708780B2010A8DF801108DF8B4
:10DC6000020040F21319082269464846FFF764F89B
:10DC70000120F9F78BF9CDF800A0641CCDF804A0C1
:10DC80008DF8004037F8940F5546010A8DF80110C1
:10DC90008DF80200082269464846FFF74DF801203A
:10DCA000F9F774F90095641C01958DF800403088EF
:10DCB0000822010A8DF801108DF8020069464846D5
:10DCC000FFF73AF80120F9F761F90095641C019516
:10DCD0008DF8004070880822010A8DF801108DF837
:10DCE000020069464846FFF727F80120F9F74EF988
:10DCF0000095641C01958DF80040B8880822010A3F
:10DD00008DF801108DF8020069464846FFF714F8B7
:10DD10000120F9F73BF9DFF874800095641C019548
:10DD20008DF80040B8F800000822010A8DF80110B3
:10DD30008DF8020069464846FEF7FEFF0120F9F71C
:10DD400025F90095641C01958DF80040B0880822E3
:10DD5000010A8DF801108DF8020069464846FEF769
:10DD6000EBFF0120F9F712F9009511E06E13002086
:10DD7000441A0020A2000020A40000209A000020E5
:10DD8000BA000020B6000020B8000020AC1300202C
:10DD9000641C01958DF80040F0880822010A8DF876
:10DDA00001108DF8020069464846FEF7C5FF0120C4
:10DDB000F9F7ECF80095641C01958DF80040F8889F
:10DDC0000822010A8DF801108DF8020069464846C4
:10DDD000FEF7B2FF0120F9F7D9F80095641C019510
:10DDE0008DF80040B8F802000822010A8DF80110F1
:10DDF0008DF8020069464846FEF79EFF0120F9F7BC
:10DE0000C5F80095641C01958DF800403089082202
:10DE1000010A8DF801108DF8020069464846FEF7A8
:10DE20008BFF0120F9F7B2F80095641C01958DF87D
:10DE3000004030890822000A8DF80100B07A8DF880
:10DE4000020069464846FEF777FF0120F9F79EF881
:10DE50000095641C01958DF8004038890822010A5C
:10DE60008DF801108DF8020069464846FEF764FF00
:10DE70000120F9F78BF80095641C01958DF800409E
:10DE800078890822010A8DF801108DF80200694690
:10DE90004846FEF751FF0120F9F778F80095641C19
:10DEA00001958DF80040B8890822010A8DF801100B
:10DEB0008DF8020069464846FEF73EFF0120F9F75B
:10DEC00065F80095641C01958DF80040B8F80400D1
:10DED0000822010A8DF801108DF8020069464846B3
:10DEE000FEF72AFF0120F9F751F80095641C01950F
:10DEF0008DF80040B8F806000822010A8DF80110DC
:10DF00008DF8020069464846FEF716FF0120F9F732
:10DF10003DF80095641C01958DF80040B8F80800A4
:10DF20000822010A8DF801108DF802006946484662
:10DF3000FEF702FF0120F9F729F80095641C01950E
:10DF40008DF80040B0890822010A8DF801108DF883
:10DF5000020069464846FEF7EFFE0120F9F716F881
:10DF60000095641C01958DF80040F0890822010A93
:10DF70008DF801108DF8020069464846FEF7DCFE78
:10DF80000120F9F703F80095641C01958DF8004015
:10DF9000F8890822010A8DF801108DF802006946FF
:10DFA0004846FEF7C9FE0120F8F7F0FF0095641C13
:10DFB00001958DF80040388A0822010A8DF8011079
:10DFC0008DF8020069464846FEF7B6FE0120F8F7D4
:10DFD000DDFF0095641C01958DF80040788A0822C9
:10DFE000010A8DF801108DF8020069464846FEF7D7
:10DFF000A3FE0120F8F7CAFF0095641C01958DF877
:10E000000040B8F80A00C246010A8DF801108DF8E8
:10E010000200082269464846FEF78EFE0120F8F706
:10E02000B5FF0095641C01958DF80040B8F80C0010
:10E030000822010A8DF801108DF802006946484651
:10E04000FEF77AFE0120F8F7A1FF0095641C019508
:10E050008DF80040B8F80E000822010A8DF8011072
:10E060008DF8020069464846FEF766FE0120F8F783
:10E070008DFF0095641C01958DF80040308AB346F1
:10E08000010A8DF801108DF8020008226946484601
:10E09000FEF752FE0120F8F779FF0095641C019508
:10E0A0008DF80040708A0822010A8DF801108DF861
:10E0B000020069464846FEF73FFE0120F8F766FF7A
:10E0C0000095641C01958DF80040B88A0822010A69
:10E0D0008DF801108DF8020069464846FEF72CFEC7
:10E0E0000120F8F753FF0095641C01958DF800405E
:10E0F000B8F810000822010A8DF801108DF802000E
:10E1000069464846FEF718FE0120F8F73FFF0095E4
:10E11000641C01958DF80040B08A0822010A8DF830
:10E1200001108DF8020069464846FEF705FE012001
:10E13000F8F72CFF0095641C01958DF80040F08ADB
:10E140000822010A8DF801108DF802006946484640
:10E15000FEF7F2FD0120F8F719FF0095641C019508
:10E160008DF80040F88A0822010A8DF801108DF818
:10E17000020069464846FEF7DFFD0120F8F706FF7A
:10E180000095641C01958DF80040388B0822010A27
:10E190008DF801108DF8020069464846FEF7CCFD67
:10E1A0000120F8F7F3FE0095641C01958DF80040FE
:10E1B000B7F8A2000822010A8DF801108DF80200BC
:10E1C00069464846FEF7B8FD0120F8F7DFFE0095E6
:10E1D000641C01958DF80040B7F8A4000822010ADC
:10E1E0008DF801108DF8020069464846FEF7A4FD3F
:10E1F0000120F8F7CBFE0095641C01958DF80040D6
:10E20000308B0822010A8DF801108DF80200694652
:10E210004846FEF791FD0120F8F7B8FE0095641C12
:10E2200001958DF80040708B0822010A8DF80110CD
:10E230008DF8020069464846FEF77EFD0120F8F79A
:10E24000A5FE0095641C01958DF80040788B08228E
:10E25000010A8DF801108DF8020069464846FEF764
:10E260006BFD0120F8F792FE641C009504F0FF0896
:10E2700001958DF80080B88B0822010A8DF80110F5
:10E280008DF8020069464846943FFEF755FD01208F
:10E29000F8F77CFE2C460095019508F101058DF8F4
:10E2A0000050BAF81200D046010A8DF801108DF81E
:10E2B0000200082269464846FEF73EFD0120F8F7B5
:10E2C00065FE00946D1C01948DF80050B8F81400A0
:10E2D0000822010A8DF801108DF8020069464846AF
:10E2E000FEF72AFD0120F8F751FE00946D1C019401
:10E2F0008DF80050B7F8B2000822010A8DF801101D
:10E300008DF802006946484607F1B406FEF714FD91
:10E310000120F8F73BFE00946D1C8DF800508DF83D
:10E32000014001948DF80240082269464846FEF7F4
:10E3300003FD0120F8F72AFE00946D1C01948DF86E
:10E34000005030880822010A8DF801108DF8020073
:10E3500069464846FEF7F0FC0120F8F717FE0094E6
:10E360006D1C8DF800508DF8014001948DF802402D
:10E37000082269464846FEF7DFFC0120F8F706FE52
:10E3800000946D1C8DF800508DF8014001948DF8BB
:10E390000240082269464846FEF7CEFC0120F8F705
:10E3A000F5FD00946D1C01948DF80050B0788DF847
:10E3B0000100082269464846FEF7BEFC0120F8F736
:10E3C000E5FD00946D1C01948DF80050BBF81C0015
:10E3D0005F46010A8DF801108DF802000822694697
:10E3E0004846FEF7A9FC0120F8F7D0FD00946D1C0B
:10E3F00001948DF80050F88B0822010A8DF8011065
:10E400008DF8020069464846FEF796FC0120F8F7B1
:10E41000BDFD00946D1C01948DF80050B088082259
:10E42000010A8DF801108DF8020069464846FEF792
:10E4300083FC0120F8F7AAFD00946D1C01948DF86F
:10E440000050F0880822010A8DF801108DF80200B2
:10E4500069464846FEF770FC0120F8F797FD0094E6
:10E460006D1C01948DF80050388C0822010A8DF83B
:10E4700001108DF8020069464846FEF75DFC012058
:10E48000F8F784FD00946D1C01948DF80050788C91
:10E490000822010A8DF801108DF8020069464846ED
:10E4A000FEF74AFC0120F8F771FD00946D1C019401
:10E4B0008DF8005030890822010A8DF801108DF87E
:10E4C000020069464846FEF737FC0120F8F75EFD7A
:10E4D00000946D1C01948DF8005070890822010A87
:10E4E0008DF801108DF8020069464846FEF724FCBD
:10E4F0000120F8F74BFD00946D1C01948DF800503D
:10E50000B88C0822010A8DF801108DF802006946C6
:10E510004846FEF711FC0120F8F738FD00946D1C09
:10E5200001948DF80050F88C0822010A8DF8011032
:10E530008DF8020069464846FEF7FEFB0120F8F719
:10E5400025FD00946D1C01948DF80050B0890822BF
:10E55000010A8DF801108DF8020069464846FEF761
:10E56000EBFB0120F8F712FD00946D1C01948DF86F
:10E570000050B8F816000822010A8DF801108DF835
:10E58000020069464846FEF7D7FB0120F8F7FEFC7B
:10E5900000946D1C01948DF80050388D0822010AFA
:10E5A0008DF801108DF8020069464846FEF7C4FB5D
:10E5B0000120F8F7EBFC00946D1C01948DF80050DD
:10E5C000788D0822010A8DF801108DF80200694645
:10E5D0004846FEF7B1FB0120F8F7D8FC00946D1C0B
:10E5E00001948DF80050F0890822010A8DF801107D
:10E5F0008DF8020069464846FEF79EFB0120F8F7B9
:10E60000C5FC00946D1C01948DF80050308A0822DE
:10E61000010A8DF801108DF8020069464846FEF7A0
:10E620008BFB0120F8F7B2FC00946D1C01948DF86F
:10E630000050B88D0822010A8DF801108DF80200F3
:10E6400069464846FEF778FB0120F8F79FFC0094E6
:10E650006D1C01948DF80050F88D0822010A8DF888
:10E6600001108DF8020069464846FEF765FB01205F
:10E67000F8F78CFC00946D1C01948DF80050708AA2
:10E680000822010A8DF801108DF8020069464846FB
:10E69000FEF752FB0120F8F779FC00946D1C019401
:10E6A0008DF80050B08A0822010A8DF801108DF80B
:10E6B000020069464846FEF73FFB0120F8F766FC7A
:10E6C00000946D1C01948DF80050388E0822010AC8
:10E6D0008DF801108DF8020069464846FEF72CFBC4
:10E6E0000120F8F753FC00946D1C01948DF8005044
:10E6F000788E0822010A8DF801108DF80200694613
:10E700004846FEF719FB0120F8F740FC00946D1C09
:10E7100001948DF80050F08A0822010A8DF801104A
:10E720008DF8020069464846FEF706FB0120F8F71F
:10E730002DFC00946D1C01948DF80050308B082244
:10E74000010A8DF801108DF8020069464846FEF76F
:10E75000F3FA0120F8F71AFC00946D1C01948DF86F
:10E760000050B88E0822010A8DF801108DF80200C1
:10E7700069464846FEF7E0FA0120F8F707FC0094E6
:10E780006D1C01948DF80050F88E0822010A8DF856
:10E7900001108DF8020069464846FEF7CDFA0120C7
:10E7A000F8F7F4FB00946D1C01948DF80050708B09
:10E7B0000822010A8DF801108DF8020069464846CA
:10E7C000FEF7BAFA0120F8F7E1FB00946D1C019402
:10E7D0008DF80050B08B0822010A8DF801108DF8D9
:10E7E000020069464846FEF7A7FA0120F8F7CEFB7B
:10E7F00000946D1C01948DF80050B07F8DF80100DD
:10E80000082269464846FEF797FA0120F8F7BEFB52
:10E8100000946D1C01948DF80050306A8DF804004E
:10E82000010E8DF80110010C8DF80210010A8DF80F
:10E830000310082269464846FEF77EFA0120F8F7E1
:10E84000A5FB00946D1C01948DF80050B06D8DF8FF
:10E850000400010E8DF80110010C8DF80210010A60
:10E860008DF80310082269464846FEF765FA012034
:10E87000F8F78CFB6D1C0094EDB201948DF80050FC
:10E8800016F8300CB16D41436420B1FBF0F2120E6A
:10E890008DF80120B1FBF0F2120C8DF80220B1FBD3
:10E8A000F0F2B1FBF0F0120A8DF803208DF80400AD
:10E8B000082269464846FEF73FFA0120F8F766FB52
:10E8C00000946D1C01948DF8005096F824008DF88A
:10E8D0000100082269464846FEF72EFA0120F8F7A3
:10E8E00055FB00946D1C01948DF8005096F825009E
:10E8F0008DF80100082269464846FEF71DFA0120FE
:10E90000F8F744FB00946D1C01948DF80050F08CD6
:10E910000822010A8DF801108DF802006946484668
:10E92000FEF70AFA0120F8F731FB00946D1C019400
:10E930008DF8005096F857008DF8010008226946BE
:10E940004846FEF7F9F90120F8F720FB00946D1C0A
:10E9500001948DF80050D8F818008DF80400010ECD
:10E960008DF80110010C8DF80210010A8DF80310CA
:10E970004746082269464846FEF7DEF90120F8F7C7
:10E9800005FB00946D1C01948DF80050387F8DF8C4
:10E990000100082269464846FEF7CEF90120F8F743
:10E9A000F5FA00946D1C01948DF8005096F828003B
:10E9B0008DF80100082269464846FEF7BDF901209E
:10E9C000F8F7E4FA00946D1C01948DF8005096F865
:10E9D00029008DF80100082269464846FEF7ACF987
:10E9E0000120F8F7D3FA00946D1C01948DF80050C3
:10E9F000708D0822010A8DF801108DF80200694619
:10EA00004846FEF799F90120F8F7C0FA00946D1C0A
:10EA100001948DF8005096F82C008DF80100082222
:10EA2000694648465436FEF787F900946D1C0194F8
:10EA30008DF800509BF838008DF8010008226946D7
:10EA40004846FEF779F900946D1C01948DF800504A
:10EA500016F81C0C8DF8010016F81B0C8DF802003E
:10EA600016F81A0C8DF8030016F8190C8DF804002E
:10EA7000082269464846FEF75FF90120F8F786FA52
:10EA800000946D1C01948DF8005016F8180C8DF848
:10EA9000010016F8170C8DF8020016F8160C8DF808
:10EAA000030016F8150C8DF8040008226946484644
:10EAB000FEF742F90120F8F769FA00946D1C019401
:10EAC0008DF8005016F8140C8DF8010016F8130C90
:10EAD0008DF8020016F8120C8DF8030016F8110CD0
:10EAE0008DF80400082269464846FEF725F9012002
:10EAF000F8F74CFA00946D1C01948DF8005056F80C
:10EB0000100C8DF80400010E8DF80110010C8DF829
:10EB10000210010A8DF80310082269464846FEF7E4
:10EB20000BF90120F8F732FABD4800946D1C0194EE
:10EB30008DF8005001880A0A8DF801208DF8021026
:10EB400081788DF80310C1788DF8041041798DF823
:10EB5000051081798DF80610C0798DF8070008221C
:10EB600069464846FEF7E8F80120F8F70FFAAD4F7E
:10EB700000946D1C01948DF8005038788DF80100D8
:10EB800078788DF80200B8788DF80300F8788DF861
:10EB9000040038798DF80500082269464846FEF7DA
:10EBA000CBF80120F8F7F2F900946D1C01948DF870
:10EBB000005078798DF80100B8798DF80200F87965
:10EBC0008DF80300387A8DF80400787A8DF8050006
:10EBD000082269464846FEF7AFF80120F8F7D6F953
:10EBE00000946D1C01948DF80050B87A8DF80100E6
:10EBF000F87A8DF80200387B8DF80300787B8DF869
:10EC00000400B87B8DF80500082269464846FEF7E7
:10EC100093F80120F8F7BAF900946D1C01948DF86F
:10EC20000050307A8DF80100707A8DF80200B07AC9
:10EC30008DF80300F07A8DF80400307B8DF8050024
:10EC4000707B8DF80600082269464846FEF774F886
:10EC50000120F8F79BF900946D1C01948DF8005089
:10EC6000B07B8DF80100F07B8DF80200307C8DF8D0
:10EC70000300707C8DF80400B07C8DF80500F07CFA
:10EC80008DF80600082269464846FEF755F801202F
:10EC9000F8F77CF900946D1C01948DF80050307DDC
:10ECA0008DF80100707D8DF80200B07D8DF80300B5
:10ECB000F07D8DF80400307E8DF80500707E8DF8B3
:10ECC0000600082269464846FEF736F80120F8F7A4
:10ECD0005DF900946D1C01948DF80050B07E8DF8A4
:10ECE0000100F07E8DF80200307F8DF80300707F08
:10ECF0008DF80400B07F8DF80500F07F8DF80600D8
:10ED0000082269464846FEF717F80120F8F73EF951
:10ED100000946D1C01948DF8005096F829008DF830
:10ED20000100082269464846FEF706F80120F8F778
:10ED30002DF900946D1C01948DF80050708D0822FF
:10ED4000010A8DF801108DF8020069464846FDF76A
:10ED5000F3FF0120F8F71AF900946D1C01948DF867
:10ED60000050B08D0822010A8DF801108DF80200C4
:10ED700069464846FDF7E0FF0120F8F707F9BDE8CE
:10ED8000FF9F2DE9F043FDB04FF4FA71684604F09F
:10ED90009EFCDFF8948000254FF4C8796E464FF44E
:10EDA0008B7700BF03F075F808EB85214A4668466B
:10EDB00001F08AF80024311908223846FDF7BCFF1B
:10EDC0000120F8F7E3F80834A4B2892CF3D36D1CC2
:10EDD000ADB21E2DE6D37DB0BDE8F0830FB413486D
:10EDE0002DE9F047017801292AD1114A0021124C5E
:10EDF000118001709DF829C00E4A104BBDF82A0001
:10EE00009DF82A10BDF82C70BDF82E60ACF1370CBF
:10EE10000DF1290540F21519BCF1800F10D210E058
:10EE20007C0300204400002000780108300300200B
:10EE3000120000206E130020E00E0020AC13002012
:10EE400013E15FEA8C08F844D8F80680C744000054
:10EE50000002000008020000220200002C02000054
:10EE6000340200003C020000440200004E02000098
:10EE7000560200005E020000660200007002000000
:10EE80007A020000840200008C020000940200005C
:10EE90009C020000A4020000AC020000B6020000C8
:10EEA000C0020000CA020000D2020000DA02000024
:10EEB000E2020000EA020000F2020000FC02000090
:10EEC000040300000C030000140300001E030000F4
:10EED00028030000320300003C030000440300004C
:10EEE0004C030000560300006003000068030000AC
:10EEF000700300001A0200007A0300001A020000EA
:10EF00001A020000840300008C0300009403000038
:10EF10009C030000A6030000B0030000B80300003B
:10EF2000C0030000CA030000D4030000DC0300009B
:10EF3000E4030000EE030000F6030000FE030000FF
:10EF400006040000100400001A040000220400005F
:10EF50002A040000340400003E04000046040000BF
:10EF60004E04000058040000620400006A0400001F
:10EF7000720400007C04000088040000900400007B
:10EF8000A00400001A020000B0040000B804000051
:10EF9000C0040000CC040000D2040000E004000023
:10EFA000E4040000EC040000F4040000000500008C
:10EFB00008050000100500001C0500002A050000DF
:10EFC00038050000480500001A0200001A0200007F
:10EFD0001A02000070050000800500009005000086
:10EFE000A0050000C4050000CC050000D605000007
:10EFF0001A0200001A0200001A0200001A020000A1
:10F000001A0200001A0200001A0200001A02000090
:10F010001A0200001A0200001A0200001A02000080
:10F020001A0200001A0200001A0200001A02000070
:10F030001A0200001A020000E40500001406000095
:10F0400054060000700600007C0600008C060000DC
:10F0500040BA10804620EAE140BA50804720E6E1FD
:10F06000082229464846FDF767FEBDE8F0075DF82F
:10F0700014FB40BAA4F898000A20D8E140BA1880DE
:10F080006320D4E140BA90804820D0E140BAD080DB
:10F090004920CCE140BAA4F89A000B20C7E140BA5D
:10F0A00058806420C3E140BA10814A20BFE140BAD1
:10F0B00050814B20BBE140BAA4F89C000C20B6E183
:10F0C00040BAA4F89E000D20B1E140BAA4F8A00017
:10F0D0000E20ACE140BA98806520A8E140BAD88003
:10F0E0006620A4E140BA18816720A0E140BA90816F
:10F0F0004C209CE140BAD0814D2098E140BAA4F860
:10F10000A2000F2093E140BAA4F8A40010208EE1E1
:10F1100040BAA4F8A600112089E140BA58816820BD
:10F1200085E140BA9881692081E140BAD8816A209E
:10F130007DE140BA10824E2079E140BA50824F20E2
:10F1400075E140BAA4F8A800122070E140BA188214
:10F150006B206CE140BA9082502068E140BAD082C6
:10F16000512064E140BAA4F8AA0013205FE140BA3C
:10F17000A4F8AC0014205AE140BAA4F836014320A8
:10F1800055E140BAA4F83801442050E140BA108358
:10F1900052204CE140BA5083532048E140BAA4F8D1
:10F1A000AE00152043E140BAA4F8B00016203EE1BD
:10F1B00040BA58826C203AE140BA98826D2036E11C
:10F1C00040BAA4F8B200172031E140BAA4F8B40064
:10F1D00018202CE184F8B610192028E140BA908359
:10F1E000542024E140BAD083552020E140BAA4F84D
:10F1F000B8001A201BE140BAA4F8BA001B2016E19F
:10F2000040BA1084562012E140BA508457200EE1D3
:10F2100040BAA4F8BC001C2009E140BAA4F8BE0022
:10F220001D2004E140BA9084582000E140BAD08407
:10F230005920FCE040BAA4F8C0001E20F7E040BA14
:10F24000D8826E20F3E040BA10855A20EFE040BA31
:10F2500050855B20EBE040BAA4F8C2001F20E6E036
:10F2600040BAA4F8C4007220E1E040BA90855C2066
:10F27000DDE040BAD0855D20D9E040BAA4F8C600F0
:10F280002020D4E040BAA4F8C8007320CFE040BAF0
:10F2900010865E20CBE040BA50865F20C7E040BABF
:10F2A000A4F8CA002120C2E040BAA4F8CC00222071
:10F2B000BDE040BA90866020B9E040BAD0866120B7
:10F2C000B5E040BAA4F8CE002320B0E040BAA4F8DC
:10F2D000D0002420ABE000BF84F8D2102520A6E0A7
:10F2E00041BA78BA61F31F40C4F8D40026209EE0EA
:10F2F00041BA78BA61F31F40C4F80C01342096E09B
:10F3000084F8D810272092E084F8D91028208EE0C5
:10F3100040BAA4F8DA00292089E000BF84F80B1174
:10F320009EE641BA78BA61F31F40986170207EE092
:10F33000197795E684F8DC102A2078E084F8DD104F
:10F340002B2074E040BAA4F8DE002C206FE000BF50
:10F3500084F8E0102D206AE082F83810622066E020
:10F36000FD48DDF82A10C0F8EC1079E6FA48DDF81F
:10F370002A10C0F8F010302059E0F748DDF82A10C4
:10F38000C0F8F410312052E041BA78BA61F31F405E
:10F39000C4F8F80032204AE041BAF04801809DF8F4
:10F3A0002C1081709DF82D10C1709DF82E104171A8
:10F3B0009DF82F1081719DF83010C171712036E0D9
:10F3C000E548DDF82A10C0F81011A0F8146147E6EE
:10F3D000E148DDF82A10C0F81611A0F81A613FE6DE
:10F3E000DD48DDF82A10C0F81C11A0F8206137E6CE
:10F3F000D948DDF82A10C0F82211A0F8266135207E
:10F40000FBF745FF3620FBF742FF3720FBF73FFFB6
:10F4100038200CE084F83111402008E040BAA4F80C
:10F420003201412003E040BAA4F834014220FBF746
:10F430002EFF15E684F82811082229464846FDF7D4
:10F440007BFCC7A004F0D6FE94F8280101287FF4C5
:10F450000CAEF8F750F9F8F7F1FA012080F31088B4
:10F4600000F093FA082229464846FDF765FCC1489A
:10F4700041680A68806882430A6041F28834204605
:10F48000F7F784FDBC4A51680868926890430860A9
:10F49000BA494868026889688A4302602046F7F7DB
:10F4A00075FDE2E584F82911082229464846FDF752
:10F4B00043FC94F829010128F3D1FDF775F8D4E550
:10F4C000082229464846FDF737FCC6E708222946A8
:10F4D0004846FDF731FCFDF758FEC6E508222946EF
:10F4E0004846FDF729FCFFF74CFCBEE52DE9F0414D
:10F4F000A34F0020984BF8603861B3F880200A20B1
:10F50000B2FBF0F107F10C04090A2170B2FBF0F133
:10F510006170B3F8821042F21075691A91FBF0F035
:10F52000010AA170E07093F884002071954800787A
:10F5300060719548B3F892100678184651EA0605AE
:10F54000B0F894C004D15FEA8C7001D0012003E0D0
:10F5500002205FEA8C7E02D040F00C0004E05FEAFB
:10F56000CC7C01D040F00400DFF820C2DCF800E0E1
:10F57000DEF800E0DCF808C01EEA0C0FDFF810C26D
:10F58000BCF840C003D1BCF1000F42D002E0BCF196
:10F59000000F01D040F04000A07100205FEA816CB4
:10F5A00000D508205FEA416C00D508205FEAC17CE5
:10F5B00000D00C205FEA415C00D510205FEA015CBE
:10F5C00000D514205FEAC16C00D518205FEA815C89
:10F5D00000D51C205FEA817C00D5242006B12820BC
:10F5E0005FEA017C00D530203F7907B134204F0716
:10F5F00000D53820B3F89870974200D83C20B3F873
:10F600009AC0944500D34020534BB3F8C0301DB18D
:10F6100008E040F08000BFE7002B03DD974201D9EE
:10F6200094450BD3012908D13EB9002B05DD974243
:10F6300003D9944501D2401C00E0C01C5049E07140
:10F6400008220C315348FDF78DFBBDE8F0410A203C
:10F65000F7F79CBC4A4810B50022C26002614E48D0
:10F660000A210388B3FBF1F0040AB3FBF1F3444829
:10F670000C3004704370494B1B88B3FBF1F4B3FBAF
:10F68000F1F1240A8470C170454909780171454936
:10F69000427109788171C271014608224248FDF722
:10F6A00061FBBDE810400A20F7F770BC2DE9F04F70
:10F6B000002087B0324904900390C8600446034696
:10F6C0000861334800221146B0F942903748B0F93A
:10F6D00000B03748B0F900A03648B0F900C036484D
:10F6E000B0F900703548B0F90060ADF80090ADF8A1
:10F6F00004A0ADF80870ADF802B0ADF806C0ADF8E2
:10F700000A60684601E000210FE000EB410E30F98D
:10F710001180BEF90250A84505DD0595AEF80280BE
:10F72000059D20F81150491CC9B2C2F105058D4252
:10F73000EBDC521CD2B2052AE5D3114DBDF80A10FC
:10F740000C3529705FF00001049A30F91180904562
:10F7500036D10C4638E00000E00E00207C0300208B
:10F760004E5649435F53797374656D526573657482
:10F770000D0A0000D00A0020F40A0020880A0020A8
:10F78000300300202E03002085000020180B0020ED
:10F7900054140020000F710CA2000020A4000020CF
:10F7A0008700002086000020000F7418B60000209B
:10F7B000B8000020BA000020BC000020BE000020DD
:10F7C000491CC9B20329BFD3ADF80090ADF804A01D
:10F7D000ADF808700022ADF802B0ADF806C0ADF883
:10F7E0000A60114601E000210DE000EB410730F90D
:10F7F00011C0B7F90260B44503DAA7F802C020F8D7
:10F800001160491CC9B2C2F105068E42EDDC521CE2
:10F81000D2B2052AE7D3BDF80A1069705FF0000183
:10F82000039A30F91160964201D10B4603E0491C5E
:10F83000C9B20329F4D3AB700020E8702C71687151
:10F84000A871E871082256495648FDF78BFA0A203C
:10F85000F7F79CFB07B0BDE8F08F514810B50C38A6
:10F860000021C16001610C304F4A017092F83820CC
:10F87000427006228270C170017141718171C17143
:10F88000014608224948FDF76DFABDE810400A20FC
:10F89000F7F77CBB2DE9F041414900220C39404883
:10F8A000CA60414B0A6102701E8F4B799E4201D99A
:10F8B000437001E042704A714D793D4C0A23AE42DB
:10F8C0000DD934F815706D1CB7FBF3FCB7FBF3F7DB
:10F8D0004FEA1C2C80F802C0C7704D7101E08270A5
:10F8E000C270EDB2AE420DD934F815706D1CB7FB85
:10F8F000F3FCB7FBF3F74FEA1C2C80F804C0477108
:10F900004D7101E002714271EDB2AE420BD934F893
:10F910001520B2FBF3F4B2FBF3F2240A8471C27136
:10F920006D1C4D7101E08271C27108221C49214891
:10F93000FDF718FABDE8F0410A20F7F727BB184891
:10F9400010B50C380021C1600161174890F84220C1
:10F9500013480270184A12784270184A127882705E
:10F96000174A1278C270174A12780271164A127832
:10F9700042718171C171014608221448FDF7F2F904
:10F98000BDE810400A20F7F701BB11480168114A91
:10F9900001F4E06111430160BFF34F8FFEE7000007
:10F9A0003C030020000F751854140020000F791834
:10F9B00000090020000F7218B6000020B8000020D7
:10F9C000BA000020BC000020BE000020000F731809
:10F9D0000CED00E00400FA0570B5012190B0084676
:10F9E00002F035FC0121480202F03EFC454E304653
:10F9F00001F002FC44480090444801A90024042579
:10FA000081E831008020CDE904404000069080006C
:10FA10000790202008900002CDE90904694630468D
:10FA200001F08CFC0121304601F0B3FC01208DF87F
:10FA300030008DF831000B944FF46020CDE90D04B7
:10FA4000314C8DF83C504C3C0BA9204600F079FC21
:10FA50004FF4404002F06CFB012205231146204682
:10FA600000F007FD052302220621204600F001FDDB
:10FA7000052303220721204600F0FBFC0523042276
:10FA80000821204600F0F5FC0121204600F090FC02
:10FA90000121204600F081FC204600F0A0FC204619
:10FAA00000F0A2FC0028FAD1204600F0A7FC204676
:10FAB00000F0A9FC0028FAD10121204600F0ADFC9D
:10FAC00010B070BD38B50121042002F0CDFBC2207A
:10FAD000ADF8000000248DF8034069460C4802F0A0
:10FAE00081F80121082002F0BFFB0120ADF80000E1
:10FAF0008DF803406946074802F074F8BDE83840C5
:10FB00006AE70000080002404C2401407003002016
:10FB100000080140000C0140F0B5A2490E888F7822
:10FB2000CC784B798A79CD79BF1E66F30F0017F038
:10FB3000FF0164F31F6061F317404FF00C0704D11D
:10FB400067F31740761E66F30F0081B26426B1FB9F
:10FB5000F6F6C6EB91063444C0F3074040F26F1C42
:10FB60004FF4C87600FB0CF0B1FBF6F6B0FBF7F0F3
:10FB70003044204440F26D1401FB04008A490844DB
:10FB800000EB400003EBC000C0EB001002EB800074
:10FB9000C0EB001005EB8000F0BD81070CD16421A3
:10FBA000B0FBF1F201FB120141B94FF4C871B0FB97
:10FBB000F1F201FB120008B10020704701207047EC
:10FBC00030B56424B0FBF4F3B0FBF4F5DBB204FB16
:10FBD0001500132B01D96430C0B200EB9004072349
:10FBE000B4FBF3F503FB1544704D22440D4480072C
:10FBF00015F8015C2A4492B203D1032901D2521EA6
:10FC000092B2B2FBF3F003FB102030BD2DE9F041BE
:10FC1000FFF782FF461CDFF898C16248B6FBFCF391
:10FC2000001F041D0188994230D0038040F2B27554
:10FC30004FF4B7784FF4B6770FE02846FFF7ADFFE3
:10FC400038B1434502D3A3F5B77304E06D1CADB2E0
:10FC500005E0A3F26D136D1CADB2BB42EDD825805B
:10FC6000524F00250C370BE02088FFF796FF08B1B4
:10FC7000012D2DD0785D984204D81B1A6D1CADB2B1
:10FC80001C2BF1D26D1CA5705B1CE370B6FBFCF065
:10FC90000CFB10604FF46161B0FBF1F26271B0FBDC
:10FCA000F1F201FB12033C22B3FBF2F3A371B0FBB0
:10FCB000F1F301FB1300B0FBF2F102FB1100E07164
:10FCC000E278A1782088FFF77BFF2071BDE8F08102
:10FCD0001D2BD7D31D3BD1E72DE9F041FFF71CFFCA
:10FCE00000F11906DFF8C8C02E48B6FBFCF3001F70
:10FCF000041D4188994230D0438040F2B2754FF4E0
:10FD0000B7784FF4B6770FE02846FFF746FF38B1D3
:10FD1000434502D3A3F5B77304E06D1CADB205E013
:10FD2000A3F26D136D1CADB2BB42EDD825801F4F01
:10FD300000250C370BE02088FFF72FFF08B1012DBD
:10FD40002CD0785D984204D81B1A6D1CADB21C2BC8
:10FD5000F1D26D1CA5705B1CE370B6FBFCF00CFBD4
:10FD600010604FF46161B0FBF1F26271B0FBF1F22F
:10FD700001FB12033C22B3FBF2F3A371B0FBF1F3DE
:10FD800001FB1300B0FBF2F102FB1100E071E2781D
:10FD9000A1782088FFF714FF207197E71D2BD8D397
:10FDA0001D3BD2E77C0300207505F5FF505001088C
:10FDB00080510100008870472DE9F04116460F463A
:10FDC0000546002408E000BF37F81410284601F06B
:10FDD00032FD641CA4B2AD1CB442F5D3BDE8F08181
:10FDE00010B5002306E000BF30F8024B21F81340A5
:10FDF0005B1C9BB29342F7D310BD2DE9F05FA0F1DD
:10FE0000006415468A468346B4F5003F54D201F09B
:10FE1000CAFBA70AC4F34806C6F50074A54200D879
:10FE20002C46DFF8109200BF4FF0006000EB8720F7
:10FE300080464FF400727F49FFF7D2FF00204FF653
:10FE4000FF7106E0331839F813208A4203D1401CB1
:10FE500080B2A042F6D3A04226D2404601F0E8FB91
:10FE60000020494607E000BF3AF810208319401CE3
:10FE700021F8132080B2A042F6D36E4940464FF4D9
:10FE8000007200BFFFF798FFA54211D0281B0AEBB4
:10FE9000440A0BEB440B002685B24FF400747F1C20
:10FEA000A542C1D82C46BFE7224651465846E9E74D
:10FEB000BDE8F05F01F083BBBDE8F09F13B5012200
:10FEC00001A9FFF79AFF1CBD70B5ADF5006D0E4698
:10FED000044615464FF40061684603F0F8FB05F050
:10FEE000010000EB5505AAB269463046FFF778FFDE
:10FEF000002069460BE000BF31F8102004EB4003FE
:10FF0000120A04F8102011F810205A70401CA84260
:10FF1000F2D30DF5006D70BD70B5ADF5006D0E46F8
:10FF2000054614464FF40061684603F0D0FB04F028
:10FF3000010000EB540100206A4606E005EB400397
:10FF40001B885BBA22F81030401C8842F6D38AB274
:10FF500069463046FFF751FFDBE770B5ADF5006D40
:10FF60000E46054614464FF40061684603F0AFFBA9
:10FF700004F0010000EB540100206A4606E000BFD7
:10FF800005EB40031B8822F81030401C8842F7D351
:10FF90008AB269463046FFF730FFBAE7F0B581B064
:10FFA000ADF5805D0E4605466C4617464FF4805110
:10FFB000204603F08CFB07F0010000EB5701002006
:10FFC00006E000BF05EB4002128824F81020401C18
:10FFD0008842F7D38AB221463046FFF70EFF01B0C0
:10FFE0000DF5805DF0BDF0B581B0ADF5805D0F46DB
:10FFF00006466C4615464FF48051204603F067FBD9
:020000040801F1
:1000000005F0010000EB5505AAB221463846FFF77E
:10001000E7FE00200BE000BF34F8101006EB4002B2
:10002000090A06F8101014F810105170401CA8426C
:10003000F2D3D4E7B22500200CB500200190009047
:100040006C48006840F480306A49086000BF694825
:10005000006800F4003000900198401C0190009866
:1000600018B90198B0F5A06FF1D16248006800F4AA
:10007000003010B10120009001E0002000900098B5
:10008000012843D15C48006840F010005A490860DC
:100090000846006820F0030008600846006840F049
:1000A000020008605348406852494860084640686A
:1000B00048600846406840F48060486008464068F0
:1000C00020F47C1048600846406840F4E81048601E
:1000D0000846006840F08070086000BF454800682E
:1000E00000F000700028F9D04248406820F003007A
:1000F000404948600846406840F00200486000BF40
:100100003C48406800F00C000828F9D10CBD10B53F
:10011000FFF792FF10BD10B53648006840F00100AF
:10012000344908600846406834490840314948600D
:1001300008460068324908402E49086008460068B1
:1001400020F4802008600846406820F4FE004860E3
:100150004FF41F008860FFF7DAFF4FF00060294975
:10016000086010BD10B5002100200022214B5B6803
:1001700003F00C0121B1042906D0082928D107E099
:10018000214B224C236027E01F4B204C236023E0AF
:10019000184B5B6803F47010164B5B6803F48032F5
:1001A000022303EB904022B9194B4343174C2360C1
:1001B0000DE0104B5B6803F4003323B1144B434351
:1001C000124C236003E0104B4343104C236003E0C8
:1001D0000D4B0E4C236000BF00BF064B5B68C3F3A2
:1001E00003130C4CE15C094B1B68CB40074C2360AC
:1001F00010BD000000100240002002400000FFF887
:10020000FFFFF6FE08ED00E000127A0084030020F4
:1002100000093D008803002031490143314A116043
:10022000704770B5002100230F22C47804B32D4C11
:10023000246804F4E064C4F5E064210AC1F1040315
:10024000CA40447804FA03F1847814402143090138
:10025000254C0678A155047804F01F050124AC4014
:1002600005786D11AD0005F1E025C5F8004109E004
:10027000047804F01F050124AC401C4D067876116B
:1002800045F8264070BD1A4A0A400243154B1B1F11
:100290001A60704739B1134A121D12680243114B9C
:1002A0001B1D1A6006E00F4A121D126882430D4B97
:1002B0001B1D1A607047042808D14FF0E02109691E
:1002C00041F004014FF0E022116107E04FF0E0211E
:1002D000096921F004014FF0E0221161704700002C
:1002E0000000FA050CED00E000E400E080E100E031
:1002F00080FFFF1F10B50446FA48844208D101214F
:10030000401501F0CBFF0021601501F0C7FF17E099
:10031000F548844208D10121001501F0BFFF0021FA
:10032000201501F0BBFF0BE0F048844208D1012109
:10033000C80301F0B3FF00214FF4004001F0AEFF0D
:1003400010BD30B50246002000235068E84C204024
:100350000D790C6844EA0524204350609068E54C10
:100360002040D1E902542C434D7944EA450420430E
:100370009060D06A20F470000C7C641EE4B22343C9
:1003800040EA0350D06230BD00210160017141712B
:100390008160C16001210174704721B1826842F01F
:1003A0000102826003E0826822F0010282607047ED
:1003B00021B1826842F48072826003E0826822F494
:1003C00080728260704710B50023CBB21AB14468C6
:1003D0001C43446002E044689C43446010BD816853
:1003E00041F0080181607047014600208A6802F0F0
:1003F00008020AB1012000E000207047816841F046
:10040000040181607047014600208A6802F00402FE
:100410000AB1012000E00020704721B1826842F457
:10042000A002826003E0826822F4A002826070472A
:10043000014600208A6802F480020AB1012000E02F
:100440000020704710B50A4600210023416821F4BE
:100450006041531E41EA4331416010BD21B1426801
:1004600042F40062426003E0426822F400624260AB
:100470007047F0B504460D4600200021092D11DD1E
:10048000E068A5F10A0606EB4607072606FA07F11B
:100490008843A5F10A0606EB460603FA06F108436F
:1004A000E0600CE0206905EB4507072606FA07F136
:1004B000884305EB450603FA06F108432061072A45
:1004C0000FDA606B561E06EB86071F2606FA07F149
:1004D0008843561E06EB860605FA06F1084360635C
:1004E00022E00D2A0FDA206BD61F06EB86071F26A7
:1004F00006FA07F18843D61F06EB860605FA06F1D1
:100500000843206310E0E06AA2F10D0606EB8607BF
:100510001F2606FA07F18843A2F10D0606EB8606B0
:1005200005FA06F10843E062F0BD21B1826842F4A9
:100530008012826003E0826822F480128260704739
:100540000146C86C80B2704766484C3000687047FE
:1005500021B1426842F48062426003E0426822F4C2
:1005600080624260704721B1426842F4805242602A
:1005700003E0426822F48052426070470A4600213C
:10058000816821F4E04111438160704721B18268A4
:1005900042F40042826003E0826822F400428260FA
:1005A000704721B1826842F40212826003E08268DF
:1005B00022F4021282607047014600208A6802F429
:1005C00000120AB1012000E000207047F0B5044697
:1005D0001546002000220026092911DDE068A1F15E
:1005E0000A0707EB470C072707FA0CF29043A1F123
:1005F0000A0707EB470703FA07F21043E0600CE035
:10060000206901EB410C072707FA0CF2904301EB3C
:10061000410703FA07F210432061A06BC0F30156B3
:10062000EF1C06F1010CA7EB0C0707EB870C1F274B
:1006300007FA0CF29043EF1C06F1010CA7EB0C0734
:1006400007EB870701FA07F21043A063F0BD10B56E
:100650000A4600210023816B21F44011531E41EA18
:100660000351816310BD08B5002300930090009BE7
:100670000B440093009B1A6008BD08B50246002099
:100680000090009201F12800009B1844009000980F
:10069000006880B208BD0A4600214168164B194027
:1006A0001143416070474162826270470A460021EF
:1006B000416821F01F0111434160704740B1094971
:1006C0000831096841F40001064A0832116007E068
:1006D00004490831096821F40001024A0832116016
:1006E000704700000024014000280140003C014008
:1006F000FFFEF0FFFDF7F1FFFFFD3FFF0246002088
:1007000013680B400BB1012000E000207047CA4382
:100710000260704770B502460020002300240B12CF
:100720005568CEB205EA060415681D4015B10CB136
:10073000012000E0002070BD00220A12D3430360B4
:100740007047000010B5012001F0C2FD002001F04B
:10075000BFFD10BD2A49086070472949091F08607C
:100760007047274984310860704701460020254AB8
:1007700010884FF67F4210400843224A108070478D
:10078000014600201F4A10884FF68072104008432F
:100790001C4A1080704708B500220092194A2C3A72
:1007A0000092009A02440092009A116008BD08B5B8
:1007B00001460020009013482C380090009808440F
:1007C00000900098008808BD0D489C300068C0B2B9
:1007D00070470C480830008840F001000949083192
:1007E000088070470648A0300068C0B270470548CE
:1007F0000830008840F00200024908310880704744
:1008000004860D422C6C004010B50446FE4884421C
:1008100009D10121480601F04EFD00214FF0007082
:1008200001F049FD08E00121880601F044FD0021A6
:100830004FF0806001F03FFD10BD30B50246002052
:100840000023146824F002041460146844F00104C6
:10085000146000E05B1C546804F001041CB94FF6FE
:10086000FF74A342F6D1546804F001040CB90020CF
:100870006CE08C79012C04D1146844F0800414607D
:1008800003E0146824F080041460CC79012C04D1B6
:10089000146844F04004146003E0146824F0400439
:1008A00014600C7A012C04D1146844F02004146004
:1008B00003E0146824F0200414604C7A012C04D165
:1008C000146844F01004146003E0146824F0100469
:1008D00014608C7A012C04D1146844F0080414606C
:1008E00003E0146824F008041460CC7A012C04D1CD
:1008F000146844F00404146003E0146824F0040451
:1009000014608C78A407CD7844EA05640D7944EA34
:1009100005444D7944EA05540D886D1E2C43D4617D
:10092000146824F001041460002300E05B1C546888
:1009300004F001041CB14FF6FF74A342F6D15468D1
:1009400004F001040CB1002000E0012030BD10B51E
:100950000021837A012202FA03F1AC4A126842F0C4
:100960000102AA4B1A60A94A1C3212688A43A74B9B
:100970001C331A60027BCAB9A44A0C3212688A433B
:10098000A24B0C331A604288C38842EA03439F4A51
:100990004032847A42F834300288838842EA034342
:1009A0009A4A4032847A02EBC4025360027B012AE5
:1009B00019D1964A0C3212680A43944B0C331A60D0
:1009C0004288038842EA0343904A4032847A42F8DC
:1009D0003430C288838842EA03438C4A4032847AA6
:1009E00002EBC4025360C27A3AB9884A121D1268F7
:1009F0008A43864B1B1D1A6006E0844A121D12684A
:100A00000A43824B1B1D1A60028932B97F4A143295
:100A100012688A437D4B14331A600289012A06D179
:100A20007A4A143212680A43784B14331A60427BB4
:100A3000012A06D1754A1C3212680A43734B1C33D3
:100A40001A60724A126822F00102704B1A6010BDDF
:100A500000218171C171017241728172C172817014
:100A6000C170032101710221417101210180704790
:100A70006649096841F00101644A1160114609683C
:100A800043F60E729143614A11601146096841EACA
:100A9000002111601146096821F0010111607047C1
:100AA00021B1026842F48032026003E0026822F45D
:100AB000803202607047E1B1026842F08002026059
:100AC0004FF4C272125842F480734FF4C272135042
:100AD0004FF4CA72125842F480734FF4CA72135022
:100AE0004FF4D272125842F480734FF4D272135002
:100AF0001BE0026822F0800202604FF4C2721258BA
:100B000022F480734FF4C27213504FF4CA72125819
:100B100022F480734FF4CA7213504FF4D2721258F9
:100B200022F480734FF4D2721350704710B502460E
:100B30000020936803F08063B3F1806F00D110E070
:100B4000936803F00063B3F1006F01D1012008E066
:100B5000936803F08053B3F1805F01D1022000E07D
:100B60000420042879D002F5C07303EB00131B683E
:100B700003F0010402F5C07303EB00131C600B7A51
:100B80007BB94B7A0C8843EA445302F5C07404EBFA
:100B900000142468234302F5C07404EB001423609E
:100BA00010E00B7A4C6843EAC4034C7A234302F505
:100BB000C07404EB00142468234302F5C07404EBF2
:100BC000001423608B7A03F00F038B7202F5C0735D
:100BD00003EB00135B6823F00F0402F5C07303EB13
:100BE00000135C6002F5C07303EB00135B688C7A42
:100BF000234302F5C07404EB001463608B7B1C0676
:100C00004B7B44EA034403E000640040006600407C
:100C10000B7B44EA0323CC7A234302F5C07404EB34
:100C20000014A3608B7C1C064B7C44EA03440B7CC1
:100C300044EA0323CC7B234302F5C07404EB001485
:100C4000E36002F5C07303EB00131B6843F001047B
:100C500002F5C07303EB00131C6010BD10B5024613
:100C6000002321B1012907D002290FD109E09068A2
:100C7000F94C00EA04030BE09068F84C00EA040326
:100C800006E09068F64C00EA040301E0002300BF90
:100C900000BFF44C181BA34216D007DC83B16FF0E1
:100CA0008060184470B1022818D111E0B0F5007FBF
:100CB00010D0ED4C204448B1B0F5003F0ED10BE010
:100CC00002230DE000230BE0002309E0002307E0EE
:100CD000012305E0012303E0012301E0002300BF1D
:100CE00000BFD8B210BD21B1012907D002290FD110
:100CF00009E0826842F0800282600AE0826842F481
:100D00000042826005E0826842F40002826000E0F6
:100D100000BF00BF704710B500F5D87303EB011397
:100D20001B6803F004031372137A53B900F5D873E8
:100D300003EB01131B6840F2FF7404EA5353136082
:100D400009E000F5D87303EB01131B686FF06044F2
:100D500004EAD303536000F5D87303EB01131B6857
:100D600003F00203537200F5D87303EB01135B68C1
:100D700003F00F03937200F5D87303EB01135B6864
:100D80001B0AD37400F5D87303EB01139B68D3726D
:100D900000F5D87303EB01139B681C0A147300F56C
:100DA000D87303EB01139B681C0C547300F5D873C4
:100DB00003EB01139B681B0E937300F5D87303EBD1
:100DC0000113DB68D37300F5D87303EB0113DB6801
:100DD0001C0A147400F5D87303EB0113DB681C0CB8
:100DE000547400F5D87303EB0113DB681B0E937486
:100DF00021B9C36843F02003C36003E0036943F0F3
:100E00002003036110BD21B9C26842F02002C26014
:100E100003E0026942F020020261704702460020AE
:100E200019B9D36803F0030006E0012903D113695F
:100E300003F0030000E00020704710B502460B46A7
:100E400000204FF6FF71BBB9146824F0020444F08F
:100E50000104146000E0491E546804F00304012CEE
:100E600001D00029F7D1546804F00304012C01D00B
:100E7000002032E0012030E0012B13D1146824F06F
:100E80000304146000E0491E546804F003040CB12C
:100E90000029F8D1546804F003040CB100201CE0D0
:100EA00001201AE0022B17D1146824F0010444F049
:100EB0000204146000E0491E546804F00304022C8C
:100EC00001D00029F7D1546804F00304022C01D0AA
:100ED000002002E0012000E0002010BD01460020BB
:100EE0000A6822F0010242F002020A604A6802F037
:100EF0000302022A00D10120704701464FF6FF721B
:100F000000200B6823F002030B6000E0521E4B68C8
:100F100003F00203022B01D1002AF7D14B6803F042
:100F20000203022B00D001207047014600208A698D
:100F300002F070007047014600208A69100E704769
:100F4000014600208A69C2F3074070471AB143691D
:100F50000B43436102E043698B434361704710B523
:100F60000246002001F4700343B19369C1F31304F6
:100F700023400BB101202DE000202BE001F0807315
:100F800043B15368C1F3130423400BB1012021E0A6
:100F900000201FE001F0006343B19368C1F3130424
:100FA00023400BB1012015E0002013E001F0007395
:100FB00043B1D368C1F3130423400BB1012009E00E
:100FC000002007E01369C1F3130423400BB1012093
:100FD00000E0002010BD0022244B994202D10023E2
:100FE000836111E0C1F3130201F000730BB1C26021
:100FF0000AE001F080630BB1026105E001F00063DB
:101000000BB1826000E0426070470246002002EAB5
:1010100001030BB1012000E00020704770B50446C9
:101020000D46002660692840002872D0B5F5807F03
:1010300069D01DDC082D42D006DC012D2DD0022DFB
:1010400031D0042D7FD134E0102D3ED0202D42D060
:10105000402D78D145E000000300000400030008A3
:1010600000000310000100080001FFF77000F030DD
:10107000B5F5004F61D009DCB5F5007F4AD0B5F574
:10108000806F4DD0B5F5006F5DD150E0B5F5803F74
:101090002DD0B5F5003F56D12FE0A0685549FFF798
:1010A000B4FF064651E0E0680321FFF7AEFF0646B5
:1010B0004BE0E0680821FFF7A8FF064645E0E0683E
:1010C0001021FFF7A2FF06463FE020690321FFF74A
:1010D0009CFF064639E020690821FFF796FF064687
:1010E00033E020691021FFF790FF06462DE060688D
:1010F0000821FFF78AFF064627E060681021FFF706
:1011000084FF064621E0A0690121FFF77EFF064625
:101110001BE01BE0A0690221FFF777FF064614E001
:10112000A0690421FFF771FF06460EE00BE0A069FD
:101130007021FFF76AFF064607E060680421FFF7A9
:1011400064FF064601E0002600BF00E000263046AE
:1011500070BDB1F5007F3AD00FDC202928D006DC25
:1011600001291CD004291DD0082940D11DE04029A7
:1011700021D0B1F5807F3AD126E0B1F5004F31D0D2
:1011800006DCB1F5806F25D0B1F5006F2FD124E0DA
:10119000B1F5803F12D0B1F5003F28D111E0154ADA
:1011A000826025E00822C26022E01022C2601FE0B7
:1011B000082202611CE01022026119E0082242604C
:1011C00016E01022426013E00422426010E0042284
:1011D00042600DE0042242600AE0002282610422A3
:1011E000426005E0002282610422426000E000BF0C
:1011F00000BF70470101010001684FF6FE72114007
:1012000001600021016041608160C1608D498842B8
:1012100008D18C490839496841F00F01894A083AD8
:1012200051608AE087491431884208D185490839DC
:10123000496841F0F001834A083A51607DE08149F4
:101240002831884208D17F490839496841F47061E2
:101250007C4A083A516070E07A493C31884208D1B2
:1012600078490839496841F47041764A083A516032
:1012700063E074495031884208D17249083949689D
:1012800041F470216F4A083A516056E06D4964316B
:10129000884208D16B490839496841F47001694AAC
:1012A000083A516049E067497831884208D1654978
:1012B0000839496841F07061624A083A51603CE07F
:1012C0006149884206D1011F096841F00F01021FE0
:1012D000116032E05C491431884208D15A49091F33
:1012E000096841F0F001584A121F116025E0564983
:1012F0002831884208D15449091F096841F47061B6
:10130000514A121F116018E04F493C31884208D100
:101310004D49091F096841F470414B4A121F116081
:101320000BE049495031884207D14749091F0968F4
:1013300041F47021444A121F1160704710B5002219
:10134000026847F6F0739A430C6A8B6823430C6972
:1013500023434C6923438C692343CC6923434C6A60
:1013600023438C6A23431A430260CB6843600B68B3
:1013700083604B68C36010BD0021016041608160E3
:10138000C160016141618161C1610162416281624B
:10139000704721B1026842F00102026004E0026875
:1013A0004FF6FE731A40026070471AB103680B4390
:1013B000036002E003688B4303607047416070473D
:1013C0000146486880B2704701460020002201F0C3
:1013D00080531BB11C4B083B1A6802E0194B083BB9
:1013E0001A6802EA01030BB1012000E000207047F7
:1013F00000F0805119B11449091F086002E0114939
:1014000008394860704701460020002201F08053EF
:101410001BB10D4B083B1A6802E00A4B083B1A68E7
:1014200002EA01030BB1012000E00020704700F048
:10143000805119B10449091F086002E001490839C7
:1014400048607047080002400804024000204449F8
:101450000860091D0860091D0860091D08604148F1
:101460003F4914310860704700213D498279002AC4
:101470003AD00A46126803689A430B461A600A1D5E
:10148000126803689A430B1D1A60027911440A68B6
:1014900003681A430A60324A0832126803689A43A2
:1014A0002F4B08331A601A1D126803689A432C4B9D
:1014B0000C331A604279102A0ED11A1F1268036881
:1014C0001A43274B08331A601A1D126803681A431F
:1014D000234B0C331A600DE02149427911440A680C
:1014E00003681A430A6005E0027911440A68036838
:1014F0009A430A6070470021016001710C2141711B
:101500000021817170471649103109680143144A5E
:1015100010321160704701460020114A14321268DF
:101520000A400AB1012000E0002070470C49143144
:1015300008607047014600200022094B1B6803EA3F
:101540000102074B14331B680B4013B10AB1012091
:1015500000E0002070470249143108607047000025
:1015600000040140FFFF0F0001460020FE4A106802
:1015700000F03800084310607047FB49096821F00B
:101580000801F94A1160114609680143116070476A
:10159000F549096821F01001F34A11601146096804
:1015A000014311607047F148EF494860F0484860D6
:1015B0007047EE48EC494860ED4848607047EA489B
:1015C000006940F08000E84908617047E64800691A
:1015D00040F08000E449086170470420E249C9688E
:1015E00001F0010109B101200EE0DF49C96801F0F5
:1015F000040109B1022007E0DB49C96801F01001CC
:1016000009B1032000E00420704700B5024604231E
:10161000FFF7E3FF034603E0FFF7DFFF0346521E39
:10162000012B01D1002AF7D102B90523184600BDCC
:1016300030B5044604254FF43020FFF7E6FF054699
:10164000042D17D1C848006940F00200C64908615E
:1016500008464461006940F0400008614FF43020C2
:10166000FFF7D3FF0546C048006941F6FD71084009
:10167000BD490861284630BD10B504244FF4302020
:10168000FFF7C3FF0446042C16D1B748006940F0A9
:101690000400B54908610846006940F0400008614F
:1016A0004FF43020FFF7B1FF0446AF48006941F620
:1016B000FB710840AC490861204610BD00B50246E8
:1016C0000423FFF78AFF034603E0FFF786FF034684
:1016D000521E012B01D1002AF7D102B90523184669
:1016E00000BD10B504244FF43020FFF7E7FF044697
:1016F000042C16D19C48006940F004009A49086106
:101700000846006940F0400008614FF43020FFF7C0
:10171000D5FF04469448006941F6FB7108409249A0
:101720000861204610BD00208F49C96901F00201FF
:1017300009B1012000E00020704730B5A525042440
:10174000FFF7F1FF00B100254FF43020FFF75DFFF8
:101750000446042C3AD185488349886084488860CF
:101760000846006940F0200008610846006940F022
:10177000400008614FF43020FFF747FF0446042C77
:101780001BD17948006941F6DF710840764908614C
:101790000846006940F01000086176480580E002C4
:1017A000FFF733FF0446052C10D06F48006941F65F
:1017B000EF7108406C49086108E0052C06D06A48C2
:1017C000006941F6EF71084067490861204630BD65
:1017D00078B506460C46042500200090E802FFF785
:1017E00014FF0546042D24D15F48006940F0010034
:1017F0005D4908613480E802FFF707FF0546042DC4
:1018000010D1B01C0090200C00990880E802FFF76E
:10181000FCFE05465448006941F6FE7108405249F5
:10182000086106E05048006941F6FE7108404E49E3
:101830000861284678BD70B504460D460426F002BE
:10184000FFF7E3FE0646042E11D14748006940F039
:101850000100454908612580F002FFF7D6FE0646E3
:101860004148006941F6FE7108403F490861304631
:1018700070BD70B505460E460424E002FFF7C5FEB4
:101880000446042C17D139483749886038488860A5
:101890000846006940F0100008612E80E002FFF762
:1018A000B4FE0446052C06D02F48006941F6EF71BE
:1018B00008402D490861204670BD2DE9F0430446DB
:1018C0004FF6FF763746B046B1460425E443E6B20C
:1018D000C4F30727C4F307484FEA1469E802FFF787
:1018E00094FE0546042D49D120481F4988602048B0
:1018F00088600846006940F010000861FF2E06D09D
:101900001C4808300680E802FFF77FFE0546042DDC
:1019100008D1FF2F06D017480A300780E802FFF7EA
:1019200074FE0546042D0AD1B8F1FF0F07D0114807
:101930000C30A0F80080E802FFF767FE0546042D92
:101940000AD1B9F1FF0F07D00A480E30A0F8009075
:10195000E802FFF75AFE0546052D0FD00248006940
:1019600041F6EF71084007E000200240230167457F
:10197000AB89EFCD00F8FF1F664908612846BDE836
:10198000F08330B5054604244FF43020FFF73DFEC8
:101990000446042C41D160485E4988605F488860F5
:1019A0000846006940F0200008610846006940F0E0
:1019B000400008614FF43020FFF727FE0446042C56
:1019C00022D15448006941F6DF710840514908614D
:1019D0000846006940F0100008611DB10020504920
:1019E000088002E0A5204E4908804FF43020FFF720
:1019F0000CFE0446052C10D04648006941F6EF71F4
:101A000008404449086108E0052C06D041480069B7
:101A100041F6DF7108403F490861204630BDF0B50E
:101A200005460E46174604243B483A4988603B4821
:101A30008860E002FFF7E9FD0446042C19D135481F
:101A4000006940F010003349086147F0F800304366
:101A500028433349891C0880E002FFF7D6FD04467D
:101A6000052C06D02B48006941F6EF710840294942
:101A700008612046F0BD2748C069800870472548A6
:101A8000006A704700202349096801F0200109B16C
:101A9000012000E00020704729B11E4A126902436C
:101AA0001C4B1A6104E01B4A12698243194B1A61EC
:101AB000704701460020012908D1164AD26902F078
:101AC00001020AB1012008E0002006E0114AD268B4
:101AD0000A400AB1012000E0002070470D49C860AB
:101AE000704704200B49C96801F0010109B10120C8
:101AF0000EE00849C96801F0040109B1022007E0BD
:101B00000449C96801F0100109B1032000E0042074
:101B1000704700000020024023016745AB89EFCDEC
:101B200000F8FF1F10B50446CC48844208D10121BB
:101B3000042000F0B3FB0021042000F0AFFB46E0DE
:101B4000C748844208D10121082000F0A7FB0021EA
:101B5000082000F0A3FB3AE0C248844208D10121EA
:101B6000102000F09BFB0021102000F097FB2EE0DE
:101B7000BD48844208D10121202000F08FFB0021C4
:101B8000202000F08BFB22E0B848844208D10121DC
:101B9000402000F083FB0021402000F07FFB16E096
:101BA000B348844208D10121802000F077FB002156
:101BB000802000F073FB0AE0AE48844207D1012187
:101BC000801500F06BFB0021A01500F067FB10BD35
:101BD00010B50121084600F061FB0021012000F052
:101BE0005DFB10BD2DE9F0410246002500260020D6
:101BF00000230024002791F803C00CF00F0591F892
:101C000003C00CF0100CBCF1000F03D091F802C01F
:101C10004CEA050591F800C0BCF1000F31D0146802
:101C200000202BE04FF0010C0CFA00F3B1F800C0DB
:101C30000CEA03069E4220D183004FF00F0C0CFAF1
:101C400003F7BC4305FA03FC4CEA040491F803C013
:101C5000BCF1280F06D14FF0010C0CFA00FCC2F8C1
:101C600014C00AE091F803C0BCF1480F05D14FF051
:101C7000010C0CFA00FCC2F810C0401C0828D1D39B
:101C80001460B1F800C0BCF1FF0F34DD54680020CF
:101C90002EE000F1080C4FF0010808FA0CF3B1F83F
:101CA00000C00CEA03069E4221D183004FF00F0CC6
:101CB0000CFA03F7BC4305FA03FC4CEA040491F860
:101CC00003C0BCF1280F05D100F1080C08FA0CF88C
:101CD000C2F8148091F803C0BCF1480F07D100F19D
:101CE000080C4FF0010808FA0CF8C2F81080401CEC
:101CF0000828CED35460BDE8F0814FF6FF71018013
:101D0000022181700421C17070470246002093684F
:101D10000B400BB1012000E00020704701468868AD
:101D200080B2704702460020D3680B400BB10120FF
:101D300000E0002070470146C86880B2704701612A
:101D40007047416170470AB1016100E0416170472D
:101D5000C16070474FF480320A43826181618261C1
:101D600082698269704702460020434B18684FF62B
:101D70008073184040EA021008433F4B18607047D8
:101D80003E49C8617047F0B50A460023002400218F
:101D9000002500F00046B6F1004F02D1364EF16941
:101DA00001E0354E7168C0F3034583B200F440167C
:101DB000B6F5401F08D121F070612F4E766826F0ED
:101DC00070662D4F7E6012E000F48016B6F5801F1D
:101DD00006D1032606FA05F4A14341F0706106E03E
:101DE000460D360103FA06F6B14341F0706122B1A7
:101DF000460D360103FA06F6314300F00046B6F10F
:101E0000004F02D11C4EF16101E01B4E7160F0BD2C
:101E100030B500228B071C0F0F2303FA04F2164B78
:101E200008338C1053F824309343134C08348D102E
:101E300044F8253023468C1053F824308C07240FA7
:101E400000FA04F423430C4C08348D1044F8253078
:101E500030BD0A49DC3108607047000000080140CD
:101E6000000C014000100140001401400018014026
:101E7000001C014000200140000001400000204201
:101E80000E49086070470D49486070470B498860EB
:101E900070474AF6AA200949086070474CF6CC40C2
:101EA00006490860704701460020044AD2680A408B
:101EB0000AB1012000E0002070470000003000401F
:101EC00010B50121080700F0F6F900214FF080500D
:101ED00000F0F1F910BD2A490862704728490861ED
:101EE000704701460020274A106820F0E0000843B0
:101EF000106070472249A0310860704710B5024653
:101F00000020204B186820F00300104318601E4B7F
:101F10001B6843F004031C4C2360012901D130BF2E
:101F200000E020BF184B1B6823F00403164C23600D
:101F300010BD1448006840F00400124908600846CB
:101F4000006840F0020008600F48006840F004009C
:101F50000D49086000BF00BF30BF70470146002038
:101F6000084A52680A400AB1012000E00020704788
:101F70000449096841EA8001024A11607047000083
:101F800000000E420070004010ED00E0DF480068E5
:101F900040F00100DD49086008464068DC4908401F
:101FA000DA49486008460068DA490840D7490860BD
:101FB0000846006820F4802008600846406820F445
:101FC000FE0048604FF41F0088607047CF490968E1
:101FD00021F48031CD4A11601146096821F4802135
:101FE0001160B0F5803F03D0B0F5802F0ED106E030
:101FF000C649096841F48031C44A116007E0C34909
:10200000096841F4A021C14A116000E000BF00BF8F
:10201000704710B501460022002300204A11012A12
:1020200002D1BA4C236806E0022A02D1B74C236AD7
:1020300001E0B64C636A01F01F02012494401C4089
:102040000CB1012000E0002010BD38B50020009048
:102050000024002500BF3120FFF7DBFF0546009874
:10206000401C00900098B0F5A06F01D0002DF2D078
:102070003120FFF7CEFF08B1012400E00024204604
:1020800038BD01460020A14A106820F0F80040EA5F
:10209000C10010607047A0490860704702460020E8
:1020A0009A4B586820F47C1042EA01031843974B7E
:1020B0005860704798490866704701460020934A67
:1020C000506820F003000843506070478F48406814
:1020D00000F00C007047014600208C4A506820F048
:1020E000F00008435060704701460020874A50685E
:1020F00020F4E06008435060704701460020834AA6
:10210000506820F4605040EAC1005060704729B127
:102110007E4A527A02437D4B5A7204E07B4A527ADD
:1021200082437A4B5A7270477B49D83108607047B6
:1021300001460020754A506820F440400843506032
:1021400070470021714A20321170704A82F82010C5
:10215000012802D004280AD104E001216B4A203270
:10216000117005E00521694A2032117000E000BFBE
:1021700000BF70476949086070476449096A0143B4
:10218000624A11627047654944390860704730B54A
:1021900000210022002400235C4D6D6805F00C0135
:1021A00021B1042905D0082923D105E05C4D056043
:1021B00022E05B4D05601FE0544D6D6805F4701220
:1021C000524D6D6805F48034022505EB92421CB92E
:1021D000544D554305600BE04C4D6D6805F40035DA
:1021E0001DB1504D5543056002E04D4D554305600E
:1021F00002E04B4D056000BF00BF444D6D6805F027
:10220000F0010909484D6B5C0568DD4045603F4DB4
:102210006D6805F4E061090A434D6B5C4568DD407B
:1022200085603A4D6D6805F46051C90A3E4D6B5C9E
:102230004568DD40C560354D6D6805F44041890B4A
:102240003A4D6B5CC568B5FBF3F5056130BD29B14E
:102250002E4A526902432D4B5A6104E02B4A5269BF
:1022600082432A4B5A61704729B1284A9269024336
:10227000264B9A6104E0254A92698243234B9A6176
:10228000704729B1214AD2690243204BDA6104E048
:102290001E4AD26982431D4BDA61704729B11B4A3D
:1022A000D2680243194BDA6004E0184AD2688243CC
:1022B000164BDA60704729B1144A12690243134B76
:1022C0001A6104E0114A12698243104B1A61704787
:1022D00012494039086070470F49C86470470B497C
:1022E000C87170470948406A40F0807007494862E9
:1022F000704701460020054A92680A400AB1012051
:1023000000E00020704701498872704700100240C9
:102310000000FFF8FFFFF6FE000042428004424248
:1023200000127A0000093D0098030020A803002055
:1023300029B1504A128802434E4B1A8004E04D4A9C
:10234000128882434B4B1A8070474A48001D008810
:1023500040F010004749091D088070474548001D9E
:1023600000884FF6EF7108404249091D0880704708
:10237000002140481C300188001F008841EA0040CD
:10238000704700B50246FFF7E0FF100C39491831DD
:102390000880091D0A80FFF7E1FF00BD00B5024675
:1023A000FFF7D3FFC2F30340324908310880091D0B
:1023B0000A80FFF7D3FF00BD00B50246FFF7C5FF57
:1023C000100C2C4920310880091D0A80FFF7C6FF38
:1023D00000BD00202749103109880907080B25494D
:1023E000143109880843704700BF2248001D008847
:1023F00000F020000028F8D070471E48001D00881B
:102400004FF6F77108401B49091D088000BF1948A5
:10241000001D008800F008000028F8D07047014631
:102420000020144A121D12880A400AB1012000E05F
:10243000002070470F49091D098881430D4A121D6C
:1024400011807047014600200A4A121D12880A4076
:10245000D0B2084A12880A4012B108B1012000E047
:10246000002070470349091D09888143014A121D54
:10247000118070470028004010B50446FE48844291
:1024800008D10121C014FFF709FF0021E014FFF774
:1024900005FFC4E0B4F1804F08D101210846FFF7E1
:1024A0000AFF00210120FFF706FFB8E0F34884424D
:1024B00008D101210220FFF7FEFE00210220FFF7D4
:1024C000FAFEACE0EE48844208D101210420FFF777
:1024D000F2FE00210420FFF7EEFEA0E0E94884426E
:1024E00008D101210820FFF7E6FE00210820FFF7B0
:1024F000E2FE94E0E448844208D101211020FFF775
:10250000DAFE00211020FFF7D6FE88E0DF48844283
:1025100008D101212020FFF7CEFE00212020FFF767
:10252000CAFE7CE0DA48844208D101214014FFF75A
:10253000B5FE00216014FFF7B1FE70E0D54884427B
:1025400009D10121C804FFF7A9FE00214FF40020A2
:10255000FFF7A4FE63E0D048844209D101210805B9
:10256000FFF79CFE00214FF48010FFF797FE56E026
:10257000CA48844209D101214805FFF78FFE002196
:102580004FF40010FFF78AFE49E0C548844208D1A5
:1025900001214020FFF78FFE00214020FFF78BFE36
:1025A0003DE0C048844208D101218020FFF783FE2E
:1025B00000218020FFF77FFE31E0BB48844208D134
:1025C00001218015FFF777FE0021A015FFF773FEAC
:1025D00025E0B648844209D101210804FFF75EFED8
:1025E00000214FF48030FFF759FE18E0B0488442D4
:1025F00009D101214804FFF751FE00214FF40030BA
:10260000FFF74CFE0BE0AB48844208D1012188045F
:10261000FFF744FE00214FF48020FFF73FFE10BD7E
:1026200000220288944B98420ED0994B98420BD0CE
:10263000B0F1804F08D0914B984205D0904B984212
:1026400002D0904B984204D14FF68F731A404B88BA
:102650001A438D4B984207D08C4B984204D04FF6CA
:10266000FF431A40CB881A4302808B8883850B88EE
:102670000385814B98420BD0854B984208D08B4BF9
:10268000984205D08A4B984202D08A4B984201D199
:102690000B7A038601238382704770B500240022E1
:1026A0000023058C4FF6FE7635400584028C838826
:1026B000048B4FF68F752C40B51E2C400D882C4393
:1026C000751E2A400D892A434D882A436A4DA84227
:1026D0000BD06F4DA84208D0744DA84205D0744D60
:1026E000A84202D0734DA84213D14FF6F7752A4085
:1026F0004D892A434FF6FB752A408D882A434FF6B1
:10270000FF652B404FF6FF552B408D892B43CD891C
:102710002B4383800483CD888586028470BD70B589
:10272000002400220023058C4FF6EF763540058407
:10273000028C8388048B48F6FF752C404FF6FF45CA
:102740002C400D884FF6FF7606EA05252C434FF600
:10275000DF752A400D8906EA05152A434D8806EAE9
:1027600005152A43444DA84202D0494DA8421DD127
:102770004FF67F752A404D894FF6FF7606EA05151C
:102780002A434FF6BF752A408D8806EA05152A436D
:102790004FF6FF352B404FF2FF752B408D8906EA2F
:1027A00085052B43CD8906EA85052B438380048369
:1027B000CD880587028470BD70B5002400220023F7
:1027C000058C4FF6FF6635400584028C8388848B28
:1027D0004FF68F752C404FF6FC752C400D882C431E
:1027E0004FF6FF552A400D894FF6FF7606EA05257C
:1027F0002A434D8806EA05252A431F4DA84202D0E8
:10280000234DA8421DD14FF2FF752A404D894FF646
:10281000FF7606EA05252A434FF6FF352A408D88C4
:1028200006EA05252A434EF6FF752B404DF6FF7547
:102830002B408D8906EA05152B43CD8906EA05153F
:102840002B4383808483CD888587028470BD70B5D7
:10285000002200230024058C4EF6FF7635400584C7
:10286000038C8488828B48F6FF752A404FF6FF451B
:102870002A400D8820E00000002C014000040040A8
:1028800000080040000C0040001000400014004010
:1028900000340140004C0140005001400054014010
:1028A00000180040001C0040002000400040014093
:1028B00000440140004801404FF6FF7606EA052536
:1028C0002A434DF6FF752B400D8906EA05352B434B
:1028D0004D8806EA05352B43FA4DA84202D0FA4D41
:1028E000A84208D14BF6FF752C408D894FF6FF7634
:1028F00006EA85152C4384808283CD88A0F8405059
:10290000038470BD828B4FF2FF331A408283828B27
:102910004FF6FF7303EA01231A4382837047F0B531
:102920000C461546002200210026078C4EF6FF7C3F
:1029300007EA0C070784828B018C4FF6FF7707EAC2
:10294000043640F6FF473A404FF6FF7707EA05277F
:102950003A434FF6FF7707EA03373A43D94FB84275
:102960000ED0D94FB8420BD0B0F1804F08D0D74F1E
:10297000B84205D0D64FB84202D0D64FB84206D1A1
:102980004DF6FF77394046F48057394305E047F666
:10299000FF57394044F48057394382830184F0BDA6
:1029A000828B4FF6F3731A408283828B0A438283B1
:1029B0007047F0B50C461546002200210026078C12
:1029C0004FF6FF6C07EA0C070784828B018C4FF6E9
:1029D000FF7707EA04264FF60C773A404FF6FF7769
:1029E00007EA03172F433A43B64FB8420ED0B64F0B
:1029F000B8420BD0B0F1804F08D0B44FB84205D0E8
:102A0000B34FB84202D0B34FB84206D14FF6FF578A
:102A1000394046F48077394305E04FF2FF5739409B
:102A200044F48077394382830184F0BD028B4FF2F6
:102A3000FF331A400283028B4FF6FF7303EA012330
:102A40001A4302837047F0B50C4615460022002158
:102A50000026078C4FF6EF7C07EA0C070784028BF1
:102A6000018C4FF6FF7707EA041640F6FF473A401D
:102A70004FF6FF7707EA03373A434FF6FF7707EA47
:102A800005273A438F4FB8420ED08F4FB8420BD034
:102A9000B0F1804F08D08D4FB84205D08C4FB8426E
:102AA00002D08C4FB84206D14FF6DF77394046F05E
:102AB0001007394305E04FF65F77394044F01007BF
:102AC000394302830184F0BD028B4FF6F3731A4041
:102AD0000283028B0A4302837047F0B50C46154609
:102AE00000220021068C4FF6FE773E400684028BC2
:102AF000018C4FF60C7632407E1C06EA03162E43FC
:102B00003243704EB0420ED06F4EB0420BD0B0F197
:102B1000804F08D06D4EB04205D06D4EB04202D00D
:102B20006C4EB04206D14FF6FD76314044F00106BE
:102B3000314305E04FF6F576314044F0010631436C
:102B400002830184F0BD70B505460C465D488542A0
:102B50000ED05D4885420BD0B5F1804F08D05B4860
:102B6000854205D05A48854202D05A48854200D154
:102B700000E000BF208850B92389A28861882846D8
:102B8000FFF7ABFFE1882846FFF79EFF25E020888E
:102B900004280AD12389A28861882846FFF753FFB9
:102BA000E1882846FFF742FF17E0208808280AD16D
:102BB0002389A28861882846FFF7FBFEE188284622
:102BC000FFF7EEFE09E02389A28861882846FFF717
:102BD000A6FEE1882846FFF795FE70BD2DE9F0417D
:102BE00005460C4600260127608808B9022600E049
:102BF0000026A088012801D1022700E001272088B3
:102C0000A0B92389A28861882846FFF766FFE1887A
:102C10002846FFF759FF23893A4631462846FFF7F1
:102C200012FFE1882846FFF701FF13E02389A288FD
:102C300061882846FFF707FFE1882846FFF7F6FE80
:102C400023893A4631462846FFF747FFE188284660
:102C5000FFF73AFFBDE8F0810A884B881A438B885A
:102C60001A43CB881A430B891A434B891A438B8921
:102C70001A43A0F8442070474FF6FF71818000216D
:102C80000180C18041800172704700210180418034
:102C90008180C180018141818181C1817047002192
:102CA00001804180012181800021C1800181704724
:102CB0000021018041808180C18001814181818129
:102CC00070470000002C0140003401400004004027
:102CD00000080040000C004021B1028842F00102CF
:102CE000028004E002884FF6FE731A4002807047AB
:102CF00031B1B0F8442042F40042A0F8442005E08D
:102D0000B0F84420C2F30E02A0F8442070471AB174
:102D100083890B43838102E083898B4383817047DE
:102D20008182704741EA0203A0F8483070471AB127
:102D300083890B43838102E083898B4383817047BE
:102D400001894FF6F8721140018170470A4600214F
:102D500001894FF68F73194011430181704730B5D7
:102D600004460D4629462046FFF7F0FF208940F033
:102D70000700208130BD2DE9F04104460D4616467E
:102D80001F46602D06D13B46012231462046FFF703
:102D90005AFE05E03B46012231462046FFF79DFEE4
:102DA00029462046FFF7D2FF208940F00700208106
:102DB000BDE8F08130B50C4600210189C9B24FF65B
:102DC000FF7505EA0325154325432943018130BDDD
:102DD0002DE9F04105460E46174698460024434625
:102DE0003A4631462846FFF7E5FF2C894FF6F87042
:102DF000044044F007044FF68F70044044F0700420
:102E00002C81BDE8F081F0B504460D4616461F46FC
:102E10003B46324629462046FFF7CCFF208940F446
:102E200080402081F0BD0185828270470A460021E2
:102E300001884FF68F731940114301807047F0B538
:102E40000C4615461E460021002200230189028BF4
:102E5000038C4FF6F877394021434FF6FC473A4050
:102E600040F201173A434FF6DD773B404FF6FF77CC
:102E700007EA06172F433B43018102830384F0BD19
:102E80000A460021018B4FF68F73194011430183CD
:102E900070470A460021018B48F6FF7319404FF630
:102EA000FF7303EA02231943018370470A46002196
:102EB000818B4FF68F7319401143818370470A4607
:102EC0000021818B48F6FF7319404FF6FF7303EA28
:102ED000022319438183704721B1028842F08002A6
:102EE000028004E002884FF67F731A400280704728
:102EF00021B1828842F00402828004E082884FF689
:102F0000FB731A408280704721B1828842F0080228
:102F1000828004E082884FF6F7731A4082807047FF
:102F200021B1828842F00102828004E082884FF65B
:102F3000FE731A40828070470A460021018B4FF6CB
:102F4000F77319401143018370470A460021018B32
:102F50004FF2FF7319404FF6FF7303EA0223194340
:102F6000018370470A460021818B4FF6F7731940A1
:102F70001143818370470A460021818B4FF2FF7312
:102F800019404FF6FF7303EA022319438183704708
:102F90000A460021018B4FF6FB7319401143018350
:102FA00070470A460021018B4FF6FF3319404FF658
:102FB000FF7303EA02231943018370470A46002185
:102FC000818B4FF6FB7319401143818370470A468A
:102FD0000021818B4FF6FF3319404FF6FF7303EA50
:102FE00002231943818370470A460021018B4FF663
:102FF0007F7319401143018370470A460021018BFA
:10300000C1F30E014FF6FF7303EA02231943018354
:1030100070470A460021818B4FF67F731940114398
:10302000818370470A460021818BC1F30E014FF660
:10303000FF7303EA02231943818370470A46002184
:10304000018C4FF6FD7319401143018470470A4605
:103050000021018C4FF6F77319401143018470472A
:103060000A460021018C4FF6DF7319404FF6FF73BB
:1030700003EA02131943018470470A460021018CB8
:103080004FF67F7319404FF6FF7303EA021319439B
:10309000018470470A460021018C4FF6FF53194006
:1030A0004FF6FF7303EA02231943018470470A466F
:1030B0000021018C4FF2FF7319404FF6FF7303EAB2
:1030C00002231943018470470A460021018C4DF602
:1030D000FF7319404FF6FF7303EA0233194301846B
:1030E000704730B5002301248C40A3B2048C9C436C
:1030F0000484048C02FA01F5ADB22C43048430BD83
:1031000030B5002304248C40A3B2048C9C43048477
:10311000048C02FA01F5ADB22C43048430BD70B5C5
:103120000346002000241846183001258D40ACB21B
:103130001D8CA5431D8409B1082909D100EB61004C
:10314000056825F0700505600568154305600EE00B
:103150000D1FC5F34E052844056825F4E0450560BC
:1031600005684FF6FF7606EA02263543056070BD16
:1031700021B1028842F00202028004E002884FF688
:10318000FD731A400280704721B1028842F00402A8
:10319000028004E002884FF6FB731A4002807047F9
:1031A00021B1828842F08002828004E082884FF65A
:1031B0007F731A408280704702884FF6F7731A4077
:1031C000028002880A430280704782884FF68F731C
:1031D0001A40828082880A438280704702894FF6B3
:1031E000F8731A40028102890A43028170470289FA
:1031F0004FF67F731A40028102890A4302817047A9
:103200008184704781857047818670470187704748
:1032100081877047A0F84010704702884FF6FF433F
:103220001A40028002880A43028070470146888E55
:1032300070470146088F70470146888F70470146E6
:10324000B1F8400070470146888C70470146088DF0
:10325000704702460020138A0B400BB1012000E0AA
:1032600000207047CA430282704730B502460020F2
:1032700000230024158A05EA0103958905EA010463
:1032800013B10CB1012000E0002030BDCA4302821E
:103290007047000010B50446FB48844209D1012163
:1032A0008803FEF7FBFF00214FF48040FEF7F6FF96
:1032B00032E0F648844209D101214804FEF7FBFFC1
:1032C00000214FF40030FEF7F6FF25E0F04884427D
:1032D00009D101218804FEF7EEFF00214FF4802080
:1032E000FEF7E9FF18E0EB48844209D10121C80448
:1032F000FEF7E1FF00214FF40020FEF7DCFF0BE0BA
:10330000E548844208D101210805FEF7D4FF0021D9
:103310004FF48010FEF7CFFF10BD2DE9F04786B0C7
:1033200005460E460024A24600BFA1460027B089EC
:1033300000B100BF2F462C8A4CF6FF700440F08885
:1033400004432C82AC894EF6F3100440B0883189D6
:103350000843718908430443AC81AC8A4FF6FF40AF
:103360000440B0890443AC8201A8FEF710FFC648B0
:10337000874202D1DDF810A001E0DDF80CA0A88999
:1033800000F4004040B10AEBCA0000EB0A103168BB
:103390004900B0FBF1F807E00AEBCA0000EB0A10A5
:1033A00031688900B0FBF1F86420B8FBF0F004014B
:1033B0002009642101FB1089A88900F4004040B174
:1033C000322000EBC900B0FBF1F000F0070004432D
:1033D00008E0322000EB09106421B0FBF1F000F0AE
:1033E0000F0004432C8106B0BDE8F0874FF416515E
:1033F000016000218180C18001810C214181002177
:103400008181704710B502460020108A4FF2FF03F9
:1034100018400B884C8823438C882343CC88234353
:103420001843108210BD0021018041808180C1803D
:10343000704721B1828942F40052828104E082897E
:103440004DF6FF731A4082817047F0B503460024A1
:1034500000260025002040F66A17B94200D100BFBF
:103460001846C1F3421401F01F06012707FA06F5BA
:10347000012C01D10C3004E0022C01D1103000E00D
:1034800014301AB107682F43076002E00768AF43A2
:103490000760F0BD1AB1838A0B43838202E0838AFE
:1034A0008B4383827047028A4FF6F0731A40028280
:1034B000028A0A430282704782894FF2FF731A40E0
:1034C000828182890A438281704721B1828942F0D8
:1034D0000202828104E082894FF6FD731A408281E4
:1034E0007047028A4FF6DF731A400282028A0A434B
:1034F0000282704721B1028A42F48042028204E0D3
:10350000028A4BF6FF731A4002827047C1F3080229
:103510008280704701468888C0F30800704781891F
:1035200041F0010181817047028BD2B20283028B8C
:1035300042EA012202837047028B02F47F42028337
:10354000028B0A430283704721B1828A42F0200233
:10355000828204E0828A4FF6DF731A4082827047CB
:1035600021B1828A42F01002828204E0828A4FF600
:10357000EF731A408282704721B1828A42F00802BA
:10358000828204E0828A4FF6F7731A408282704783
:1035900021B1828942F40042828103E08289C2F330
:1035A0000E028281704721B1828A42F400628282D7
:1035B00004E0828A4FF2FF731A4082827047828A47
:1035C0004FF6FB731A408282828A0A4382827047D6
:1035D00021B1828A42F00202828204E0828A4FF69E
:1035E000FD731A408282704702460020B1F5007FC9
:1035F00000D100BF13880B400BB1012000E0002078
:10360000704701F40072B2F5007F00D100BFCA43D9
:103610000280704770B50246002400230025002078
:1036200040F66A16B14200D100BFC1F3421501F065
:103630001F03012606FA03F3012D02D196893340B8
:1036400006E0022D02D1168A334001E0968A33400B
:103650000C12012606FA04F41688344013B10CB19A
:10366000012000E0002070BD10B50022002340F6CC
:103670006A14A14200D100BF0A1201249440A3B2EF
:10368000DC43048010BD00000038014000440040CD
:1036900000480040004C00400050004040EA010358
:1036A0009B0703D009E008C9121F08C0042AFAD2F8
:1036B00003E011F8013B00F8013B521EF9D27047BC
:1036C000D2B201E000F8012B491EFBD27047002264
:1036D000F6E710B513460A4604461946FFF7F0FF11
:1036E000204610BDF0B480EA0102D40F4200B2EBD4
:1036F000410F02D20246084611464A0042D0C30D8D
:10370000DDB2C1F3C752AD1A202D35DAC1F316016F
:1037100041F4000204B15242C5F1200602FA06F15A
:103720002A411044B3EBD05F23D0C4B1012DA0EBEC
:10373000C35009DCF0BC4FF0004202EAC352DBB2D6
:1037400000F5000000F04CBB400000F1807000EB81
:10375000C350A0F1807040EAD170490009E04908E7
:1037600041EAC071A0EBC35000F50000400800EB37
:10377000C350F0BC00F02BBB6142012202EB4101BF
:10378000001BF6E7F0BC704781F00041AAE780F02B
:103790000040A7E780EA010210B502F000434000B4
:1037A00022D04A001FD0010E01EB1261C0F3560077
:1037B000C2F3560240F4000042F40002A0FB0220D3
:1037C00000047F39140400D0401C50EA124001D498
:1037D0004000491EC2B20C0604EBD010401C400849
:1037E000802A02D003E0002010BD20F00100002953
:1037F00000DA0020184310BD30B480EA010202F064
:10380000004530F0004221F0004013D090B1C30DCC
:10381000D40DC2F31601C0F31600E41A41F40001FE
:1038200040F400027D34914201D3641C00E0490061
:10383000002C02DA30BC002070474FF40000002357
:10384000914201D3891A034340084FEA4101F7D15D
:1038500051B1914202D14FF0004105E002D24FF048
:10386000010101E06FF0010103EBC450284430BCBA
:1038700000F0ADBA420005D0C0F3C75252429142A7
:1038800001DC0020704700EBC15070472DE9FE4F6E
:10389000804681EA0300C00F0C46009021F00041F1
:1038A00023F00045B8EB0200A94105D2404621466D
:1038B00090461C460B46024623F00040104347D07A
:1038C000270DC7F30A00C3F30A510290401A019072
:1038D00040286BDAC3F3130040F4801B0098924633
:1038E00020B10023D2EB030A63EB0B0B019859467E
:1038F000C0F14002504600F039FA06460D465046E7
:103900005946019A00F051FA10EB08006141002479
:1039100087EA115284EAE7731A4340D0009A62B3EF
:10392000019A012A4FEA075215DC001B61EB0201E4
:103930004FF0004202EA0752CDE90042001C41F577
:10394000801132462B4600F088FA03B0BDE8F08FB4
:1039500040462146F9E7001B61EB0201001C41F5DE
:10396000801300185B412018A2F5001747EB0301F4
:1039700040EAD570B6196D4111E06D084FEA360680
:1039800045EAC0754FEA0752001B61EB0201001CBB
:1039900041F5801149084FEA300000195141324683
:1039A0002B4603B0BDE8F04F00F048BA0098012262
:1039B00040000023D0EB020263EBE0730098214645
:1039C0004FEAE074B8EB000061EB0401E9E783F033
:1039D00000435BE781F0004158E72DE9FE4F81EAA3
:1039E000030404F0004421F0004100944FF0000B68
:1039F00023F0004350EA01045ED052EA03045BD096
:103A0000C3F30A54C1F30A552C44A4F2F3340194CD
:103A1000A0FB0254C1F3130141F48011C3F313035B
:103A200043F4801301FB024400FB034E840A970A0F
:103A300044EA815447EA8357A4FB076802958D0A3C
:103A400005FB07854FEA932C04FB0C542705029DC8
:103A50004FEA065847EA1637B5EB08056EEB070C38
:103A6000870E920E47EA811742EA8312A7FB0201F2
:103A7000B6EB0B0164EB00042B0D43EA0C335E182C
:103A800044EB1C50DA465146E7FB0201C5F3130430
:103A90004FEA0B3343EA14534FEA0432019C43EAE2
:103AA0000603A4F10C040294009CCDE900B400F0DC
:103AB000D4F903B0BDE8F08F00200146F9E72DE905
:103AC000F04D81EA030404F0004B21F00045144658
:103AD0004FF0000A23F0004150EA050220D054EADA
:103AE00001021DD0C5F30A570246C5F31303C1F303
:103AF0001300C1F30A5640F4801543F48013A7EB7A
:103B00000608101BD64608F2FD3873EB050002D3F9
:103B100008F1010801E092185B41B8F1000F03DAE7
:103B200000200146BDE8F08D00204FF480110646CC
:103B300084460EE0171B73EB050705D3121B63EBDE
:103B4000050306434CEA010C49084FEA300092187D
:103B50005B4150EA0107EDD152EA030012D082EA3C
:103B6000040083EA0501084305D0101BAB4106D2CF
:103B70000122002306E000224FF0004302E06FF034
:103B8000010253101AEB06004CEB085110EB0A002F
:103B900041EB0B01BDE8F04D00F050B9C10F80EAD8
:103BA000E0700844CA079623002100F019B9962353
:103BB0000022114600F014B90EB5C10F80EAE07082
:103BC0000844CA07002140F233438DE80E000A463C
:103BD0000B4600F042F903B000BD0EB540F2334190
:103BE00002910021CDE900110A460B4600F035F99B
:103BF00003B000BD00F0004220F00040C10DC0F352
:103C0000160040F400007F2901DA00207047962951
:103C100003DCC1F19601C84001E096398840002AD2
:103C2000F4D04042704720F00040C10DC0F31600B0
:103C300040F400007F2901DA00207047962903DC58
:103C4000C1F19601C8407047963988407047C1F36A
:103C50000A5210B5C1F3130140F2FF3341F4801151
:103C60009A4201DA002010BD40F233439A42A2F298
:103C7000334203DC524200F088F810BD904010BD82
:103C800000F0004230F000400AD0C10D01F5607133
:103C9000C0F3160042EA0151C208400711437047C1
:103CA00000200146704701F0004330B421F000418C
:103CB00050EA010206D00A0DA2F56072C1F31301A9
:103CC000002A02DC30BC00207047440F44EAC104E3
:103CD000C100E01830BC00EBC25000F078B830B53D
:103CE0000B46014600202022012409E021FA02F5BA
:103CF0009D4205D303FA02F5491B04FA02F5284454
:103D0000151EA2F10102F1DC30BD2DE9F05F054680
:103D1000002092469B4688460646814640241BE08A
:103D2000284641464746224600F02FF853465A4659
:103D3000C01A914110D311461846224600F016F8D9
:103D40002D1A67EB01084F4622460120002100F0A2
:103D50000DF817EB00094E41201EA4F10104DFDC31
:103D6000484631462A464346BDE8F09F202A04DBF8
:103D7000203A00FA02F1002070479140C2F120037E
:103D800020FA03F3194390407047202A04DB203ABD
:103D900021FA02F00021704721FA02F3D040C2F16B
:103DA00020029140084319467047202A06DBCB17B2
:103DB000203A41FA02F043EAE07306E041FA02F3E6
:103DC000D040C2F1200291400843194670470029B3
:103DD000A8BF7047401C490008BF20F00100704791
:103DE00010B4B0FA80FC00FA0CF050EA010404BFF1
:103DF00010BC704749B1CCF1200421FA04F411FA47
:103E00000CF118BF012121430843A3EB0C01CB1D8A
:103E10004FEA00614FEA102042BF002010BC7047FB
:103E200000EBC35010440029A4BF10BC7047401CD5
:103E3000490008BF20F0010010BC704710B5141EE7
:103E400073F1000408DA401C41F1000192185B4153
:103E50001A4301D120F0010010BD2DE9F04D92462A
:103E60009B4611B1B1FA81F202E0B0FA80F2203241
:103E70009046FFF77BFF04460F4640EA0A0041EAFE
:103E80000B0153465A46084313D0114653EA01002A
:103E900019D0C8F140025046FFF777FF05460E469D
:103EA000504659464246FFF761FF084305D00120BE
:103EB00004E020463946BDE8F08D0020054346EA7F
:103EC000E0762C4337430A986305E40AA0EB080028
:103ED0000022FD0A44EA47540A3002D50020014678
:103EE000E9E7010510196941DDE908450019694153
:103EF000BDE8F04DA2E770B521F0004303430CD0BC
:103F0000C1F30A550024D5EB040564EB0403D6176E
:103F1000AD1AB34102DB0020014670BD201841EB11
:103F2000025170BDC1F30A52C1F3130140F2FF33D5
:103F300041F480119A4202DA00200146704740F2B3
:103F400033439A42A2F2334202DC5242FFF71DBFD2
:103F5000FFF70CBF30B5041E71F1000404DB4FF015
:103F60000044404264EB0101141E73F1000405DBC0
:103F70001C464FF00043524263EB04038B4208BFE0
:103F8000824230BD30B5041E71F1000404DB4FF0F5
:103F90000044404264EB0101141E73F1000405DB90
:103FA0001C464FF00043524263EB0403994208BFA2
:103FB000904230BD064C074D06E0E06840F001033A
:103FC00094E8070098471034AC42F6D3EFF792F824
:103FD000A8500108C850010870B58C1810F8015B92
:103FE00015F0070301D110F8013B2A1106D110F892
:103FF000012B03E010F8016B01F8016B5B1EF9D196
:104000002B0705D40023521E0DD401F8013BFAE71B
:1040100010F8013BCB1A921C03E013F8015B01F886
:10402000015B521EF9D5A142D8D3002070BD00001B
:1040300070B50029049D02DB44688C4202D84FF021
:10404000FF3070BD01EB81011126046806EB81068B
:10405000A65DD6B144F821200824026804EB81044F
:1040600013550C23026803EB81030424D550084A3E
:10407000036804EB810412681A510068102303EBF3
:10408000810101224254002070BD6FF0010070BD1B
:10409000AC03002030B50146002011224B6807E038
:1040A00000EB80050C6802EB8505645D2CB1401CBB
:1040B0008342F5D84FF0FF3030BD096800EB800433
:1040C00002EB840201238B5430BD70B501680446B5
:1040D000827E80680968012A01EA000101D009B1E5
:1040E00002E009B1012000E00020C8B16169E06888
:1040F0000125884207D3607E18B9616A09B120465C
:104100008847657670BD2169884207D3207E18B93B
:10411000E16909B1204688472576E068401C09E03E
:10412000207E012803D1216A09B12046884700205A
:1041300020766076E06070BD80E80E0003494A6832
:10414000002A02D10860012048607047B0030020B7
:1041500010B5084A04460020106001EB8100800081
:10416000616000F0DBFE206008B1002010BD4FF060
:10417000FF3010BDAC0300202DE9F05F064600259E
:104180004FF00408DFF868904FF00C0A4FF0100B66
:1041900029E005EB85041121306801EB8401415CC5
:1041A00001B30BEB8407C15DE1B108EB8401D9F8E1
:1041B0000020435850F824C0D31A634512DB425004
:1041C00030680AEB8401415811B100EB8400884744
:1041D0000821306801EB8401415C19B1012901D14A
:1041E0000021C1556D1C7068A842D2D8BDE8F09F6F
:1041F000AC0300200FB4054B10B503A9044A029884
:1042000000F046F910BC5DF814FB0000016F0008D7
:10421000B80300202DE9F0414F1E00EBC701044612
:10422000D1E9000115461E4637F006020DD02A4698
:104230003346FFF7D2FB7F1E04EBC703D3E900230D
:10424000FFF724FB37F00602F1D1022F25D0042F0F
:1042500013D0062F18BFBDE8F0812A463346FFF77A
:10426000BCFBD4E90A23FFF711FB2A463346FFF7CC
:10427000B4FBD4E90823FFF709FB2A463346FFF7CE
:10428000ACFBD4E90623FFF701FB2A463346FFF7D0
:10429000A4FBD4E90423FFF7F9FA2A463346FFF7D3
:1042A0009CFBD4E90223FFF7F1FA2A463346FFF7D5
:1042B00094FBD4E90023BDE8F041FFF7E7BA000022
:1042C0000022134610460149FFF7F9BB0000F03FFA
:1042D0000122FFF710BE0022134610461146FFF7D9
:1042E000EEBB02E008C8121F08C1002AFAD17047CD
:1042F0007047002001E001C1121F002AFBD1704766
:104300000149086070470000C40300202DE9FF5FE9
:1043100082B00021DDE90430020DDDF840B0034336
:1043200018D044F61050A2F2FF32424315141198EF
:1043300001281FD0A5EB0B00401C5FEA000A4FF0DC
:1043400000064E4FDFF83891B046504615D5CAF1F9
:10435000000413E0119801244AA3012801D16FEA57
:104360000B010298119AC0E90031C0E9024206B07F
:10437000BDE8F09FCBF10000DFE704460021404A92
:10438000491842EB0450CDE9001012E0E00707D0D5
:1043900032463B4640464946FFF71FFB804689466A
:1043A00032463B4610461946FFF717FB06460F46B6
:1043B0006410002CEAD1DDE90401DDE90023BAF143
:1043C000000F06DAFFF709FB42464B46FFF705FBF5
:1043D00005E0FFF774FB42464B46FFF770FB0446CF
:1043E0000E460022284BFFF7CDFD03D84FF0FF30DB
:1043F000014607E00022254B20463146FFF746FAEA
:10440000FFF790FD102409E0002C0ADB0A220023AC
:10441000FFF77BFC039B30321A55641E50EA010201
:10442000F2D1641C039AC4F111031444119A012AB5
:1044300003D0012208430DD10AE0084304D0002034
:104440004FF0110B119072E7A3EB0B056D1E0DE001
:104450005B4504DD4FF0000205F1010504E003DADD
:104460004FF00002A5F10105002AECD00298119945
:10447000C0E90231C0E9004579E7000000001440BE
:104480000000F03F300000000000F0430000E03F7B
:104490002DE9FF4F95B09B468946064600250FE261
:1044A000252877D100242746F84A0121059400E009
:1044B000044316F8013F203B01FA03F01042F7D104
:1044C00030782A2811D06FF02F033078A0F1300215
:1044D000092A16D8059A44F0020402EB820203EB83
:1044E00042021044761C0590EFE759F8042B059220
:1044F000002A03DA504244F40054059044F00204C8
:10450000761C30782E2816D116F8010F44F00404DA
:104510002A280DD06FF02F023078A0F13003092B3C
:1045200009D807EB870302EB4303C718761CF3E7B0
:1045300059F8047B761C30786C280FD006DC4C28A8
:1045400017D068280DD06A2814D104E0742810D040
:104550007A280FD10DE044F400140AE044F48014EA
:1045600001E044F440147278824202D104F58014D0
:10457000761C761C307866280BD013DC582877D050
:1045800009DC002875D04528F6D04628F4D0472805
:104590001AD19DE118E0632835D0642879D06528C8
:1045A00012D195E1702873D008DC6728F1D0692812
:1045B0006FD06E280DD06F2806D1B5E073282CD0AF
:1045C000752875D0782874D05A46179990476D1C75
:1045D00075E1C4F30250022809D003280DD0D9F8A0
:1045E000001004280DD00D6009F1040967E1D9F825
:1045F0000010EA17C1E90052F6E7D9F800100D8063
:10460000F2E70D70F0E719F8041B8DF80010002098
:104610008DF80100EA46012003E059F804AB4FF0A1
:10462000FF3061074FF0000102D40DE008F10101F5
:104630008846B9420FDA8045F8DB1AF808100029DD
:10464000F4D108E008F1010188468142FADB1AF84A
:1046500008100029F6D105985B46A0EB0807214613
:104660003846179A00F094FA284400EB080507E052
:104670004DE029E10DE01AF8010B5A4617999047D1
:10468000B8F10108F7D25B4621463846179A13E184
:1046900042E00A220092C4F302524FF0000A022ABA
:1046A00008D059F804CB032A4FEAEC710AD00DE088
:1046B00029E02AE009F1070121F00702F2E802C12E
:1046C000914609E00FFA8CFC4FEAEC71042A03D101
:1046D0004FFA8CFC4FEAEC71002907DA0A460021F8
:1046E000DCF1000C61EB02012D2202E0220504D571
:1046F0002B228DF80420012203E0E20701D02022C2
:10470000F7E7904659E00A2102E010220DE010215F
:104710004FF0000A00910BE010224FF0000A44F025
:1047200004040827009203E008224FF0000A0092D8
:10473000C4F30252022A05D059F804CB0021032AFF
:1047400008D009E009F1070121F00702F2E802C1EF
:10475000914605E01FFA8CFC042A01D10CF0FF0CF5
:104760004FF00008220728D5702806D0009B83F060
:10477000100353EA0A0305D00EE040228DF804200E
:10478000012208E05CEA010206D030228DF8042004
:104790008DF8050002229046009B83F0080353EA3F
:1047A0000A030AD15CEA010201D1620705D5302271
:1047B0008DF804204FF001087F1E582804D034A043
:1047C00003900EA802900DE036A0F9E7534660462C
:1047D000009AFFF79AFA84460398825C0298401E7A
:1047E000029002705CEA0100F0D1029806A9081A52
:1047F00000F1200A600702D524F4803400E001278C
:10480000574502DDA7EB0A0000E0002000EB0A019B
:10481000009005984144401A0590E00306D45B4699
:104820002146179A059800F0B3F90544002706E0E1
:1048300001A85A46C05D179990476D1C7F1C4745DB
:10484000F6DBE0030CD55B462146179A059800F08D
:104850009FF9054404E030205A46179990476D1C93
:104860000099481E00900029F5DC08E002980299A2
:104870005A460078491C0291179990476D1CBAF16D
:104880000001AAF1010AF1DC65E10000092801003C
:1048900030313233343536373839616263646566B6
:1048A0000000000030313233343536373839414278
:1048B000434445460000000000F058F90544761CCA
:1048C000307800287FF4ECAD19B02846BDE8F08FB1
:1048D000620700D4062709F1070222F0070CFCE862
:1048E0000223E14603F000485FEA080C02D00FF211
:1048F000702C0DE05FEA045C02D50FF2682C07E033
:104900005FEAC47C02D00FF2602C01E0AFF2700CC1
:104910004FF0FF3823F00043CDF850C065280CD08D
:1049200006DC452809D046281DD047283DD13DE06A
:10493000662818D067287ED138E00021112F01DBCE
:10494000112000E0781CCDE9000106A90EA8FFF7B0
:10495000DDFCDDE90F010E9A03910021009207F1C1
:10496000010A04914DE04FF000400097CDE901109D
:1049700006A90EA8FFF7CAFCDDE90F0203920E9B01
:1049800011990022DDF80CA00093049211B9791C52
:1049900000EB010AB7EB0A0004D4C0F1FF3007F1C5
:1049A000010A0490AAEB0700019044E0012F00DA0D
:1049B00001270021112F01DD112000E03846CDE94B
:1049C000000106A90EA8FFF7A1FCDDE90F010E9A70
:1049D0000391002104910092BA4621070CD4039957
:1049E000514500DA8A46BAF1010F05DD009AAAF1B5
:1049F0000101515C302908D0B84202DA10F1040FED
:104A000006DA0121CDE9011015E0AAF10101E9E77B
:104A1000002805DC049901440491AAEB000102E09E
:104A2000411C514500DD8A460499401A401C019002
:104A30004FF000400290200704D40198504501DB5C
:104A4000CDF8048000208DF84F0002980DF14F073B
:104A5000B0F1004F25D02B200E9002984FF00208A5
:104A600000280CDA404202902D200E9007E00A2127
:104A70000298FFF734F93031029007F8011DB8F1C0
:104A80000001A8F10108F2DC02980028EFD1791E9C
:104A90000E980870307800F0200040F0450007F8CC
:104AA000020D12A8C01B00F107081498007800B18D
:104AB000012000EB0A01019801EBE07105984144E7
:104AC000401A401E0590E00306D45B462146179A23
:104AD000059800F05DF805441498007818B15A461E
:104AE000179990476D1CE00324D55B462146179A21
:104AF000059800F04DF805441CE00498002807DBF9
:104B0000DDE90301884203DD0098405C179901E06C
:104B1000179930205A469047049805F10105401C2A
:104B200004900198401E019004D12E205A461799F6
:104B300090476D1CBAF10001AAF1010ADDDC05E025
:104B400017F8010B5A46179990476D1CB8F10001F0
:104B5000A8F10108F4DC5B462146179A0598ABE6FC
:104B60002D0000002B000000200000002DE9F04186
:104B7000044600251E461746880404D405E039463D
:104B80002020B0476D1C641EF9D52846BDE8F08191
:104B90002DE9F041044600251E469046C80301D584
:104BA000302700E02027880404D505E04146384638
:104BB000B0476D1C641EF9D52846BDE8F0810000A1
:104BC0002DE9F04DC84A002490B0914205DA21F059
:104BD0000043934201D805D120B110B0BDE8F04D9B
:104BE000FFF776BBB1F5801F1BDA53EA000209D04C
:104BF000002911DA0120FFF783FB10B0BDE8F04D6A
